:100000000C94B8500C94E9500C94E9500C94E950BD
:100010000C94E9500C94E9500C94E9500C94E9507C
:100020000C94E9500C94E9500C94E9500C94E9506C
:100030000C94C3740C94E9500D94D1140D941512C2
:100040000C94E9500D946A220C94E9500C94E950F8
:100050000C94E9500C94E9500C94E9500C94436DC5
:100060000C94E9500D9445990C94E9500C94E95086
:100070000C94E9500C94727D0C94E9500C94E95066
:100080000D941B170C94E9500C94E9500C94E95012
:100090000D9401990C94E9500C94E9500C94E9509A
:1000A0000C94E9500C94E9500D94700D0C94E950A7
:1000B0000C94E9500D94650D0C94E9500C94E950A2
:1000C0000C94E9500C94E9500C94E9500D94250DD2
:1000D0000C94E9500C94E9500C94E9500C94E950BC
:1000E0000C94E95000000000000000000000000037
:1000F0000000000000000000000000000000000000
:10010000A55AB44B97308101ADF8656420AA51A679
:10011000130346037C03A803D4031E044B04940476
:10012000C2040E054E0581059305A505B305C60558
:10013000D105DC05F105230647065C067E06A3060D
:10014000AA06BA06CF061A073D077A0784071203E4
:100150008F07950712039A07A307B107BE07CF07BA
:10016000E207EE07FC0707081208240837084808CA
:1001700059086C087B088C089708A108B008BB08D0
:100180001203E108EC08FF080709120313091E090E
:100190002E093A0947095A09690977098509920917
:1001A000A109B009C109D109DF09F209FC09050A51
:1001B000120A240A300A380A3F0A430A480A540A33
:1001C000650A700A760A830A870A920A990AA70AB8
:1001D000AA0AAF0ABF0ACF0AF90A070B110B3B0B99
:1001E0004B0B590B6A0B770B8B0B910B9D0BB00BC9
:1001F000C50B1203C50BD10BE40BF10B050C180C4E
:10020000200C330C430C500C5F0C700C810C8F0CC9
:100210009E0CA90CB40CC20CD00CDE0CF00C020D20
:10022000090D140D1A0D200D2B0D320D390D3E0D3B
:100230007F0DAF0DC10DCA0DD90DEB0D060E2D0EA4
:10024000970EAE0E050F5B0F970FE10F1C104010BD
:100250006510701081108C109B10AC10B710FC1042
:1002600044118B11D7111E126A12B112E5122A1312
:100270005513D8136C148614B314FB1409151B15ED
:100280002A153A1547154F155E156C1576157D150F
:100290008B159615A515B415C415D715E615F215C9
:1002A000FF150B1619162A163B16451653165A1625
:1002B0006F1681169316A616B916CD16DE16E7161A
:1002C00010171A176C177E179017A117AB17BB17CB
:1002D000C317D817DE17E517F017FE170A181D18F1
:1002E000281834183F184B18561868189318001916
:1002F0006B198D191203F719001A091A121A4B1AE1
:100300006A1A721AC61AE81A371B9C1B3C1C741C0A
:10031000D81C1D1D481D731D961D191E461E961EB8
:10032000151F4F1F9B1FD71FED1F1920492073203A
:100330009A20E9204D21BB211203682272227822E3
:10034000852291229822A522AA22B722BE22C32268
:10035000D622FB14E622FA220D231C233123432349
:10036000542367237C238F239A23AA23B823CD23E6
:10037000E023F3230324172428243D244F2464245A
:10038000120379248C249C24B124C124D324E7248F
:10039000F22407251C253125442553256825782579
:1003A0008D259F25B225C525DA25EF25042618269B
:1003B0002D2642265326632678268C26A126B6268D
:1003C000C926D826E926F7262D273E278A279427EF
:1003D00098279B27C42715285A28DC282329652914
:1003E00095291E2A812AD12A192B312BA62BD62BEF
:1003F000132C962C2B2DBE2D3F2E9E2E332F982F57
:100400001C30120325302B30120332303730853048
:100410009230004665686C65722061756667657428
:10042000726574656E2C205A2D4B616C696272691D
:100430006572756E67206572666F726465726C694D
:1004400063682E2E2E004D657368426574742041DA
:100450007573676C65696368206665686C6765734A
:1004600063686C6167656E2E20447275636B2061F2
:1004700062676562726F6368656E2E004865697AAF
:10048000756E67206475726368205369636865726E
:10049000686569747374696D6572206465616B74F5
:1004A0006976696572742E00472D436F6465206913
:1004B00073742066F5722065696E656E20616E64E6
:1004C0006572656E204C6576656C206765736C6936
:1004D00063742E00472D436F646520697374206632
:1004E000F5722065696E656E20616E646572656E79
:1004F000204C6576656C206765736C6963742E208B
:10050000536C6963656E2053696520646173204D87
:100510006F64656C6C2065726E6575742E00472D76
:10052000436F6465206973742066F5722065696E97
:1005300065206E6575657265204669726D776172BA
:1005400065206765736C6963742E00472D436F6483
:1005500065206973742066F5722065696E65206E8A
:100560006575657265204669726D77617265206791
:1005700065736C6963742E20416B7475616C69736B
:10058000696572656E20646965204669726D776180
:1005900072652E00472D436F646520697374206671
:1005A000F5722065696E656E20616E646572656EB8
:1005B00020447275636B6572206765736C69637440
:1005C0002E00472D436F6465206973742066F572B1
:1005D0002065696E656E20616E646572656E20448B
:1005E0007275636B6572206765736C6963742E2026
:1005F000536C6963656E2053696520646173204D97
:100600006F64656C6C2065726E6575742E00447243
:10061000F5636B656E205369652064656E204B6ED3
:100620006F706620756D206469652044F5736520E0
:10063000766F727A756865697A656E20756E64206A
:10064000666F72747A7566616872656E2E004472A8
:10065000F5636B656E205369652064656E204B6E93
:100660006F706620756D206461732046696C616DE2
:10067000656E74207A7520656E746C6164656E2E8B
:1006800000756E64204B6E6F7066206472F5636B4C
:10069000656E0046696C616D656E742065696E6C8F
:1006A0006567656E0046616C7363686520466172BC
:1006B00062650046696C2E206E6963687420676508
:1006C0006C6164656E005765636873656C206F6B61
:1006D000004C61646520466172626500576563681D
:1006E00073656C206572666F6C67726569636821FB
:1006F000005370616E6E726F6C6C6520EF66666E93
:10070000656E20756E642046696C616D656E74203F
:10071000766F6E2048616E6420656E746665726ED9
:10072000656E004B6F6E6E74656E20536965206454
:1007300061732046696C616D656E7420656E746EC0
:1007400065686D656E3F00426974746520616B7405
:1007500075616C6973696572656E2E004E657565AD
:10076000204669726D776172652D205665727369D6
:100770006F6E2076657266F5676261723A00576146
:10078000727465206269732050494E44412D205394
:100790006F6E646520616267656BF5686C742069D3
:1007A00073740057617274656E004B65696E6520E5
:1007B0004265776567756E672E00576172746520B4
:1007C0006175662042656E75747A65722E2E0053CF
:1007D000746162696C6520556D676562756E6773DB
:1007E0002D2074656D706572617475722032312DC3
:1007F00032364320756E64206665737465205374C9
:10080000616E642D20666CE1636865206572666FB9
:10081000726465726C6963682E005A7565727374D0
:100820002058595A204B616C696272696572756E05
:10083000672061757366F56872656E2E00456E748B
:100840006C6164656E205369652065727374206401
:1008500061732046696C616D656E7420756E6420ED
:1008600076657273756368656E205369652065737C
:10087000206E6F63686D616C2E004B6F6E74726FCB
:100880006C6C650044F573656E204469612E0053FD
:100890006F72742E005A656974005344204B617264
:1008A00074650057E1686C65205370726163686518
:1008B0000044F573656E7765636873656C0048572F
:1008C0002045696E7374656C6C756E67656E004C5F
:1008D0006164652046696C616D656E742054657352
:1008E00074004D6F746F72656E20617573004163A3
:1008F000687365206265776567656E0054656D7025
:100900006572617475720050494E4441204B616CB0
:100910002E0052657365742058595A204B616C69DA
:1009200062722E00456E64736368616C7465722038
:1009300053746174757300504944204B616C696253
:1009400072696572756E670042657474204C6576D5
:10095000656C204B6F72722E004D65736842657432
:100960007420417573676C65696368005A204B6138
:100970006C696272696572756E670058595A204BCE
:10098000616C696272696572756E670053656C624D
:1009900073747465737400417373697374656E74F2
:1009A0000054657374652066696C616D656E7400D2
:1009B000416C6C65206C6164656E005A69656865A0
:1009C0006E20536965206461732046696C616D65B2
:1009D0006E7420736F666F727420686572617573D0
:1009E00000556D62656E656E6E656E00457273745E
:1009F000652D53636869636874204B616C2E0041F8
:100A000075737761686C00537461686C626C6563C0
:100A10006865004D4D552D4665686C6572004665EC
:100A2000686C657273746174697374696B00537474
:100A30006174697374696B656E004B616C69627295
:100A4000696572756E67004175746F4C6164656E9F
:100A50002046696C616D656E740046696C616D65F8
:100A60006E74206C6164656E0046696C2E20656E44
:100A7000746C6164656E00496E2044F57365206C8A
:100A80006164656E00496E204D4D55206C61646552
:100A90006E004B65696E65205344204B617274652E
:100AA00000447275636B656E20766F6E2053440050
:100AB000447275636B20666F72747365747A656EC9
:100AC00000447275636B2070617573696572656E41
:100AD00000426572656974207365747A656E004EB4
:100AE00069636874206272656974207365747A65DD
:100AF0006E00566F726865697A656E00416E70614E
:100B00007373656E005A2065696E7374656C6C65ED
:100B10006E00447275636B20776965646572686FF7
:100B20006C656E00496E666F616E7A656967650017
:100B30004173736973742E0045696E6D616C005466
:100B40006F6E004C6175740046696C2E2053656EA3
:100B5000736F720046696C616D656E742D576563C5
:100B60006873656C004475726368666C75737300B6
:100B700054656D706F004D61676E6574204B6F6DCD
:100B8000702E004E2F56005A2D54657374204E72ED
:100B90002E004769747465720045696E7374656CE4
:100BA0006C756E67656E004A61004E65696E004443
:100BB0007275636B2061626272656368656E00C105
:100BC0006265727072F566652044617465690044FF
:100BD0006174656920756E766F6C6C7374E16E6418
:100BE00069672E2054726F747A64656D20666F7227
:100BF0007466616872656E3F0084416B7475616CE8
:100C00006973696572650048617570746D656EF52C
:100C100000576172746520626973204865697A754E
:100C20006E6720756E64204265747420616267652A
:100C30006BF5686C742073696E640057E1686C65CD
:100C40002066696C616D656E743A0053656C627301
:100C50007474657374204F4B0053656C62737474C5
:100C60006573742073746172740041757367657481
:100C700061757363687400447275636B2F486F7499
:100C8000656E64204CF56674657200416368736537
:100C90000041636873656E6CE16E6765004C6F734D
:100CA00065205269656D656E73636865696265008C
:100CB000456E6465206E6963687420676574726F41
:100CC0006666656E00456E64736368616C74657218
:100CD000005665726472616874756E6773666568E4
:100CE0006C657200426574742F4865697A756E6729
:100CF000004E6963687420616E67657363686C6F2A
:100D00007373656E004865697A756E672F54686500
:100D1000726D6973746F72005072F566656E3A0099
:100D200053656C62737474657374204665686C6592
:100D300072210046696C616D656E742D53656E732A
:100D40006F7200447275636B6CF5667465723A007D
:100D5000486F74656E642D4CF5667465723A004B8D
:100D6000616C6962726965726520537461727400A6
:100D700053656C62737474657374204572726F721C
:100D800000416C6C65732072696368746967005018
:100D900072F566652053656E736F72656E005072F2
:100DA000F566652044F57365005072F5666520426E
:100DB000657474005072F56665205A20416368734B
:100DC00065005072F56665205920416368736500BF
:100DD0005072F56665205820416368736500507253
:100DE000F5666520456E64736368616C74657200B6
:100DF0005344204B6172746520656E746665726E33
:100E000074005A7572F5636B004175746F204C6500
:100E1000697374004C65697365004D6F6475730088
:100E2000486F6865204C6569737400537472696B10
:100E300074005761726E656E004F686E6500486F92
:100E400074656E6420626569203238304321204425
:100E5000F573652067657765636873656C742C202E
:100E600067656DE1BD205370657A6966696B617471
:100E7000696F6E20616E67657A6F67656E3F0046C9
:100E8000F5722044F573656E7765636873656C2051
:100E90006C6573656E205369650A70727573612E97
:100EA000696F2F6E6F7A7A6C652D6D6B337300509E
:100EB0004944204B616C69622E20666572746967D3
:100EC00000504944204B616C2E00447275636B20C6
:100ED000706175736965727400447275636B20612B
:100EE00062676562726F6368656E00476577E16887
:100EF0006C74652053707261636865206B6F7069F4
:100F00006572656E3F0044F573656E647572636863
:100F10006D65737365722077656963687420766F99
:100F20006D20472D436F64652061622E0044657219
:100F30002044757263686D657373657220646572B1
:100F400020447275636B657264F57365207765691B
:100F500063687420766F6D20472D436F6465206150
:100F6000622E20426974746520F56265727072F5B4
:100F700066656E205369652064656E2057657274DE
:100F800020696E2064656E2045696E7374656C6CB3
:100F9000756E67656E2E004B65696E2046696C61E3
:100FA0006D656E742067656C6164656E2E004469C2
:100FB00065205A2D4B616C696272696572756E6746
:100FC000206973206E6F6368206E6F7477656E643E
:100FD00069672E20466F6C67656E205369652064D3
:100FE000656D2048616E64627563682C204B61708A
:100FF0006974656C20457273746520536368726907
:101000007474652E00447275636B65722077757217
:101010006465206E6F6368206E69636874206B611D
:101020006C696272696572742E20466F6C67656EBA
:10103000205369652064656D2048616E6462756344
:10104000682C204B61706974656C204572737465FF
:101050002053636872697474652E0053656C627303
:101060007474657374207769726420676573746142
:10107000727465742C20756D205374617274706F76
:10108000736974696F6E207A75206B616C69627226
:10109000696572656E2E00416C74652045696E73DA
:1010A00074656C6C756E67656E20676566756E64D9
:1010B000656E2E205374616E6461726420504944E1
:1010C0002C20452D537465707320752E732E772E4A
:1010D0002077657264656E2067657365747A742E17
:1010E000005761726E756E673A20447275636B6566
:1010F0007274797020756E6420506C6174696E65CD
:101100006E7479702077757264656E2062656964AB
:1011100065206765E16E646572742E005761726EBA
:10112000756E673A20447275636B657274797020CE
:101130007775726465206765E16E646572742E0070
:101140005761726E756E673A20506C6174696E6596
:101150006E747970207775726465206765E16E64DE
:101160006572742E00537461686C626C656368000C
:1011700044726568742073696368206E696368747B
:101180000044726568742073696368004C696E6B13
:101190006572204CF5667465723F00566F72646527
:1011A000726572204CF5667465723F004CF566748A
:1011B0006572746573740058595A204B616C69628A
:1011C00072696572756E6720696E204F72646E7504
:1011D0006E672E2053636872E1676C6175662077D5
:1011E000697264206175746F6D61746973636820DE
:1011F0006B6F72726967696572742E0058595A2054
:101200004B616C696272696572756E6720696E20E8
:101210004F72646E756E672E20582F592041636897
:1012200073656E2073696E642065747761732073D3
:10123000636872E1672E204775742067656D61638E
:101240006874210058595A2D4B616C696272696546
:1012500072756E67206F6B2E20582F592D41636871
:1012600073656E2073696E642073656E6B7265635F
:101270006874207A7565696E616E64657220476C6A
:10128000F5636B77756E736368210058595A2D4B5F
:10129000616C696272696572756E67206265656905
:1012A0006E7472E16368746967742E204B616C2EF2
:1012B000202D50756E6B7420766F726E652072658E
:1012C00063687473206E69636874206572726569FF
:1012D00063686261722E0058595A2D4B616C6962C5
:1012E00072696572756E6720626565696E7472E118
:1012F0006368746967742E20566F72646572652026
:101300004B616C2E2D50756E6B7465206E69636831
:101310007420657272656963686261722E00585943
:101320005A2D4B616C696272696572756E672066D1
:1013300065686C67657363686C6167656E2E204BCA
:10134000616C2E202D50756E6B7420766F726E65F9
:1013500020726563687473206E69636874206572B7
:1013600072656963686261722E0058595A2D4B612B
:101370006C696272696572756E67206665686C6714
:10138000657363686C6167656E2E20566F72646565
:101390007265204B616C2E2D50756E6B7465206EDE
:1013A0006963687420657272656963686261722E30
:1013B0000058595A2D4B616C696272696572756E7D
:1013C00067206665686C67657363686C6167656EE6
:1013D000202D206D65687220696D2048616E646201
:1013E0007563682E0058595A2D4B616C6962726999
:1013F0006572756E67206665686C67657363686C97
:101400006167656E2E20426574742D4B616C696254
:101410007269657270756E6B74206E696368742092
:10142000676566756E64656E2E004C6567656E2037
:101430005369652064617320537461686C626C65E4
:1014400063682061756620646173204865697A620B
:101450006574742E004465722041627374616E6419
:10146000207A7769736368656E20646572205370B3
:1014700069747A65206465722044F5736520756E21
:10148000642064656D204265747420697374206EF5
:101490006F6368206E696368742065696E67657341
:1014A00074656C6C742E20466F6C67656E20536992
:1014B000652064656D2048616E64627563682C20E8
:1014C0004B61706974656C20457273746520536359
:1014D0006872697474652E004C6567656E20536987
:1014E000652065696E20426C61747420506170697A
:1014F000657220756E746572206469652044F573A9
:10150000652077E16872656E6420646572204B61C6
:101510006C696272696572756E67206465722065B8
:10152000727374656E20342050756E6B74652E2056
:10153000447275636B657220736F666F727420619D
:1015400075732D20736368616C74656E2C207765EC
:101550006E6E2064617320506170696572206572DF
:10156000666173737420776972642E0053756368C3
:10157000652042657474204B616C696272696572A2
:1015800070756E6B74004D657373656E2064657263
:10159000205265666572656E7A68EF6865206465DD
:1015A00073204B616C69627269657270756E6B74E1
:1015B000657300456E746665726E656E205369656D
:1015C00020F562657273746568656E6465732046A4
:1015D000696C616D656E7420766F6E206465722033
:1015E00044F573652E204B6C69636B656E207765DF
:1015F0006E6E207361756265722E00537461727431
:10160000706F736974696F6E00447275636B2066E6
:101610006F727467657365747A740050494E444103
:1016200020657277E1726D656E004B616C69627264
:10163000696572756E67204F4B004B616C69627211
:1016400069657265205A0042657474204F4B0042F0
:101650006574742061756677E1726D656E00417521
:101660006677E1726D656E204F4B2E00417566778F
:10167000E1726D656E00476573616D74004C657451
:101680007A74657220447275636B004D4D55204627
:1016900065686C6572004D4D55204C6164656665EA
:1016A000686C6572004D4D55204E65747A666568AC
:1016B0006C6572004D6174657269616C7765636811
:1016C00073656C004C65747A746520447275636B45
:1016D0006665686C657200476573616D7465204668
:1016E00065686C65720046696C2E204DE16E676519
:1016F0006C0054656D70657261747572656E00532F
:10170000656E736F7220496E666F004578747275EE
:1017100064657220496E666F0058595A204B616C9F
:101720002E2044657461696C7300447275636B6547
:1017300072204950204164722E3A00756E62656BCA
:10174000616E6E74004D4D552076657262756E64E3
:10175000656E00446174756D3A00756D2046696C64
:10176000616D656E7420656E746C6164656E007584
:101770006D2046696C616D656E74206C6164656E88
:10178000004B6E6F7066206472F5636B656E207A35
:10179000756D004865697A656E207A756D205363B2
:1017A000686E697474004865697A656E207A756D33
:1017B0002041757377757266004865697A656E2099
:1017C0007A756D20456E746C6164656E004865695C
:1017D0007A656E207A756D204C6164656E00416299
:1017E0006BF5686C656E0046696C616D656E7420A2
:1017F00065787472756469657274206D697420729D
:1018000069636874696765722046617262653F004A
:1018100041757377657266656E004175746F6D61B1
:10182000746973636865732046696C612D206D650A
:101830006E74204C6164656E2069737420616B74F2
:101840006976202C204B6E6F7066206472F5636B96
:10185000656E20756E642046696C616D656E7420DE
:1018600065696E6C6567656E2E2E2E004765736127
:101870006D7465732046696C616D656E74004765B3
:1018800073616D746520447275636B7A6569740069
:1018900046696C616D656E742062656E75747A74EC
:1018A00000447275636B7A6569740044F573652052
:1018B000766F726865697A656E21004645484C45C9
:1018C000523A005920456E746665726E756E6720D7
:1018D000766F6D204D696E004C696E6B73005265BA
:1018E000636874730053636872E1676C61756600C6
:1018F0004C65696368742073636872E167005365BF
:1019000068722073636872E167005B303B305D2072
:1019100050756E6B747665727361747A005A2041EB
:101920006E70617373656E0048696E74656E205BDE
:10193000E46D5D00566F726E65205BE46D5D005274
:101940006563687473205BE46D5D004C696E6B7356
:10195000205BE46D5D0054656D702E2065696E73CB
:1019600074656C6C656E3A0053696E64206C696EC8
:101970006B65722B72656368746572205A2D5363B0
:10198000686C697474656E2067616E7A206F626539
:101990006E3F0058595A204B616C696272696572DA
:1019A000656E3A2044726568656E205369652064EF
:1019B000656E204B6E6F706620626973206465727D
:1019C000206F6265726520416E7363686C61672089
:1019D000657272656963687420776972642E20414C
:1019E0006E7363686C69657373656E642064656E9D
:1019F000204B6E6F7066206472F5636B656E2E000F
:101A00005A204B616C696272696572656E3A204456
:101A1000726568656E205369652064656E204B6E43
:101A20006F70662062697320646572206F626572F0
:101A30006520416E7363686C6167206572726569C9
:101A400063687420776972642E20416E7363686CDA
:101A500069657373656E642064656E204B6E6F708C
:101A600066206472F5636B656E2E0050494E4441EA
:101A70002D4B616C696272696572756E672066656F
:101A8000686C67657363686C6167656E0050494E8A
:101A90004441204B616C696272696572756E6720A2
:101AA00069737420666572746967202B20616B749A
:101AB00069762E204573206B616E6E2061757367A9
:101AC000652D20736368616C74657420776572643A
:101AD000656E20696D204D656EF52045696E7374E5
:101AE000656C6C756E67656E202D3E2050494E44C6
:101AF00041206B616C2E00426577656765205A0056
:101B0000426577656765205900426577656765209E
:101B10005800537461686C626C65636820252E37C9
:101B2000730A5A205665727361747A3A20252B31F4
:101B30002E33666D6D0A2563466F72747365747A11
:101B4000656E0A25635265736574004C6164656E49
:101B500020536965207A75657273742064617320FF
:101B600046696C616D656E742E00416262727563C8
:101B7000680044657220417373697374656E7420E4
:101B8000776972642064696520616B7475656C6C3B
:101B9000656E204B616C696272696572756E677300
:101BA000646174656E206CEF736368656E20756E9A
:101BB0006420766F6E20766F726E6520626567694D
:101BC0006E6E656E2E00566F726865697A656E205E
:101BD0006465722044F573652E2042697474652033
:101BE00077617274656E2E004C6567656E2053696F
:101BF000652046696C2E20696E2064656E204578EC
:101C00007472756465722065696E20756E642064F7
:101C100072F5636B656E205369652064616E6E209A
:101C200064656E204B6E6F70662C756D207A752022
:101C30006C6164656E2E00537465636B656E205332
:101C40006965206461732046696C616D656E7420FE
:101C5000696E2064656E2065727374656E205363CF
:101C6000686C6175636820646572204D4D552E2047
:101C70004472F5636B656E205369652064616E6E16
:101C80002064656E204B6E6F70662C20756D20652C
:101C900073207A75206C6164656E2E004465722035
:101CA000447275636B657220626567696E6E74203D
:101CB0006D69742064656D20447275636B656E2078
:101CC00065696E6572205A69636B7A61636B6C69D2
:101CD0006E69652E2044726568656E2053696520C3
:101CE00064656E204B6E6F70662C206269732053A2
:101CF000696520646965206F7074696D616C652029
:101D000048EF686520657272656963687420686170
:101D100062656E2E20C16265727072F566656E2016
:101D2000536965206469652042696C646572206945
:101D30006D2048616E64627563682E0057E1686CBF
:101D4000656E20536965206469652054656D706512
:101D500072617475722C20646965207A75204968F7
:101D600072656D204D6174657269616C207061737C
:101D700073742E0057E1686C656E205369652065A9
:101D8000696E2046696C616D656E742066F572201F
:101D900045727374652D20536368696368746B6161
:101DA0006C696272696572756E6720617573207502
:101DB0006E642077E1686C656E20536965206573F9
:101DC00020696D204F6E2D53637265656E2D4D65D4
:101DD0006EF5206175732E004A65747A74206B610C
:101DE0006C69627269657265206963682064656EFA
:101DF0002041627374616E64207A776973636865E9
:101E00006E2044F573656E737069747A6520756E23
:101E10006420447275636B626574742E005A2D4B96
:101E2000616C696272696572756E6720656D706656
:101E30006F686C656E2E204A65747A7420617573C4
:101E400066F56872656E3F00456E746665726E6514
:101E50006E205369652064617320537461686C62FD
:101E60006C65636820766F6D204865697A62657479
:101E7000742E004C6965677420537461686C626CE1
:101E8000656368206175662064656D204865697AC0
:101E9000626574743F004C6573656E2053696520FC
:101EA000756E7365722048616E6462756368207533
:101EB0006E64206265686562656E205369652064A2
:101EC00061732050726F626C656D2E20466168727E
:101ED000656E205369652064616E6E206D697420A3
:101EE00064656D20417373697374656E74656E20EB
:101EF000666F72742C20696E64656D20536965206D
:101F000064656E20447275636B6572206E65752022
:101F10007374617274656E2E00416C6C6573206120
:101F20006267657363686C6F7373656E2E205669A4
:101F3000656C20537061BD206265696D20447275C7
:101F4000636B656E2100496D204D656EF5204B6118
:101F50006C696272696572756E67202D3E204173EF
:101F600073697374656E74206BEF6E6E656E2053CB
:101F700069652064656E20417373697374656E745E
:101F8000656E20696D6D6572206E65752073746174
:101F90007274656E2E0057656E6E20536965207AE7
:101FA0007573E1747A6C6963686520537461686C59
:101FB000626C6563686520686162656E2C206B6188
:101FC0006C696272696572656E205369652064652B
:101FD00072656E20566F7265696E2D207374656C24
:101FE0006C756E67656E20756E7465722045696EDE
:101FF0007374656C6C756E67656E202D2048572074
:102000005365747570202D20537461686C626C6523
:102010006368652E005265696E6967656E20536955
:102020006520646173204865697A626574742075FF
:102030006E64206472F5636B656E2053696520647D
:10204000616E6E2064656E204B6E6F70662E005759
:10205000696C6C73742064752064656E206C6574A3
:102060007A74656E20536368726974742077696549
:10207000646572686F6C656E2C20756D2064656E8A
:102080002041627374616E64206E65752065696EAF
:102090007A757374656C6C656E3F00566F72686517
:1020A000697A74656D70657261747572206175739B
:1020B00077E1686C656E2C206469652049687265FB
:1020C0006D204D6174657269616C20656E7473700A
:1020D00072696368742E004973742046696C616D7F
:1020E000656E742067656C6164656E3F004A657457
:1020F0007A74207765726465206963682064696515
:102100002044F573652066F57220504C4120766FAF
:10211000726865697A656E2E00496368207765721A
:102120006465206A65747A7420646965205A204B5E
:10213000616C696272696572756E6720647572633D
:102140006866F56872656E2E005465737464727506
:10215000636B206A65747A7420766F6D20537461A6
:10216000686C626C65636820656E746665726E6526
:102170006E2E005A7565727374205472616E73709E
:102180006F7274736963686572756E67656E2065DA
:102190006E746665726E656E2E00496368207765A1
:1021A000726465206A65747A742064696520585980
:1021B0005A2D4B616C696272696572756E67206435
:1021C0007572636866F56872656E2E204573206BC4
:1021D000616E20626973207A75203234204D696EF9
:1021E0002E64617565726E2E005A756EE1636873B8
:1021F000742066F5687265206963682064656E20E6
:1022000053656C627374746573742064757263686B
:102210002C20756D206469652068E17566696773B7
:1022200074656E2050726F626C656D6520626569C1
:102230006D205A7573616D6D656E626175207A757A
:1022400020F56265727072F566656E2E0048616CED
:102250006C6F2C206963682062696E204968722067
:102260004F726967696E616C205072757361206985
:102270003320447275636B65722E204DEF63687472
:10228000656E205369652C206461737320696368EF
:10229000205369652064757263682064656E20450B
:1022A000696E72696368742D20756E677361626C04
:1022B0006175662066F56872653F0048616C6C6FF9
:1022C0002C206963682062696E20496872204F7211
:1022D0006967696E616C2050727573612069332083
:1022E000447275636B65722E20496368207765724E
:1022F0006465205369652064757263682065696E42
:10230000656E206B75727A656E2045696E726963C1
:102310006874756E67732D2070726F7A65737320A1
:1023200066F56872656E2C206265692064656D20B3
:10233000646965205A2D4163687365206B616C691F
:1023400062726965727420776972642E2044616ECE
:10235000616368206BEF6E6E656E20536965206463
:102360007275636B656E2E00465320416B74696F06
:102370006E00576569742E00462E206175746F6C6F
:102380006164656E0046532E204175736C617566FD
:10239000004D6573736572004CF5667465722D545B
:1023A000656D706F0042657474004CF566746572FB
:1023B00020436865636B004D6F64656C6C0044F589
:1023C0007365005A7566756872207A756D2046537C
:1023D000656E736F72004265776567652053656C43
:1023E000656B746F720045696E7A696568656E2009
:1023F000766F6E2046494E444100576572666520EF
:1024000046696C616D656E74206175730050617210
:102410006B652053656C656B746F720053656C65FA
:102420006B746F72207A7572F5636B666168722ED9
:102430000046F5687265205363686E6974742061A4
:10244000757300536368696562652046696C616DE8
:10245000656E740042657265697465204D657373BD
:10246000657220766F720057E1686C652046696C72
:10247000616D656E7420506C61747A0046696C61A0
:102480006D656E742061757377657266656E004662
:1024900045484C455220544D43004645484C2E205B
:1024A00046696C2E48696C6665004645484C455245
:1024B00020496E7465726E004645484C2E20576167
:1024C0007274652042656E75747A65720042657734
:1024D0006567756E67656E206265656E64656E0022
:1024E0005665726D65696465207363686C656966BD
:1024F000656E005A7566756872207A75722044F5AB
:102500007365005A7566756872207A756D20457816
:10251000747275646572005A7566756872207A7592
:10252000722046494E444100456E746C61646520DA
:102530007A7572205269656D656E732E00456E74F2
:102540006C616465207A75722046494E444100539F
:1025500070616E6E726F6C2E206175736B7570702A
:10256000656C6E005370616E6E726F6C2E206569C3
:102570006E6B757070656C6E00554E42454B414EEA
:102580004E544552204645484C45520046494C4120
:102590004D454E545745434853454C0046494C41E0
:1025A0004D454E54204155534745574F5246454E91
:1025B00000454E544C414445204D414E55454C4CF0
:1025C0000046572D4C4155465A4549544645484CBE
:1025D0004552004D4D5520465720555044415445D5
:1025E000204EB354494700515545554520564F4C50
:1025F0004C00554E47C14C54494745522046494C22
:102600002E504C41545A0046494C2E2042455245CA
:102610004954532047454C4144454E004B4F4D4D86
:10262000554E494B4154494F4E534645484C4552EF
:10263000004D4D55205245414749455254204E4981
:10264000434854004D4D55204D4355204645484C78
:102650004552004D4D552053454C4253545445531B
:1026600054204645484C2E00544D43204B55525A59
:102670005343484C55535300544D4320554E5445F5
:10268000525350414E4E2E4645484C2E00544D4319
:102690002054524549424552205245534554005416
:1026A0004D432054524549424552204645484C45E9
:1026B0005200544D4320C14245524849545A2E4677
:1026C00045484C2E005741524E554E4720544D43DD
:1026D000205A55204845495353005350414E4E52BD
:1026E0004F4C2E205349545A5420464553540053BE
:1026F00050414E4E524F2E205354415254502E466C
:1027000045482E0053454C454B544F522053495495
:102710005A5420464553540053454C454B2E2053A4
:1027200054415254504F534645484C2E004645485C
:102730004C204C4144454E205A554D20455854524A
:102740003A00494E5350495A494552452046494E50
:102750004441004653454E534F52205A552046524D
:10276000C14800524945484D454E532E20534954C7
:102770005A542046455354004653454E534F522019
:102780004E2E2046494C2E46524549004653454E52
:10279000534F52204E2E2041555347454CB353546E
:1027A0000046494E4441204E494348542046494C36
:1027B0002E465245490046494E4441204E2E204166
:1027C000555347454CB353540046696C2E207363F0
:1027D000686E656964656E00417573204D4D5520C6
:1027E000617573776572662E0046696C616D656E02
:1027F00074206CE16474004D4D552D4E6575766501
:1028000072737563683A205374656C6C65206469F3
:10281000652054656D706572612D20747572207726
:102820006965646572206865722E2E2E00536F7282
:102830007469657265204461746569656E004569F7
:102840006E696765204461746569656E207775728D
:102850002D2064656E206E6963687420736F7274D6
:10286000696572742E204D61782E2044617465690B
:10287000656E2070726F205665727A656963686E46
:102880006973203D203130302E00474553544F505E
:1028900050542E0041757300416E0045696E2075DD
:1028A0006E65727761727465746572204665686CD6
:1028B00065722069737420617566676574726574EA
:1028C000656E2E004D3630302046696C616D656E48
:1028D000747765636873656C2E204C6164656E2047
:1028E0005369652065696E206E657565732046695C
:1028F0006C616D656E74206F6465722077657266B9
:10290000656E205369652064617320616C74652075
:102910006175732E00456E746665726E656E205328
:10292000696520646173206175736765776F72668E
:10293000656E652046696C616D656E7420766F6E9C
:102940002064657220566F72646572736569746580
:1029500020646572204D4D552E0046696C616D6591
:102960006E7420756E65727761727465742065721D
:102970006B616E6E742E205374656C6C656E2053A3
:102980006965207369636865722C206461737320C4
:102990006B65696E2046696C616D656E7420676554
:1029A0006C6164656E206973742E20C162657270FB
:1029B00072F566656E20536965206469652053650C
:1029C0006E736F72656E20756E6420646965205643
:1029D00065726B6162656C756E672E00496E746519
:1029E000726E6572204C6175667A65697466656899
:1029F0006C65722E204D4D55207A7572F5636B73A0
:102A000065747A656E206F646572204669726D77B1
:102A100061726520616B7475616C6973696572655B
:102A20006E2E004D4D552046572069737420696EF7
:102A30006B6F6D7061746962656C206D69742044A0
:102A40007275636B65722046572E205570646174F1
:102A500065206175662056657273696F6E20332E2E
:102A6000302E332E004D4D55204669726D776172C0
:102A700065204665686C65722C207365747A656E96
:102A80002053696520646965204D4D55207A757223
:102A9000F5636B2E0044657220616E6765666F7228
:102AA00064657274652046696C616D656E74706CE6
:102AB00061747A2069737420617566206469657336
:102AC0006572204861726477617265206E6963681F
:102AD000742076657266F5676261722E205072F519
:102AE00066656E205369652064656E20472D436FCF
:102AF00064652061756620506CE1747A65206175AB
:102B0000BD657268616C62206465732042657265A0
:102B100069636873202854302D5434292E00446989
:102B20006520416B74696F6E206B616E6E206E69FB
:102B300063687420617573676566F56872742077E1
:102B4000657264656E2C206461732046696C616DEA
:102B5000656E742069737420626572656974732090
:102B600067656C6164656E2E20456E746C6164658A
:102B70006E20536965206573207A75657273742EB3
:102B8000004D4D5520616E74776F72746574206EC0
:102B900069636874206B6F7272656B742E20C162FA
:102BA00065727072F566656E2053696520646965AB
:102BB000205665726B6162656C756E6720756E6418
:102BC0002064696520416E7363686CF57373652ECC
:102BD000004D4D5520616E74776F72746574206E70
:102BE000696368742E20C16265727072F566656EE5
:102BF0002053696520646965205665726B61626562
:102C00006C756E6720756E642064696520416E7313
:102C100063686CF57373652E00576569746572653A
:102C20002044657461696C73206F6E6C696E652EEB
:102C300000446965205370616E6E726F6C6C652024
:102C40006B616E6E20646965205374617274706F7D
:102C5000736974696F6E206E69636874207269634A
:102C6000687469672065727265696368656E2E2095
:102C70005072F566656E205369652C206F6220697D
:102C80007267656E646574776173206465737365DC
:102C90006E204265776567756E6720626C6F636B47
:102CA000696572742E004B616E6E2053656C656BA6
:102CB000746F72206F646572205269656D656E7302
:102CC000636865696265206E696368742062657710
:102CD0006567656E2E0053656C656B746F72206559
:102CE00072726569636874205374617274706F7373
:102CF0002E206E696368742E205072F5662C206F4A
:102D00006220657477617320626C6F636B696572B2
:102D1000742E004C6164656E20696E2064656E20BF
:102D20004578747275646572206665686C67657352
:102D300063686C6167656E2E20C16265727072F5A2
:102D400066652064696520466F726D206465722037
:102D500046696C616D656E74737069747A652E2056
:102D60005665726665696E65722064696520536593
:102D70006E736F726B616C696272696572756E6792
:102D80002C2066616C6C73206572666F726465726C
:102D90006C6963682E0053656C656B746F72206B91
:102DA000616E6E2073696368206E69636874206267
:102DB00065776567656E2C2064612046494E444105
:102DC0002046696C2E2065726B616E6E742068619E
:102DD000742E205374656C6C65207369636865722A
:102DE0002C20646173732073696368206B65696E5E
:102DF0002046696C2E20696D2053656C656B746F7D
:102E00007220626566696E64657420756E64204622
:102E1000494E444120726963687469672066756E23
:102E20006B74696F6E696572742E0044657220461A
:102E300053656E736F722077757264652062656981
:102E40006D204C6164656E20696E2064656E20455E
:102E500078747275646572207A75206672F56820E0
:102E600061757367656CEF73742E205072F566653B
:102E70006E205369652C2064617373206E696368EA
:102E8000747320696D20505446452D5363686C61FE
:102E900075636820666573742D207369747A742075
:102EA000756E64206465722053656E736F72207254
:102EB000696368746967206C696573742E00446582
:102EC00072205269656D656E736368656962656ECF
:102ED0002D206D6F746F722069737420626C6F6344
:102EE0006B696572742E20536963686572737465CB
:102EF0006C6C656E2C206461737320736963682049
:102F0000646965205269656D656E736368656962A1
:102F100065206265776567656E206B616E6E2075F2
:102F20006E6420646965205665726B6162656C75BC
:102F30006E6720F56265727072F566656E2E0046EA
:102F400053656E732E206265696D20456E746C61E9
:102F500064656E206E69636874206162676573637F
:102F600068616C7465742E2053696368657273744C
:102F7000656C6C656E3A2046696C2E2062657765DB
:102F80006762617220756E642053656E736F722084
:102F900066756E6B74696F6E696572743F00446527
:102FA00072204653656E736F72206861742062658B
:102FB000696D204C6164656E206465732046696CA0
:102FC000616D656E7473206E6963687420617573DA
:102FD00067656CEF73742E205374656C6C656E209E
:102FE000536965207369636865722C20646173732B
:102FF000206461732046696C616D656E7420646540
:103000006E2053656E736F722065727265696368B6
:10301000742068617420756E642064657220536545
:103020006E736F722066756E6B74696F6E69657210
:10303000742E0046494E4441206E696368742061D5
:1030400075736765736368616C7465742062656924
:103050006D20456E746C6164656E2E20456E746CD7
:103060006164652046696C2E206D616E75656C6CBF
:103070002E2042657765677420736963682046690E
:103080006C2E3F2046756E6B74696F6E6965727445
:103090002046494E44413F0046494E444120686124
:1030A00074206265696D204C6164656E206465738F
:1030B0002046696C616D656E7473206E6963687417
:1030C0002061757367656CEF73742E205374656CA3
:1030D0006C656E20536965207369636865722C2086
:1030E0006461737320736963682064617320466947
:1030F0006C616D656E74206265776567656E206BC7
:10310000616E6E20756E642046494E44412066759E
:103110006E6B74696F6E696572742E004465616BC5
:103120007469762E004C6164656E00456E746C6146
:103130002E005764682E005A2D4B616C2E20666558
:10314000686C67657363686C672E2053656E736F78
:1031500072206E696368742061757367656CEF73C4
:10316000742E205363686D75747A6967652044F521
:1031700073653F20576172746520617566205265E2
:103180007365742E0053656E73697469766974E1B2
:1031900074004B6C61720000000000000000000031
:1031A000000000000000000000000000000000001F
:1031B000000000000000000000000000000000000F
:1031C00000000000000000000000000000000000FF
:1031D00000000000000000000000000000000000EF
:103600000000536F6D652070726F626C656D206590
:103610006E636F756E74657265642C205A2D6C65CF
:1036200076656C696E6720656E666F72636564208F
:103630002E2E2E0001004D65736820626564206C9B
:103640006576656C696E67206661696C65642E20BD
:103650005072696E742063616E63656C65642E00E0
:10366000020048656174696E672064697361626C09
:103670006564206279207361666574792074696D70
:1036800065722E000300472D636F646520736C69BB
:1036900063656420666F7220612064696666657286
:1036A000656E74206C6576656C2E000400472D6392
:1036B0006F646520736C6963656420666F72206156
:1036C00020646966666572656E74206C6576656CEB
:1036D0002E20506C656173652072652D736C696373
:1036E0006520746865206D6F64656C206167616931
:1036F0006E2E000500472D636F646520736C69634F
:10370000656420666F722061206E65776572206641
:1037100069726D776172652E000600472D636F64D4
:103720006520736C6963656420666F722061206E2A
:1037300065776572206669726D776172652E2050BB
:103740006C6561736520757064617465207468656B
:10375000206669726D776172652E000700472D63E0
:103760006F646520736C6963656420666F722061A5
:1037700020646966666572656E74207072696E7425
:10378000657220747970652E000800472D636F64A0
:103790006520736C6963656420666F7220612064C4
:1037A0006966666572656E74207072696E746572A2
:1037B00020747970652E20506C6561736520726588
:1037C0002D736C69636520746865206D6F64656C2A
:1037D00020616761696E2E00090050726573732065
:1037E000746865206B6E6F6220746F2070726568FC
:1037F000656174206E6F7A7A6C6520616E642063F7
:103800006F6E74696E75652E000A00506C65617389
:103810006520707265737320746865206B6E6F62CB
:1038200020746F20756E6C6F61642066696C616DC9
:10383000656E74000B00616E642070726573732096
:10384000746865206B6E6F62000C00496E73657260
:10385000742066696C616D656E74000D00436F6C59
:103860006F72206E6F7420636F7272656374000EE6
:103870000046696C616D656E74206E6F74206C6FAC
:1038800061646564000F004368616E67656420636E
:103890006F72726563746C790010004C6F616469BB
:1038A0006E6720636F6C6F720011004368616E6712
:1038B00065207375636365737321001200506C6536
:1038C000617365206F70656E2069646C657220613C
:1038D0006E642072656D6F76652066696C616D65DA
:1038E0006E74206D616E75616C6C792E00130057DB
:1038F00061732066696C616D656E7420756E6C6FA6
:103900006164207375636365737366756C3F00143F
:1039100000506C6561736520757067726164652E17
:103920000015004E6577206669726D7761726520BB
:1039300076657273696F6E20617661696C61626C25
:10394000653A00160057616974696E6720666F7288
:103950002050494E44412070726F626520636F6F42
:103960006C696E67001700506C6561736520776144
:1039700069740018004E6F206D6F76652E00190077
:103980005761697420666F7220757365722E2E2ED2
:10399000001A00537461626C6520616D6269656E26
:1039A000742074656D706572617475726520323152
:1039B0002D323643206973206E656564656420612D
:1039C000207269676964207374616E642069732072
:1039D00072657175697265642E001B00506C6561BB
:1039E00073652072756E2058595A2063616C696244
:1039F000726174696F6E2066697273742E001C00A8
:103A0000506C6561736520756E6C6F6164207468BD
:103A1000652066696C616D656E7420666972737489
:103A20002C207468656E20726570656174207468FE
:103A3000697320616374696F6E2E001D00436865B1
:103A4000636B73001E004E6F7A7A6C6520642E00E3
:103A50001F00416C706861626574002000536F72D2
:103A60007400210054696D650022004E6F726D6113
:103A70006C0023005344206361726400240053658A
:103A80006C656374206C616E677561676500250005
:103A90004E6F7A7A6C65206368616E6765002600F8
:103AA00048572053657475700027004C6F61646936
:103AB0006E67205465737400280044697361626CFA
:103AC000652073746570706572730029004D6F76A0
:103AD000652061786973002A0054656D70657261B4
:103AE00074757265002B0050494E44412063616C2F
:103AF0002E002C0052657365742058595A2063615A
:103B00006C6962722E002D0053686F7720656E64B9
:103B10002073746F7073002E005049442063616CF1
:103B20006962726174696F6E002F00426564206C77
:103B30006576656C20636F72726563740030004D4A
:103B400065736820426564204C6576656C696E67B4
:103B500000310043616C696272617465205A003201
:103B60000043616C6962726174652058595A003370
:103B70000053656C667465737400340057697A612C
:103B8000726400350054657374696E672066696CF1
:103B9000616D656E740036004C6F616420416C6C21
:103BA000003700506C656173652070756C6C206F18
:103BB00075742066696C616D656E7420696D6D65E4
:103BC00064696174656C79003800526573657400CE
:103BD000390052656E616D65003A00466972737412
:103BE000206C617965722063616C2E003B00536527
:103BF0006C656374003C00537465656C2073686584
:103C0000657473003D00537570706F7274003E00F0
:103C10004661696C207374617473204D4D55003F8B
:103C2000004661696C2073746174730040005374C2
:103C3000617469737469637300410043616C696204
:103C4000726174696F6E0042004175746F4C6F61F0
:103C5000642066696C616D656E740043004C6F6131
:103C6000642066696C616D656E74004400556E6C0D
:103C70006F61642066696C616D656E740045004C0F
:103C80006F616420746F206E6F7A7A6C65004600F5
:103C90005072656C6F616420746F204D4D55004704
:103CA000004E6F20534420636172640048005072DC
:103CB000696E742066726F6D20534400490052652E
:103CC00073756D65207072696E74004A005061757D
:103CD0007365207072696E74004B005365742052D6
:103CE00065616479004C00536574206E6F742052D6
:103CF00065616479004D0050726568656174004EBD
:103D00000054756E65004F004C6976652061646AE9
:103D1000757374205A00500052657072696E740099
:103D20005100496E666F2073637265656E005200C4
:103D30004173736973740053004F6E6365005400E0
:103D4000536F756E640055004C6F756400560046E5
:103D5000696C2E2073656E736F7200570043686143
:103D60006E67652066696C616D656E74005800460B
:103D70006C6F770059005370656564005A004D619F
:103D8000676E65747320636F6D702E005B004E2F3D
:103D900041005C005A2D70726F6265206E722E00B9
:103DA0005D004D657368005E0053657474696E67ED
:103DB00073005F005965730060004E6F006100532F
:103DC000746F70207072696E74006200436865637E
:103DD0006B696E672066696C6500630046696C6597
:103DE00020696E636F6D706C6574652E006400846D
:103DF000526566726573680065004D61696E0066A4
:103E00000057616974696E6720666F72206E6F7A01
:103E10007A6C6520616E642062656420636F6F6CEC
:103E2000696E6700670053656C6563742066696C32
:103E3000616D656E743A00680053656C66746573F5
:103E400074204F4B00690053656C66746573742071
:103E50007374617274006A005377617070656400F6
:103E60006B0046726F6E742F6C6566742066616EAF
:103E700073006C0041786973006D004178697320AC
:103E80006C656E677468006E004C6F6F73652070B0
:103E9000756C6C6579006F00456E6473746F70208B
:103EA0006E6F7420686974007000456E6473746F7F
:103EB000700071004D6F746F72007200456E647314
:103EC000746F7073007300576972696E6720657252
:103ED000726F720074004265642F48656174657288
:103EE0000075004E6F7420636F6E6E656374656459
:103EF0000076004865617465722F546865726D695B
:103F000073746F72007700506C656173652063682D
:103F100065636B3A00780053656C66746573742052
:103F20006572726F722100790046696C616D656E11
:103F3000742073656E736F72007A005072696E74CC
:103F40002066616E3A007B00486F74656E6420667F
:103F5000616E3A007C0043616C6962726174696EE3
:103F60006720686F6D65007D0053656C66746573CE
:103F700074206661696C6564007E00416C6C20632E
:103F80006F7272656374007F00436865636B696E6E
:103F9000672073656E736F7273008000436865639A
:103FA0006B696E6720686F74656E6400810043689A
:103FB00065636B696E6720626564008200436865B3
:103FC000636B696E67205A206178697300830043D0
:103FD0006865636B696E6720592061786973008436
:103FE00000436865636B696E672058206178697368
:103FF000008500436865636B696E6720656E647356
:10400000746F7073008600436172642072656D6F17
:104010007665640087004261636B008800417574B7
:104020006F20706F77657200890053696C656E74DC
:10403000008A004D6F6465008B00486967682070D6
:104040006F776572008C00537472696374008D0021
:104050005761726E008E004E6F6E65008F00486F64
:1040600074656E64206174203238304321204E6FB5
:104070007A7A6C65206368616E67656420616E643E
:10408000207469676874656E656420746F2073704E
:104090006563733F009000466F722061204E6F7A17
:1040A0007A6C65206368616E676520706C6561730A
:1040B0006520726561640A70727573612E696F2F75
:1040C0006E6F7A7A6C652D6D6B3373009100504979
:1040D000442063616C2E2066696E697368656400B4
:1040E00092005049442063616C2E00930050726925
:1040F0006E74207061757365640094005072696E0F
:10410000742061626F72746564009500436F70790A
:104110002073656C6563746564206C616E6775619E
:1041200067653F0096004E6F7A7A6C65206469611E
:104130006D65746572206469666665727320667267
:104140006F6D2074686520472D636F64652E00973E
:10415000004E6F7A7A6C65206469616D6574657272
:1041600020646966666572732066726F6D2074687C
:104170006520472D636F64652E20506C6561736503
:1041800020636865636B207468652076616C756573
:1041900020696E2073657474696E67732E009800D1
:1041A0005468657265206973206E6F2066696C6162
:1041B0006D656E74206C6F616465642E00990054A7
:1041C00068657265206973207374696C6C20612066
:1041D0006E65656420746F206D616B65205A206385
:1041E000616C6962726174696F6E2E20506C6561DA
:1041F000736520666F6C6C6F7720746865206D61E5
:104200006E75616C2C2063686170746572204669FC
:104210007273742073746570732C20736563746992
:104220006F6E2043616C6962726174696F6E2066A3
:104230006C6F772E009A005072696E7465722068F8
:104240006173206E6F74206265656E2063616C69B6
:10425000627261746564207965742E20506C6561AA
:10426000736520666F6C6C6F7720746865206D6174
:104270006E75616C2C20636861707465722046698C
:104280007273742073746570732C20736563746922
:104290006F6E2043616C6962726174696F6E206633
:1042A0006C6F772E009B0053656C66746573742089
:1042B00077696C6C2062652072756E20746F206364
:1042C000616C6962726174652061636375726174A7
:1042D000652073656E736F726C65737320726568A9
:1042E0006F6D696E672E009C004F6C64207365745F
:1042F00074696E677320666F756E642E2044656600
:1043000061756C74205049442C204573746570733A
:10431000206574632E2077696C6C2062652073655C
:10432000742E009D005761726E696E673A20626F4D
:104330007468207072696E7465722074797065207B
:10434000616E64206D6F74686572626F6172642063
:1043500074797065206368616E6765642E009E00E5
:104360005761726E696E673A207072696E74657219
:104370002074797065206368616E6765642E009FA4
:10438000005761726E696E673A206D6F746865726E
:10439000626F6172642074797065206368616E6712
:1043A00065642E00A000536865657400A1004E6F1F
:1043B00074207370696E6E696E6700A20053706935
:1043C0006E6E696E6700A3004C65667420686F743A
:1043D000656E642066616E3F00A40046726F6E7465
:1043E000207072696E742066616E3F00A5004661A0
:1043F0006E207465737400A60058595A2063616C6E
:104400006962726174696F6E20616C6C2072696799
:1044100068742E20536B65772077696C6C20626519
:1044200020636F72726563746564206175746F6D6B
:1044300061746963616C6C792E00A70058595A2029
:1044400063616C6962726174696F6E20616C6C206B
:1044500072696768742E20582F592061786573201F
:1044600061726520736C696768746C7920736B6521
:104470007765642E20476F6F64206A6F622100A801
:104480000058595A2063616C6962726174696F6E79
:10449000206F6B2E20582F59206178657320617230
:1044A000652070657270656E646963756C61722EEB
:1044B00020436F6E67726174756C6174696F6E739F
:1044C0002100A90058595A2063616C6962726174B5
:1044D000696F6E20636F6D70726F6D697365642EA6
:1044E0002052696768742066726F6E742063616C15
:1044F0006962726174696F6E20706F696E74206E8C
:104500006F7420726561636861626C652E00AA0039
:1045100058595A2063616C6962726174696F6E20C8
:10452000636F6D70726F6D697365642E2046726F74
:104530006E742063616C6962726174696F6E207061
:104540006F696E7473206E6F742072656163686149
:10455000626C652E00AB0058595A2063616C696229
:10456000726174696F6E206661696C65642E205299
:10457000696768742066726F6E742063616C69622B
:10458000726174696F6E20706F696E74206E6F74E3
:1045900020726561636861626C652E00AC005859D9
:1045A0005A2063616C6962726174696F6E20666122
:1045B000696C65642E2046726F6E742063616C694D
:1045C00062726174696F6E20706F696E7473206EB1
:1045D0006F7420726561636861626C652E00AD0066
:1045E00058595A2063616C6962726174696F6E20F8
:1045F0006661696C65642E20506C6561736520632B
:104600006F6E73756C7420746865206D616E756172
:104610006C2E00AE0058595A2063616C6962726159
:1046200074696F6E206661696C65642E20426564F2
:104630002063616C6962726174696F6E20706F696A
:104640006E7420776173206E6F7420666F756E6470
:104650002E00AF00506C6561736520706C616365FE
:1046600020737465656C207368656574206F6E20B7
:10467000686561746265642E00B00044697374619A
:104680006E6365206265747765656E20746970205D
:104690006F6620746865206E6F7A7A6C6520616E33
:1046A0006420746865206265642073757266616356
:1046B0006520686173206E6F74206265656E20737B
:1046C0006574207965742E20506C65617365206671
:1046D0006F6C6C6F7720746865206D616E75616CAE
:1046E0002C2063686170746572204669727374204F
:1046F00073746570732C2073656374696F6E2046E4
:1047000069727374206C617965722063616C69628F
:10471000726174696F6E2E00B100506C6163652028
:1047200061207368656574206F66207061706572C2
:1047300020756E64657220746865206E6F7A7A6C7D
:104740006520647572696E67207468652063616CAA
:104750006962726174696F6E206F66206669727338
:1047600074203420706F696E74732E204966207433
:104770006865206E6F7A7A6C652063617463686522
:1047800073207468652070617065722C20706F777B
:104790006572206F666620746865207072696E7439
:1047A000657220696D6D6564696174656C792E0050
:1047B000B200536561726368696E67206265642048
:1047C00063616C6962726174696F6E20706F696E8B
:1047D0007400B3004D6561737572696E6720726510
:1047E000666572656E636520686569676874206FC9
:1047F000662063616C6962726174696F6E20706FAC
:10480000696E7400B400506C6561736520636C65FB
:10481000616E20746865206E6F7A7A6C6520666FB1
:10482000722063616C6962726174696F6E2E2043DD
:104830006C69636B207768656E20646F6E652E000F
:10484000B5004175746F20686F6D6500B6005265E4
:1048500073756D696E67207072696E7400B7005071
:10486000494E44412048656174696E6700B8004351
:10487000616C6962726174696F6E20646F6E65004D
:10488000B90043616C6962726174696E67205A0095
:10489000BA0042656420646F6E6500BB00426564C7
:1048A0002048656174696E6700BC00486561746981
:1048B0006E6720646F6E652E00BD00486561746987
:1048C0006E6700BE00546F74616C00BF004C617372
:1048D00074207072696E7400C0004D4D5520666181
:1048E000696C7300C1004D4D55206C6F616420668A
:1048F00061696C7300C2004D4D5520706F77657211
:10490000206661696C7300C3004D617465726961F2
:104910006C206368616E67657300C4004C617374DA
:10492000207072696E74206661696C7572657300BF
:10493000C500546F74616C206661696C7572657333
:1049400000C60046696C2E2072756E6F7574730018
:10495000C70054656D70657261747572657300C8C7
:104960000053656E736F7220696E666F00C90045F3
:104970007874727564657220696E666F00CA00583B
:10498000595A2063616C2E2064657461696C7300F0
:10499000CB005072696E7465722049502041646486
:1049A000723A00CC00756E6B6E6F776E00CD004D65
:1049B0004D5520636F6E6E656374656400CE004470
:1049C0006174653A00CF00746F20756E6C6F61641E
:1049D0002066696C616D656E7400D000746F206C28
:1049E0006F61642066696C616D656E7400D1005002
:1049F0007265737320746865206B6E6F6200D200FD
:104A000050726568656174696E6720746F206375A4
:104A10007400D30050726568656174696E672074B4
:104A20006F20656A65637400D400507265686561C3
:104A300074696E6720746F20756E6C6F616400D549
:104A40000050726568656174696E6720746F206CD0
:104A50006F616400D600436F6F6C646F776E00D730
:104A60000046696C616D656E74206578747275645A
:104A7000696E672026207769746820636F7272659B
:104A8000637420636F6C6F723F00D800456A656382
:104A90007400D9004175746F6C6F6164696E672032
:104AA00066696C616D656E742069732061637469F9
:104AB00076652C206A757374207072657373207428
:104AC0006865206B6E6F6220616E6420696E73652D
:104AD00072742066696C616D656E742E2E2E00DA1C
:104AE00000546F74616C2066696C616D656E740052
:104AF000DB00546F74616C207072696E742074698D
:104B00006D6500DC0046696C616D656E74207573BF
:104B1000656400DD005072696E742074696D650013
:104B2000DE005072656865617420746865206E6F80
:104B30007A7A6C652100DF004552524F523A00E00C
:104B400000592064697374616E63652066726F6DCD
:104B5000206D696E00E1004C65667400E2005269E8
:104B600067687400E3004D65617375726564207356
:104B70006B657700E400536C6967687420736B653C
:104B80007700E50053657665726520736B65770085
:104B9000E6005B303B305D20706F696E74206F669D
:104BA0006673657400E70041646A757374696E67C3
:104BB000205A00E800526561722073696465205BC9
:104BC000E46D5D00E90046726F6E74207369646580
:104BD0005BE46D5D00EA0052696768742073696484
:104BE000655BE46D5D00EB004C6566742073696481
:104BF00065205BE46D5D00EC005365742074656DA9
:104C000070657261747572653A00ED0041726520DD
:104C10006C65667420616E64207269676874205ADE
:104C20002D63617272696167657320616C6C2075B8
:104C3000703F00EE0043616C6962726174696E6777
:104C40002058595A2E20526F74617465207468651B
:104C5000206B6E6F6220746F206D6F7665207468B4
:104C600065205A20636172726961676520757020E2
:104C7000746F2074686520656E642073746F707043
:104C80006572732E20436C69636B207768656E20B4
:104C9000646F6E652E00EF0043616C69627261742F
:104CA000696E67205A2E20526F7461746520746893
:104CB00065206B6E6F6220746F206D6F7665207457
:104CC0006865205A2063617272696167652075703A
:104CD00020746F2074686520656E642073746F7033
:104CE000706572732E20436C69636B207768656E04
:104CF00020646F6E652E00F00050494E44412063E1
:104D0000616C6962726174696F6E206661696C655D
:104D10006400F10050494E44412063616C69627245
:104D20006174696F6E2069732066696E6973686566
:104D30006420616E64206163746976652E20497415
:104D40002063616E2062652064697361626C6564D2
:104D500020696E206D656E752053657474696E6789
:104D6000732D3E50494E44412063616C2E00F20089
:104D7000457874727564657200F3004D6F76652036
:104D80005A00F4004D6F7665205900F5004D6F769E
:104D900065205800F600536865657420252E37732A
:104DA0000A5A206F66667365743A20252B312E33BC
:104DB000666D6D0A2563436F6E74696E75650A25AD
:104DC00063526573657400F700506C65617365200C
:104DD0006C6F61642066696C616D656E74206669D4
:104DE0007273742E00F80043616E63656C00F90005
:104DF00052756E6E696E672057697A6172642077AA
:104E0000696C6C2064656C6574652063757272658D
:104E10006E742063616C6962726174696F6E207276
:104E20006573756C747320616E6420737461727441
:104E30002066726F6D2074686520626567696E6EAA
:104E4000696E672E00FA0050726568656174696E5C
:104E500067206E6F7A7A6C652E20506C6561736581
:104E600020776169742E00FB00506C6561736520CA
:104E7000696E736572742066696C616D656E74200D
:104E8000696E746F207468652065787472756465E6
:104E9000722C207468656E2070726573732074685C
:104EA00065206B6E6F6220746F206C6F6164206987
:104EB000742E00FC00506C6561736520696E73652B
:104EC00072742066696C616D656E7420696E746FB2
:104ED0002074686520666972737420747562652039
:104EE0006F6620746865204D4D552C207468656E82
:104EF00020707265737320746865206B6E6F62201A
:104F0000746F206C6F61642069742E00FD0054681A
:104F100065207072696E7465722077696C6C20739D
:104F200074617274207072696E74696E672061209A
:104F30007A69672D7A6167206C696E652E20526FE1
:104F40007461746520746865206B6E6F6220756E85
:104F500074696C20796F752072656163682074686C
:104F600065206F7074696D616C206865696768742D
:104F70002E20436865636B207468652070696374D4
:104F80007572657320696E207468652068616E644F
:104F9000626F6F6B202843616C6962726174696F24
:104FA0006E2063686170746572292E00FE0053657F
:104FB0006C6563742074656D70657261747572657B
:104FC000207768696368206D617463686573207910
:104FD0006F7572206D6174657269616C2E00FF00DF
:104FE00053656C65637420612066696C616D656EE4
:104FF0007420666F7220746865204669727374202D
:105000004C617965722043616C6962726174696F89
:105010006E20616E642073656C6563742069742012
:10502000696E20746865206F6E2D73637265656E9E
:10503000206D656E752E0000014E6F772049207738
:10504000696C6C2063616C6962726174652064696B
:105050007374616E6365206265747765656E207434
:105060006970206F6620746865206E6F7A7A6C654F
:1050700020616E6420686561746265642073757276
:10508000666163652E0001015A2063616C6962727A
:105090006174696F6E207265636F6D6D656E6465B6
:1050A000642E2052756E206974206E6F773F000267
:1050B00001506C656173652072656D6F7665207354
:1050C0007465656C2073686565742066726F6D2009
:1050D000686561746265642E00030149732073740E
:1050E00065656C207368656574206F6E2068656106
:1050F000746265643F000401506C656173652063F0
:105100006865636B206F75722068616E64626F6F93
:105110006B20616E64206669782074686520707207
:105120006F626C656D2E205468656E2072657375B4
:105130006D65207468652057697A617264206279B0
:10514000207265626F6F74696E6720746865207085
:1051500072696E7465722E000501416C6C20697372
:1051600020646F6E652E20486170707920707269BE
:105170006E74696E6721000601596F752063616E58
:1051800020616C7761797320726573756D65207429
:1051900068652057697A6172642066726F6D20437A
:1051A000616C6962726174696F6E202D3E2057696F
:1051B0007A6172642E000701496620796F75206854
:1051C000617665206164646974696F6E616C2073D7
:1051D0007465656C207368656574732C2063616CFD
:1051E00069627261746520746865697220707265A5
:1051F0007365747320696E2053657474696E677388
:10520000202D204857205365747570202D2053742D
:1052100065656C207368656574732E000801506CB9
:105220006561736520636C65616E20686561746299
:10523000656420616E64207468656E2070726573A9
:105240007320746865206B6E6F622E000901446FD5
:1052500020796F752077616E7420746F207265708D
:10526000656174206C617374207374657020746F51
:1052700020726561646A7573742064697374616E09
:105280006365206265747765656E206E6F7A7A6CEF
:105290006520616E6420686561746265643F000A20
:1052A0000153656C656374206E6F7A7A6C6520704B
:1052B0007265686561742074656D7065726174757E
:1052C0007265207768696368206D617463686573CF
:1052D00020796F7572206D6174657269616C2E0042
:1052E0000B0149732066696C616D656E74206C6F8B
:1052F000616465643F000C014E6F77204920776937
:105300006C6C2070726568656174206E6F7A7A6C5F
:105310006520666F7220504C412E000D01492077A8
:10532000696C6C2072756E207A2063616C696272A0
:105330006174696F6E206E6F772E000E014E6F776D
:105340002072656D6F76652074686520746573746E
:10535000207072696E742066726F6D20737465655B
:105360006C2073686565742E000F01506C65617365
:10537000652072656D6F7665207368697070696EFF
:10538000672068656C706572732066697273742E2D
:10539000001001492077696C6C2072756E20787955
:1053A0007A2063616C6962726174696F6E206E6FDE
:1053B000772E2049742077696C6C2074616B6520AE
:1053C000757020746F203234206D696E732E001159
:1053D0000146697273742C20492077696C6C2072C5
:1053E000756E207468652073656C667465737420CF
:1053F000746F20636865636B206D6F737420636FD7
:105400006D6D6F6E20617373656D626C7920707263
:105410006F626C656D732E00120148692C20492063
:10542000616D20796F7572204F726967696E616C6A
:10543000205072757361206933207072696E7465D3
:10544000722E20576F756C6420796F75206C696BB4
:1054500065206D6520746F20677569646520796FBC
:1054600075207468726F756768207468652073654D
:105470007475702070726F636573733F0013014819
:10548000692C204920616D20796F7572204F7269F7
:1054900067696E616C20507275736120693320708A
:1054A00072696E7465722E20492077696C6C206772
:1054B0007569646520796F75207468726F756768A7
:1054C00020612073686F727420736574757020702A
:1054D000726F636573732C20696E207768696368E7
:1054E00020746865205A2D617869732077696C6C27
:1054F0002062652063616C696272617465642E204C
:105500005468656E2C20796F752077696C6C206209
:105510006520726561647920746F207072696E74A1
:105520002E0014015061757365001501465320412A
:105530006374696F6E001601436F6E742E0017015D
:10554000462E206175746F6C6F6164001801462EE1
:105550002072756E6F7574001901437574746572ED
:10556000001A0146616E207370656564001B01427C
:105570006564001C0146616E7320636865636B009F
:105580001D014D6F64656C001E014E6F7A7A6C656B
:10559000001F0146656564696E6720746F2046537D
:1055A000656E736F720020014D6F76696E672073B0
:1055B000656C6563746F72002101486F6D696E6779
:1055C000002201526574726163742066726F6D20EF
:1055D00046494E4441002301456A656374696E671C
:1055E0002066696C616D656E740024015061726B98
:1055F000696E672073656C6563746F720025015274
:10560000657475726E696E672073656C6563746F1F
:1056100072002601506572666F726D696E67206355
:10562000757400270150757368696E672066696C30
:10563000616D656E74002801507265706172696EEB
:105640006720626C61646500290153656C65637451
:10565000696E672066696C2E20736C6F74002A0176
:10566000556E6C6F6164696E672066696C616D650B
:105670006E74002B0145525220544D4320666169DF
:105680006C6564002C014552522048656C702066A0
:10569000696C616D656E74002D0145525220496E32
:1056A0007465726E616C002E01455252205761691B
:1056B0007420666F722055736572002F0146696E03
:1056C000697368696E67206D6F76656D656E74735A
:1056D00000300141766F6964696E67206772696E98
:1056E0006400310146656564696E6720746F206EE1
:1056F0006F7A7A6C6500320146656564696E672071
:10570000746F206578747275646572003301466544
:105710006564696E6720746F2046494E44410034C9
:1057200001556E6C6F6164696E6720746F207075CF
:105730006C6C6579003501556E6C6F6164696E67DC
:1057400020746F2046494E44410036014469736518
:105750006E676167696E672069646C657200370106
:10576000456E676167696E672069646C65720038B1
:10577000014F4B003901554E4B4E4F574E2045526D
:10578000524F52003A0146494C414D454E54204338
:1057900048414E4745003B0146494C414D454E541A
:1057A00020454A4543544544003C01554E4C4F4129
:1057B00044204D414E55414C4C59003D0146572027
:1057C00052554E54494D45204552524F52003E01CC
:1057D0004D4D5520465720555044415445204E4587
:1057E00045444544003F0151554555452046554CDB
:1057F0004C004001494E56414C494420544F4F4CB7
:1058000000410146494C2E20414C5245414459200B
:105810004C4F41444544004201434F4D4D554E4984
:10582000434154494F4E204552524F520043014D7F
:105830004D55204E4F5420524553504F4E44494EE3
:10584000470044014D4D55204D4355204552524F80
:10585000520045014D4D552053454C465445535437
:10586000204641494C4544004601544D4320445292
:10587000495645522053484F52544544004701541D
:105880004D4320554E444552564F4C5441474520B8
:10589000455252004801544D432044524956455206
:1058A000205245534554004901544D432044524928
:1058B000564552204552524F52004A01544D432002
:1058C0004F56455248454154204552524F52004B85
:1058D000015741524E494E4720544D4320544F4F9B
:1058E00020484F54004C0149444C45522043414EFE
:1058F0004E4F54204D4F5645004D0149444C4552A2
:105900002043414E4E4F5420484F4D45004E0153C9
:10591000454C4543544F522043414E4E4F54204D29
:105920004F5645004F0153454C4543544F52204379
:10593000414E4E4F5420484F4D450050014C4F4171
:105940004420544F20455854522E204641494C453E
:1059500044005101494E53504543542046494E445A
:10596000410052014653454E534F5220544F4F2051
:105970004541524C5900530150554C4C4559204318
:10598000414E4E4F54204D4F56450054014653450D
:105990004E534F522046494C2E20535455434B00F2
:1059A00055014653454E534F52204449444E5420CE
:1059B00054524947472E00560146494E444120461D
:1059C000494C414D2E20535455434B0057014649F5
:1059D0004E4441204449444E54205452494747457F
:1059E000520058014375742066696C616D656E7470
:1059F000005901456A6563742066726F6D204D4DD4
:105A000055005A014C6F6164696E672066696C616C
:105A10006D656E74005B014D4D5520526574727951
:105A20003A20526573746F72696E672074656D7089
:105A3000657261747572652E2E2E005C01536F7253
:105A400074696E672066696C6573005D01536F6DE4
:105A5000652066696C65732077696C6C206E6F7465
:105A600020626520736F727465642E204D61782EFC
:105A7000204E6F2E206F662066696C657320696EFC
:105A8000203120666F6C64657220666F7220736FC0
:105A90007274696E67206973203130302E005E01A8
:105AA00053544F505045442E005F014F66660060CE
:105AB000014F6E006101556E6578706563746564B1
:105AC000206572726F72206F636375727265642EE7
:105AD0000062014D3630302046696C616D656E7430
:105AE000204368616E67652E204C6F6164206120E1
:105AF0006E65772066696C616D656E74206F7220CB
:105B0000656A65637420746865206F6C64206F6ECD
:105B1000652E00630152656D6F766520746865209F
:105B2000656A65637465642066696C616D656E7431
:105B30002066726F6D207468652066726F6E7420C7
:105B40006F6620746865204D4D552E0064014669CE
:105B50006C616D656E742064657465637465642042
:105B6000756E65787065637465646C792E20456E1A
:105B700073757265206E6F2066696C616D656E74F9
:105B8000206973206C6F616465642E2043686563CF
:105B90006B207468652073656E736F727320616E1D
:105BA0006420776972696E672E006501496E7465BD
:105BB000726E616C2072756E74696D6520657272AB
:105BC0006F722E2054727920726573657474696ED9
:105BD0006720746865204D4D55206F722075706484
:105BE0006174696E6720746865206669726D77619B
:105BF00072652E0066014D4D552046572076657220
:105C000073696F6E20697320696E636F6D70617464
:105C100069626C652077697468207072696E74655A
:105C2000722046572E55706461746520746F20761B
:105C3000657273696F6E20332E302E332E0067012C
:105C40004D4D55204669726D7761726520696E749D
:105C500065726E616C206572726F722C20706C655B
:105C600061736520726573657420746865204D4D9D
:105C7000552E006801526571756573746564206600
:105C8000696C616D656E7420746F6F6C2069732030
:105C90006E6F7420617661696C61626C65206F6EF5
:105CA00020746869732068617264776172652E2060
:105CB000436865636B2074686520472D636F646576
:105CC00020666F7220746F6F6C20696E6465782037
:105CD0006F7574206F662072616E6765202854307E
:105CE0002D5434292E00690143616E6E6F7420704B
:105CF0006572666F726D2074686520616374696F88
:105D00006E2C2066696C616D656E7420697320610C
:105D10006C7265616479206C6F616465642E2055D6
:105D20006E6C6F61642069742066697273742E00F2
:105D30006A014D4D55206E6F7420726573706F6EE1
:105D400064696E6720636F72726563746C792E206C
:105D5000436865636B2074686520776972696E6754
:105D600020616E6420636F6E6E6563746F72732E54
:105D7000006B014D4D55206E6F7420726573706F0E
:105D80006E64696E672E20436865636B2074686576
:105D900020776972696E6720616E6420636F6E6E32
:105DA0006563746F72732E006C014D6F72652064B1
:105DB000657461696C73206F6E6C696E652E006D21
:105DC000015468652049646C65722063616E6E6F72
:105DD0007420686F6D652070726F7065726C792EBB
:105DE00020436865636B20666F7220616E7974680A
:105DF000696E6720626C6F636B696E67206974738C
:105E0000206D6F76656D656E742E006E0143616E58
:105E10002774206D6F76652053656C6563746F72AF
:105E2000206F722049646C65722E006F01546865A2
:105E30002053656C6563746F722063616E6E6F745E
:105E400020686F6D652070726F7065726C792E209E
:105E5000436865636B20666F7220616E7974686950
:105E60006E6720626C6F636B696E67206974732064
:105E70006D6F76656D656E742E0070014C6F616498
:105E8000696E6720746F206578747275646572201E
:105E90006661696C65642E20496E73706563742059
:105EA0007468652066696C616D656E7420746970D4
:105EB0002073686170652E20526566696E65207476
:105EC00068652073656E736F722063616C696272BE
:105ED0006174696F6E2C206966206E656564656407
:105EE0002E00710153656C6563746F722063616E7F
:105EF0002774206D6F76652064756520746F204669
:105F0000494E444120646574656374696E6720611D
:105F10002066696C616D656E742E204D616B652025
:105F200073757265206E6F2066696C616D656E7445
:105F300020697320696E2053656C6563746F7220ED
:105F4000616E642046494E444120776F726B732026
:105F500070726F7065726C792E00720146696C61A7
:105F60006D656E742073656E736F722074726967ED
:105F7000676572656420746F6F206561726C79204B
:105F80007768696C65206C6F6164696E6720746FF7
:105F90002065787472756465722E20436865636B42
:105FA0002074686572652069736E277420616E794C
:105FB0007468696E6720737475636B20696E205016
:105FC00054464520747562652E20436865636B20D6
:105FD000746861742073656E736F7220726561649A
:105FE000732070726F7065726C792E00730150753A
:105FF0006C6C6579206D6F746F72207374616C6C5A
:1060000065642E20456E7375726520746865207016
:10601000756C6C65792063616E206D6F76652061AB
:106020006E6420636865636B2074686520776972AD
:10603000696E672E00740146696C616D656E74202F
:1060400073656E736F72206469646E277420737752
:1060500069746368206F6666207768696C6520756F
:106060006E6C6F6164696E672066696C616D656EE8
:10607000742E20456E737572652066696C616D655E
:106080006E742063616E206D6F766520616E642092
:106090007468652073656E736F7220776F726B73AF
:1060A0002E00750146696C616D656E742073656EB6
:1060B000736F72206469646E2774207472696767F5
:1060C0006572207768696C65206C6F6164696E67C2
:1060D000207468652066696C616D656E742E20455C
:1060E0006E73757265207468652073656E736F7268
:1060F0002069732063616C696272617465642061F8
:106100006E64207468652066696C616D656E7420CC
:10611000726561636865642069742E007601464982
:106120004E4441206469646E2774207377697463F8
:1061300068206F6666207768696C6520756E6C6F85
:106140006164696E672066696C616D656E742E208E
:1061500054727920756E6C6F6164696E67206D6131
:106160006E75616C6C792E20456E73757265206654
:10617000696C616D656E742063616E206D6F76650C
:1061800020616E642046494E444120776F726B73E4
:106190002E00770146494E4441206469646E27749D
:1061A0002074726967676572207768696C65206C16
:1061B0006F6164696E67207468652066696C616DE3
:1061C000656E742E20456E73757265207468652047
:1061D00066696C616D656E742063616E206D6F76AB
:1061E0006520616E642046494E444120776F726B92
:1061F000732E00780144697361626C650079015304
:10620000746F70007A014C6F6164007B01556E6C95
:106210006F6164007C0152657365744D4D55007D5E
:10622000015265747279007E01426564206C657666
:10623000656C696E67206661696C65642E205365C4
:106240006E736F72206469646E277420747269675C
:106250006765722E20446562726973206F6E206ECE
:106260006F7A7A6C653F2057616974696E67206642
:106270006F722072657365742E007F0153656E73B3
:1062800069746976697479008001446F6E65006590
:106290006E717565696E67202200446F6E652070AF
:1062A00072696E74696E672066696C65004E6F2056
:1062B0004C696E65204E756D6265722077697468F1
:1062C00020636865636B73756D2C204C617374205B
:1062D0004C696E653A20004E6F20436865636B73AE
:1062E000756D2077697468206C696E65206E756DB8
:1062F0006265722C204C617374204C696E653A2083
:1063000000636865636B73756D206D69736D61748F
:1063100063682C204C617374204C696E653A2000D0
:106320004C696E65204E756D626572206973206ED2
:106330006F74204C617374204C696E65204E756DCE
:106340006265722B312C204C617374204C696E6530
:106350003A2000257520627974657320777269741C
:1063600074656E20746F202553206174206164640D
:1063700072657373203078253038780A00442564BC
:10638000202D20526561642F577269746520255352
:106390000A003F3F00526F6D616E61004872766186
:1063A00074736B69004D616779617200536C6F762D
:1063B000656E63696E61004E6F72736B0053766534
:1063C0006E736B61004E656465726C616E64730020
:1063D000506F6C736B69004974616C69616E6F001A
:1063E0004672616E6361697300457370616E6F6CB4
:1063F00000446575747363680043657374696E6106
:1064000000456E676C6973680020436F756E742079
:10641000583A200045303A25642052504D205052C1
:106420004E313A25642052504D204530403A257572
:106430002050524E31403A25750A00526573656E00
:10644000640025533A20256C640A25530A002F2F37
:10645000616374696F6E3A6E6F74696669636174C3
:10646000696F6E2025530A0046696C616D656E7414
:106470002072756E6F7574206465746563746564ED
:10648000210064697361626C656400656E61626CB1
:10649000656400454550524F4D005352414D0044F4
:1064A0002D31202D20456E646C657373206C6F6FE9
:1064B000700A00416374697665204578747275646A
:1064C00065723A203000496E76616C6964206578A7
:1064D000747275646572004D323230205325640049
:1064E0005344207072696E74696E672062797465B6
:1064F0002000257500556E6B6E6F776E20636F6D93
:106500006D616E643A2022004D32303020496E7643
:10651000616C696420657874727564657220007AB4
:106520005F6D61783A20007A5F6D696E3A2000797C
:106530005F6D696E3A2000545249474745524544C1
:10654000006F70656E00785F6D696E3A200052656D
:10655000706F7274696E6720656E6473746F7020FB
:10656000737461747573004D3131322063616C6CEA
:1065700065642E20456D657267656E63792053747E
:106580006F702E002F2F616374696F6E3A75766C91
:106590006F5F7265636F766572795F72656164794A
:1065A0000025533A256C7520636D0A25533A256CF6
:1065B00075206D696E0A0053494C454E54004E4F8C
:1065C000524D414C002553204D4F44453A205065D3
:1065D0007263656E7420646F6E653A202568686426
:1065E0003B207072696E742074696D652072656DF0
:1065F00061696E696E6720696E206D696E733A20FD
:1066000025643B204368616E676520696E206D6973
:106610006E733A2025640A005072696E7465725375
:10662000746174653A2025640A00456E64206669C9
:106630006C65206C69737400426567696E206669D9
:106640006C65206C69737400556E6B6E6F776E208D
:10665000256320636F64653A2025730A000A504958
:106660004E44412074656D70657261747572653A4F
:1066700020252E3166205A20736869667420286DA3
:106680006D293A20252E3366000A537465703A202E
:1066900025642F360A000A537465703A2025642F4A
:1066A000362028736B6970706564290A50494E441E
:1066B000412074656D70657261747572653A20254C
:1066C00064205A20736869667420286D6D293A30F9
:1066D0000A000A5A45524F3A20252E33660A0073A3
:1066E000746172742074656D706572617475726521
:1066F0003A20252E31660A0025642020252E326698
:1067000000255320583A20252E356620593A202559
:106710002E3566205A3A20252E35660A00536C65C0
:1067200065702E2E2E0045303A25642052504D0AB9
:1067300050524E303A25642052504D0A00473930AD
:10674000004D31303700537570657250494E4441E9
:106750000048426564206F6E206C6F616400466C77
:10676000617368416972004572723A484F54454EF0
:10677000442046414E204552524F52002F2F616314
:1067800074696F6E3A726573756D6564002F2F6161
:106790006374696F6E3A726573756D65002F2F6152
:1067A0006374696F6E3A7265616479002F2F61635B
:1067B00074696F6E3A6E6F745F7265616479002FF1
:1067C0002F616374696F6E3A63616E63656C004D2F
:1067D0003834004F4B004C4344207374617475731C
:1067E000206368616E67656400534420636172646E
:1067F0002072656C6561736564002F2F6163746935
:106800006F6E3A737461727400473931004D3730DE
:1068100032004732382057004D3530300042616435
:1068200020696E7465727275707400576174636864
:10683000646F672074696D656F757400537461745B
:106840006963206D656D6F7279206861730A626596
:10685000656E206F7665727772697474656E004636
:1068600049524D57415245204352415348210A4312
:106870007261736820726561736F6E3A0A0020203E
:10688000506C616E6E6572427566666572427974AF
:1068900065733A20002046726565204D656D6F7204
:1068A000793A2000207C20417574686F723A20008C
:1068B000204C61737420557064617465643A2000E3
:1068C00020536F667477617265205265736574003A
:1068D000205761746368646F672052657365740044
:1068E0002042726F776E206F7574205265736574E5
:1068F000002045787465726E616C20526573657412
:1069000000506F7765725570006572726F722077F4
:10691000726974696E6720746F2066696C650044E3
:106920006F6E6520736176696E672066696C652E8F
:10693000006F6B0046696C616D656E74004D65613A
:10694000737572656420736B6577733A20256620D2
:1069500025660A0046697474696E67206661696C11
:106960006564203D3E2063616C6962726174696F89
:106970006E206661696C65642E0A0043616C696211
:10698000726174696F6E20737563636573732E0A29
:1069900000416C6C20342063616C696272617469BF
:1069A0006F6E20706F696E747320666F756E642EE3
:1069B0000A00312F3400312F3400312F3900457255
:1069C000723A5052494E542046414E204552524F41
:1069D000520025632533642F256481005A25362E05
:1069E00032662563005A2020202D2D2D200086257B
:1069F00033642525002D2D2D2525002533642525DF
:106A000000205344002020200020484F0020465200
:106A10004D2000872D2D3A2D2D2020008725337500
:106A20006820256325630087253032753A2530328A
:106A30007525632563002F2F616374696F6E3A704B
:106A40006175736564002F2F616374696F6E3A70AE
:106A5000617573650044756D7020746F2073657285
:106A600069616C0068656C702E7072757361336457
:106A70002E636F6D00666F72756D2E707275736127
:106A800033642E636F6D00707275736133642E63AF
:106A90006F6D004D3730310025533A0A2531382EBD
:106AA00032666D200A25533A0A2531306C64642021
:106AB000253032646820253032646D0025533A0A4F
:106AC0002531382E32666D200A25533A0A25313099
:106AD0006C646820253032646D2025303264730088
:106AE00025362E32666D6D0025530A25530A25532F
:106AF0003A0A25533A0025332E32668100252D317E
:106B0000342E3134533A0A25530A252D31342E318F
:106B100034533A25332E3266810A252D31342E31F5
:106B200034533A25332E3266810020203000202055
:106B3000310046494E44410050494E444100576996
:106B40007A61726420656E642073746174653A20A2
:106B500025640A0053706F6F6C4A6F696E00466956
:106B6000726D7761726500507275736120693320B0
:106B70004D4B322E3553204F4B2E004D36303000CA
:106B800053442063617264206F6B006F70656E52B6
:106B90006F6F74206661696C656400766F6C756DEB
:106BA000652E696E6974206661696C656400534482
:106BB00020696E6974206661696C006F70656E2073
:106BC0006661696C65642C2046696C653A200043F7
:106BD000616E6E6F7420656E746572207375626489
:106BE00069723A20004D3234004D32332025730053
:106BF0005072696E7465722073746F707065642072
:106C000064756520746F206572726F72732E2053E5
:106C100075706572766973696F6E207265717569DA
:106C20007265642E0047312045252D2E336620469F
:106C300032373030004D383300312F390088002092
:106C4000746F6F206C6F6E672065787472757369EE
:106C50006F6E2070726576656E7465640020636F78
:106C60006C6420657874727573696F6E20707265DC
:106C700076656E746564004D6F76652061626F7233
:106C800074656400084AD73B3BCE016E84BCBFFDEF
:106C9000C12F3D6C74319ABD56833DDA3D00C77FEC
:106CA00011BED9E4BB4C3E916BAAAABE0000008085
:106CB0003F05A84CCDB2D44EB93836A9020C50B914
:106CC000918688083CA6AAAA2ABE000000803F0739
:106CD000634236B79BD8A71A39685618AEBAAB5577
:106CE0008C1D3CB7CC5763BD6DEDFD753EF617723C
:106CF00031BF000000803F08000000BE922449120E
:106D00003EABAAAA2ABECDCCCC4C3E00000080BE31
:106D1000ABAAAAAA3E00000000BF000000803F000E
:106D200000000000084178D3BB4387D1133D190E02
:106D30003CC3BD4282AD2B3E68EC8276BED98FE16A
:106D4000A93E4C80EFFFBE01C4FF7F3F0000000062
:106D500000000C9408EA0C94C8B00D9491300D9486
:106D600040640C9402C10D94E7020C9456B50C9447
:106D700046B30C9443C10D94D4010C94AB6D0C94A8
:106D8000B4E20C942CEC0C9496BC0D9417400D942A
:106D90009F060C948E6B0D94F5100D9428020C94A4
:106DA000D3BB0D94B8040C941EB50C94E8B50C94A8
:106DB000C6E70C94ADFD0D94A8060C94CCE20D949E
:106DC00075310C94CAFC0D94AE0D0D94A5310C9444
:106DD0009FFC0C94FCE20C94EDE20C9405B50C9431
:106DE00077E90C9425C10C94D7BA0D94662F0C94B6
:106DF000F9E20C94C0C00D94C0300C942FC10D94D6
:106E0000D3390C94C5FD0C94D0FD0D94E2100C9474
:106E10003BB30D94492F0C94CDBB0C940AB50C9444
:106E2000ACFE0D945F310C9452EF0D9465310C94CF
:106E3000A9FC0C94E2FE0D94AC950D943F6A0C9461
:106E400028FE0C9470BC0D9429040C94E96D0C94EC
:106E50007C6D0C94F6B00C9423B50C9494B10C9406
:106E6000E3B00D94372F0D94202F0D94C3300C9464
:106E7000D9BB0C94CCF60C94CCE70D94C5630D945F
:106E80002E3A0C941DC60D9482110C94D76D0D945E
:106E90003E110C949AB10C94F2FD0C94C0B00D9478
:106EA000962E0D9469070D940A220D946D310C9461
:106EB000B3FC0C94F8C00C946CB50D94C5040C9400
:106EC00002BB0D94B5310D94466A0C94D1F70C9425
:106ED000E9F70C9415FE0D9494010C9411C10C94D7
:106EE0003EEF0C94CFB50D94522F0C9452FE0C949F
:106EF00087BC0D94B6300C94956D0C9406E90C94F7
:106F00009BBC0C942BEB0C94B46D0C94D4C00D94DE
:106F1000DD690C9467FE0C94CDEA0D949E110D94DE
:106F20008D310C9462B00D9462310C94A8E20C94F3
:106F300060BC0C94D1B00D94A5930D94AD310C941C
:106F4000CDBA0D94872F0D94FC300D942B310C94F9
:106F50001DFC0C94B6C00C946BFC0D940A050C94AB
:106F600002E30D94781D0C94B1C00C94CBB00D9439
:106F7000DE630C9439C10C946BF70C94A9C00C948B
:106F800002C40D94B9300C9417FE0C949BFF0C9422
:106F90007CBC0C94626D0D94312F0D948F020C9477
:106FA000D5B00D944E010D94BD310C9493BB0C944F
:106FB00003B10C9459FE0C94575E0D941D090D9469
:106FC00085310C94B9FD0D9420640C94DBEF0D9485
:106FD00027000D94B62E0D947D310C94DBFC0D949E
:106FE0003B2F0C9420B30C943FC60C9461B40D94C9
:106FF000DF0E0C94E2BB0C9497B60C9458BC0C9426
:1070000055B70C94876D0D945C310C94BCB00C9406
:10701000CAF60C94FFB00C94EDB00C9495FC0C9453
:10702000E1F60D9416070C9428B50D94320C0C94CF
:1070300075FC0C94C4B00D94B1060D94E4000D944D
:1070400028310C94DCC00C941BC10D9474120C9468
:1070500060FE0C94C9EA0C94FBB00C9468BC0D94CF
:107060004F6A0C94DBB00D9495310D94C0040D94CF
:107070003D640C94E4C00D9444640D946C070C942E
:1070800098BC0C9461FC0C9409FD0D94800F0D9438
:10709000236A0C9455700C94EEC00C94B5B30D9407
:1070A000062F0C94CABB0C94F1B00D94546A0C9446
:1070B000FFE20C940EE30D9471110C9473E90C949F
:1070C00014B30C94D6BB0C9447BA0C94B1B80D947D
:1070D000CC2E0C945CE60C945FEA0C9414B50C94E2
:1070E00077B60C947FFC0D94EF0C0D946B0A0D9405
:1070F00079300D949D310C94F7B00C94B6B00C948B
:1071000089FC0C94DFB00D94426A0C94CAC00D94B3
:10711000981C0C947FB40C94E9B00C946EFE0C9403
:107120003A6F0C9419B50D942E310D94C22E0C9417
:107130000FB50C942FB30C940EFE0C94D0BB6E6163
:107140006E00696E660000407A10F35A00A0724E1D
:1071500018090010A5D4E80000E87648170000E4FC
:107160000B54020000CA9A3B000000E1F505000044
:1071700080969800000040420F000000A0860100A9
:107180000000102700000000E80300000000640079
:10719000000000000A0000000000010000000000E4
:1071A0002C76D888DC674F0823DFC1DFAE59E1B108
:1071B000B796E5E3E453C63AE651997696E8E6C217
:1071C0008426EB898C9B62ED407C6FFCEFBC9C9F1E
:1071D00040F2BAA56FA5F490055A2AF75C936B6C40
:1071E000F9676DC11BFCE0E40D47FEF520E6B50034
:1071F000D0ED902E0300943577050080841E0800A2
:1072000000204E0A000000C80C333333330F986E51
:1072100012831141EF8D2114893BE65516CFFEE60E
:10722000DB18D1844B381BF77C1D901DA4BBE424D4
:10723000203284725E228100C9F124ECA1E53D2751
:107240002200002045535000204E535000204F464E
:107250004600204F4E005056303100205B4D505DAF
:107260002000256920686F757273202569206D697B
:107270006E757465730052582074696D656F75740E
:10728000004D333130004D313132004D313130005D
:1072900046756C6C205258204275666665720053C4
:1072A000657474696E67732053746F7265640053FC
:1072B000746F7265642073657474696E677320728D
:1072C00065747269657665640048617264636F64B1
:1072D00065642044656661756C74205365747469D7
:1072E0006E6773204C6F6164656400563200000065
:1072F00000C8420000C8420000C843000005430027
:1073000000484300004843000040410000F042E8CC
:10731000030000E8030000C800000088130000001C
:10732000409C4400409C44000000000000000020FD
:107330004E00000000204100002041CDCCCC3E009A
:10734000009040000000000000000000000000CDA0
:10735000CCCC3E3D0A8141FF08433EB099AB438F00
:1073600042FC42E65A343F4C62B045000000000047
:107370004040000034420000000000000000000017
:107380000041000000E03F00002C4300002C4300BF
:107390000040410000F042C0030000C0030000C8EC
:1073A000000000881300001010101000409C4400E2
:1073B00000803F0000003F191400000020307800DA
:1073C000203078006572726F723A200044323320A8
:1073D0002D20656D657267656E63792073657269CE
:1073E000616C2064756D7000437573746F6D004E31
:1073F000796C6F6E504100536174696E20200054A7
:10740000657874757200536D6F6F746800312E303B
:1074100000312E3500554E4B4E4F574E004C4131EA
:1074200030433A204C696E65617220416476616E2A
:107430006365206D6F64653A20004C413130433AFA
:107440002041646A757374656420452D4A65726BCA
:107450003A200020AA51A63E0FA8AF004800699626
:107460000000DF6025555887680427F2E0005E348D
:1074700003CC1960F33C0EF88F00DB0802949200F5
:107480003E1C079A8700E524008528527E06001BD3
:10749000E4007E781270787061F812788F884178F5
:1074A0004270787061782570787061F850788F88B4
:1074B000D1F02527078761F025278F88412C0D27DC
:1074C000AA50D1BC0707871161BE788F8811417817
:1074D0005270787061F852788F88412012788870E5
:1074E0006320527888706348527888874303111765
:1074F000997064181278F870654412F8F8F045181D
:107500004278F87065182578F87065185278F87028
:1075100065185078F870650C078F872365A20F8F68
:107520008F114500120622706900120722274900B8
:107530002506227069002507222749001206222706
:107540006C026236A2706C40456C44704C0362223F
:1075500022706C43888888F04C7812BC88806E78E2
:1075600052BC88806E38127888706F78127888875D
:107570004F38427888706F38257888706F3A007974
:10758000AC786F3D079AAC786F7850788887EF3980
:10759000497888706F0852BC8880729852F88F982A
:1075A0005220127870F07348127863875320527813
:1075B00070F0734852786387531007870F24731253
:1075C000786387245360699A988BE22304E44430FB
:1075D00074104E444324747C12888960753C508832
:1075E0008870557825288960757949088960753CC7
:1075F00012887070790C12885222594412F124F0CA
:107600007A4452F124F07A8C52F0368F5A4420F1A9
:1076100024F07A00401454CDCCCC3D0AD7233C173B
:10762000B7D13877CC2B329595E6241FB14F0A009D
:107630000020410000C84200401C4620BCBE4CCA8D
:107640001B0E5AAEC59D744E414E494E4600007AFF
:10765000430000524300005243000000000000803D
:10766000C09A99193E00000000000080C09A991944
:107670003E20503A002042403A0020403A00202F5D
:10768000002054303A00202F0020423A00202F00E2
:10769000543A0025534578636573736976652062B3
:1076A0006564206C6576656C696E6720636F7272C5
:1076B000656374696F6E3A202569206D6963726F26
:1076C0006E730A00426564206C6576656C696E674E
:1076D000206661696C65642E20546F6F206D756340
:1076E0006820766172696174696F6E2066726F6D71
:1076F00020656570726F6D206D657368004265640A
:10770000206C6576656C696E67206661696C65647E
:107710002E2053656E736F7220747269676765728D
:10772000656420746F6F20736F6F6E002020004DB2
:107730006561737572656420706F696E74733A0069
:107740005A20736561726368206865696768743A76
:1077500020352E3066004E756D20582C593A203752
:107760002C37004D65736820626564206C65766512
:107770006C696E67206E6F74206163746976652E24
:107780000020453A00205A3A0020593A0020453A54
:1077900000205A3A0020593A00583A00202D3E2045
:1077A0000053706F6F6C4A6F696E3A20002C200096
:1077B000496E61637469766974792053687574647D
:1077C0006F776E004B494C4C45442E005072696EE9
:1077D0007465722068616C7465642E206B696C6CD2
:1077E00028292063616C6C656421005A206C6976DD
:1077F000652061646A757374206F7574206F6620EC
:1078000072616E67652E2053657474696E672074AB
:107810006F20302E20436C69636B20746F20636F80
:107820006E74696E75652E005A206C6976652061EC
:10783000646A757374206F7574206F662072616E50
:1078400067652E2053657474696E6720746F2030ED
:107850000020453A3020423A00543A00627573796C
:107860003A2070617573656420666F7220696E706E
:10787000757400627573793A207061757365642060
:10788000666F72207573657200627573793A207045
:10789000726F63657373696E670073657269616C9B
:1078A0002064756D702000496E76616C69642054A7
:1078B00020636F64652E004475706C696361746544
:1078C00020542D636F64652069676E6F7265642E46
:1078D00000416476616E6365204B3D004B206F75FF
:1078E00074206F6620616C6C6F7765642072616EC6
:1078F000676521004D4B322E3553004D4B322E35EE
:10790000534D4D553253001C4FFC002533642F2539
:1079100033640025336400200A200A200A20002551
:1079200053537461746973746963733A0A255320FD
:10793000204D37382053256C752054256C750A006E
:1079400025534172632053657474696E67733A20DE
:10795000503A4D6178206C656E677468286D6D29AA
:1079600020533A4D696E206C656E67746820286DEF
:107970006D29204E3A436F7272656374696F6E733E
:1079800020523A4D696E207365676D656E74732081
:10799000463A5365676D656E74732F7365632E0A7F
:1079A000255320204D3231342050252E326620536D
:1079B000252E3266204E25642052256420462564FB
:1079C0000A00255346696C616D656E742073657499
:1079D00074696E67733A2044697361626C65640A06
:1079E00000255346696C616D656E7420736574740F
:1079F000696E67733A0A25532020204D32303020BB
:107A000044252E32660A00255352657472616374F0
:107A10003A20533D4C656E67746820286D6D2920AF
:107A2000463A537065656420286D6D2F6D29205A84
:107A30003A205A4C69667420286D6D290A25532016
:107A400020204D3230372053252E32662046252EF9
:107A50003266205A252E32660A25535265636F76A8
:107A600065723A20533D4578747261206C656E678B
:107A7000746820286D6D2920463A5370656564202E
:107A8000286D6D2F6D290A25532020204D32303866
:107A90002053252E32662046252E32660A25534174
:107AA00075746F2D526574726163743A20533D3062
:107AB00020746F2064697361626C652C20312074BE
:107AC0006F20696E74657270726574206578747267
:107AD0007564652D6F6E6C79206D6F7665732061AE
:107AE00073207265747261637473206F72207265A3
:107AF000636F7665726965730A25532020204D32C5
:107B00003039205325640A002553504944206865C4
:107B100061746265642073657474696E67733A0A90
:107B200025532020204D3330342050252E3266201E
:107B300049252E32662044252E32660A00255350F0
:107B400049442073657474696E67733A0A2553203B
:107B500020204D3330312050252E32662049252EED
:107B600032662044252E32660A0025535374657010
:107B7000732070657220756E69743A0A255320204F
:107B80004D39322058252E32662059252E32662056
:107B90005A252E32662045252E32660A25534D6120
:107BA00078696D756D2066656564726174657320B2
:107BB000286D6D2F73293A0A255320204D3230331A
:107BC0002058252E32662059252E3266205A252E21
:107BD00032662045252E32660A25534D6178696D3F
:107BE000756D20616363656C65726174696F6E2089
:107BF000286D6D2F7332293A0A255320204D3230DB
:107C0000312058256C752059256C75205A256C75C6
:107C10002045256C750A2553416363656C65726167
:107C200074696F6E3A20503D7072696E742C2052E8
:107C30003D726574726163742C20543D7472617678
:107C4000656C0A255320204D3230342050252E32C9
:107C5000662052252E32662054252E32660A255380
:107C6000416476616E636564207661726961626CFD
:107C700065733A20533D4D696E2066656564726197
:107C8000746520286D6D2F73292C20543D4D696E2D
:107C90002074726176656C206665656472617465D6
:107CA00020286D6D2F73292C20423D6D696E696D02
:107CB000756D207365676D656E742074696D6520E0
:107CC000287573292C20583D6D6178696D756D207C
:107CD0005859206A65726B20286D6D2F73292C20EE
:107CE000205A3D6D6178696D756D205A206A657204
:107CF0006B20286D6D2F73292C2020453D6D6178F8
:107D0000696D756D2045206A65726B20286D6D2F39
:107D100073290A255320204D3230352053252E3229
:107D2000662054252E32662042256C752058252E5B
:107D300032662059252E3266205A252E326620457D
:107D4000252E32660A2553486F6D65206F6666736F
:107D5000657420286D6D293A0A255320204D323054
:107D6000362058252E32662059252E3266205A2577
:107D70002E32660A004361703A25533A25630A00A1
:107D800050525553415F4D4D553200455854454E64
:107D90004445445F4D3230004155544F5245504F99
:107DA00052545F504F534954494F4E004155544F20
:107DB0005245504F52545F46414E53004155544F27
:107DC0005245504F52545F54454D50000044656C2D
:107DD0006574696F6E206661696C65642C20466904
:107DE0006C653A200046696C652064656C65746555
:107DF000643A004E6F74205344207072696E746947
:107E00006E67005072696E7420736176656400530A
:107E100044207072696E742070617573656400250A
:107E200033642F25336400667600746878005052FE
:107E30004E0022283229006E6F2076616C69642022
:107E4000636F6D6D616E64007A65726F72697A65D9
:107E50006400666163746F727920726573746F7207
:107E6000656400696E6465782C2074656D702C20E3
:107E700075737465702C20756D0050494E44412017
:107E800063616C207374617475733A2000503A001A
:107E90005761697420666F722050494E44412074C6
:107EA00061726765742074656D7065726174757256
:107EB000653A00204100205000204200204C002064
:107EC0005200205A00204E4F5420494E49544941F7
:107ED0004C495A45440053686565742000205A2077
:107EE00056414C5545204F5554204F462052414E47
:107EF000474500496E76616C6964207368656574F6
:107F00002049442E20416C6C6F7765643A20302EF6
:107F10002E004155544F004C414E472053454C20B4
:107F2000464F524345440020643A0020693A0020FD
:107F3000703A0020643A0020693A0020703A002527
:107F40006925250A00256925250A002228312900EE
:107F50002F2F00002045585452554445525F434F3F
:107F6000554E543A3100204D414348494E455F54E7
:107F70005950453A00312E3000206261736564200B
:107F80006F6E204D61726C696E204649524D5741AB
:107F900052455F55524C3A68747470733A2F2F678C
:107FA00069746875622E636F6D2F707275736133BB
:107FB000642F50727573612D4669726D77617265B9
:107FC0002050524F544F434F4C5F56455253494FE8
:107FD0004E3A00373733313032346564005F003851
:107FE000323739002B004649524D574152455F4EBA
:107FF000414D453A50727573612D4669726D7761D6
:10800000726520004D3131332053006F6B20006EBC
:108010002F61003F546F736869626120466C617321
:1080200068416972204765744950206661696C65D2
:10803000640A00000125301D0CFF24311C0BFF23B6
:108040002F1B0A17FF0406222B1A03363535382555
:1080500069206D696E2C2025692073656300496E67
:1080600076616C6964204D20636F64653A202573E6
:108070000A0050494E44412070726F62652063616E
:108080006C6962726174696F6E20737461727400DE
:108090004E6F2050494E444120746865726D69737B
:1080A000746F7200736574006E6F7A7A6C65004D40
:1080B000424C004652004C7A004C616E6700315FC2
:1080C00037356D6D5F4D4B3235532D52414D426FFB
:1080D0003130612D453344763666756C6C005265DF
:1080E0007600332E31342E312D383237390046693F
:1080F0007200534E20696E76616C696400534E00C5
:108100005245534554004D4D555245530075766CBC
:108110006F0046414E0046414E50494E5453540064
:108120005052555341004D3130345330004731588F
:1081300031305931383046343030300047315A31DF
:10814000304631333030004D313430533000473118
:10815000452D302E3037354632313030004D3230FB
:108160003453313030300047315A354637323030B1
:10817000004731452D312E35463231303000473100
:108180005A302E32004731583230322E354538467B
:1081900031343030004731592D32463130303000E3
:1081A000473158323430453235463232303000476C
:1081B000315A302E33463130303000473158353562
:1081C000453846323030300047315835453239462F
:1081D0003138303000473158353545323946313045
:1081E000373300473932453000473238004D31309F
:1081F00039004D313930001000C90210012C014006
:1082000001220170011801B0010E01F001040150BA
:1082100002FA00B002F0003003E600D003DC009068
:1082200004D2007005C800A006BE000008B400B06B
:1082300009AA00D00BA000600E960060118C00000F
:1082400015820020197800C01D6E00A0226400B0C5
:10825000275A00902C500000314600E0343C0010BA
:10826000383200903A2800603C1E00A03D14008087
:108270003E0A00203F00004578706572696D656EAA
:1082800074616C00302E383000302E363000302EC5
:10829000343000302E32350044697361626C6520E1
:1082A0006661726D206D6F64650052657365742040
:1082B0004D4D55004D4D55004D3434004739390072
:1082C00044697361626C65206661726D206D6F64D4
:1082D000653F00473238205859004D20383400851A
:1082E0002E2E002533642F30002533642F30006C90
:1082F00063645F73656C66636865636B5F6178690F
:10830000732025642C2025640A00486F74656E6410
:1083100000426564005A00590058002D2D2D2D2D66
:108320002D2D2D2D2D2D2D2D2D2D2D2D2D2D2D00AA
:10833000537570657250494E44413A003D6741673C
:108340004E8147813C812D810D682681CF67473161
:1083500059252E346645252E34660047315A252E80
:1083600032660047315835305931353500E3813DAB
:1083700067356C718167815D81473158252E346680
:1083800045252E3466004731463130383000D581DE
:10839000C881BB81AF81E381A081958185817E8188
:1083A0005425640047315A302E34004731592D335B
:1083B0004631303030004167F281ED81E981E3815F
:1083C0004D3834205859004D31303920533238302F
:1083D0000047312058313235205A32303020463172
:1083E00030303000496E76616C6964205049442019
:1083F00063616C2E20726573756C74732E204E6FE2
:10840000742073746F72656420746F2045455052F8
:108410004F4D2E004D3330312050252E32662049ED
:10842000252E32662044252E3266004D333033200F
:1084300045302053253375005243004445560042D1
:1084400045544100414C50484100000021002400A7
:1084500027002A002D003000330001010000040134
:1084600007010A0100002200250028002B002E0031
:108470003100340002010000050108010B01000079
:1084800020002300260029002C002F0032000001CC
:108490000000030106010901050505050705080897
:1084A0000808020202020A0A08080404040401017E
:1084B0000101010101010303030303030303040793
:1084C00007070C0C0C0C0C0C0C0C0202020206062A
:1084D0000606060606060B0B0B0B0B0B0B0B070712
:1084E0000A0A0A0A0A0A0505050404040808010222
:1084F00010202008081020401020408002010201B6
:10850000080402010102040810204080804020106D
:1085100008040201800402018040201008040201C6
:10852000080402010102040810204080010204082E
:108530001020408010080408801020400440801063
:108540002040048000000A0B02090C0D0E080703EE
:108550000401000000000000000000000000000016
:10856000000000000000000000000000000000000B
:1085700012111000000000000000000000000000C8
:1085800000000000000000000000000000000000EB
:1085900000000000000000000000332E31342E31B6
:1085A000000A204F726967696E616C2050727573A2
:1085B000612069330A202020507275736120526552
:1085C0007365617263680A2532302E32305300536E
:1085D000706F6F6C4A6F696E20697320006164630D
:1085E0005F696E697400200A200A200A2000416C2D
:1085F0006C20446174610053657276696365207014
:10860000726570005368697070696E67207072657A
:10861000700053746174697374696373004C616EA4
:1086200067756167650045524153494E4720616C4B
:108630006C206461746100466163746F72792052CA
:108640004553455400505255534133444657000357
:10865000000E000100400003000200000004007052
:1086600072757361336400323032352D30342D32FF
:10867000322032323A30333A35330020332E31341F
:108680002E312D383237395F373733313032346558
:1086900064007374617274004D323900252D392ED7
:1086A00039535B0033332942000058419A998D4178
:1086B00033335340200A200A20004D4D55323A00F2
:1086C0004D6561737572652063656E7465722020F7
:1086D0000078797A63616C5F6D6561737572655F4F
:1086E000656E7465720A0078797A63616C5F737085
:1086F0006972616C382063783D25642063793D257B
:1087000064207A303D256420647A3D2564207261BE
:10871000646975733D25642061643D25640A0078B1
:10872000797A63616C5F7365617263685A206E6FFA
:10873000207369676E616C0A20783D256C6420792E
:108740003D256C64207A3D256C640A00204F4E2D37
:108750005349474E414C20617420783D256420796F
:108760003D2564207A3D25642061643D25640A002E
:1087700078797A63616C5F7365617263685A207897
:108780003D256C6420793D256C64207A3D256C6420
:108790000A002530327800205B25662025665D20A2
:1087A0006D6D207061747465726E2063656E7465A2
:1087B000720A00205B25662025665D5B25665D20CC
:1087C0006D6D20646976657267656E63650A000089
:1087D00000F000F801FC03FE07FE07FE07FE07FCA1
:1087E00003F801F000000000000000F000F801FCB8
:1087F00003FC03FC03FC03F801F000000000007818
:10880000797A63616C5F6D6561737572655F6C65C4
:108810006176650A00203C20005741524E494E4780
:108820003A2046726F6E7420706F696E74206E6F9E
:108830007420726561636861626C652E20592063E3
:108840006F6F7264696E6174653A000000004041A8
:108850000000804000005C430000804000005C435A
:1088600000004443000040410000444325642F348D
:1088700000497465726174696F6E3A200043616CDF
:108880006962726174696F6E206661696C656421EA
:1088900020436865636B2074686520617865732088
:1088A000616E642072756E20616761696E2E004D85
:1088B000494E54454D5020424544206669786564D0
:1088C000004D494E54454D5020484F54454E44208C
:1088D00066697865640024F4D43050C38E20C2A247
:1088E0004017828B7011127A910D816CD90AA861A0
:1088F000E108C7586607615143061E4B5D05C14537
:10890000A7041A411104093D980371393103403617
:10891000DB0265339102D4305402802E1D02632C99
:10892000EE01752AC501B028A001102781018F250D
:1089300064012B244B01E0223401AC211F018D2066
:108940000D01801FFC00841EED00971DDF00B81C88
:10895000D200E61BC600201BBC00641AB200B2198C
:10896000A8000A19A0006A189900D11791004017B1
:108970008B00B516840031167E00B31579003A15C8
:108980007300C7146F0058146A00EE136600881352
:10899000630025135E00C7125B006C1257001512AE
:1089A0005400C111510070114F0021114B00D6101D
:1089B00049008D1047004610440002104200C00FCD
:1089C0004000800F3E00420F3C00060F3B00CB0EE4
:1089D0003800930E37005C0E3500270E3400F30D7F
:1089E0003200C10D3100900D3000600D2E00320DAF
:1089F0002D00050D2C00D90C2B00AE0C2900850C88
:108A000029005C0C2700350C27000E0C2600E80B13
:108A10002400C40B2400A00B23007D0B23005A0B61
:108A20002100390B2100180B2000F80A1F00D90A79
:108A30001E00BB0A1E009D0A1D00800A1D00630A5D
:108A40001C00470A1B002C0A1B00110A1A00F70918
:108A50001A00DD091900C4091900AB0919009209AF
:108A600017007B091800630917004C091600360926
:108A70001600200916000A091500F5081500E0087F
:108A80001400CC081400B8081400A40814009008BE
:108A900013007D0812006B081300580812004608E6
:108AA00012003408110023081100120811000108F7
:108AB0001100F0071000E0071000D0071000C007F9
:108AC0001000B0070F00A107100091070E008307E8
:108AD0000F0074070F0065070E0057070E004907C7
:108AE0000E003B070D002E070E0020070D00130798
:108AF0000D0006070D00F9060C00ED060D00E0065E
:108B00000C00D4060C00C8060C00BC060C00B00615
:108B10000C00A4060B0099060C008D060B008206C3
:108B20000B0077060B006C060B0061060A00570667
:108B30000B004C060A0042060A0038060A002E0600
:108B40000A0024060A001A060A0010060900070691
:108B50000A00FD050900F4050900EB050900E2051E
:108B60000900D9050900D0050900C7050900BE059F
:108B70000900B5050800AD050800A50509009C051C
:108B80000800940508008C050800840508007C0591
:108B90000800740508006C050700650508005D0500
:108BA0000700560508004E05070047050700400569
:108BB000080038050700310507002A0507002305CE
:108BC00007001C050600160507000F05070008052D
:108BD000060002050700FB040600F5040700EE048A
:108BE0000600E8040600E2040700DB040600D504E2
:108BF0000600CF040600C9040600C3040600BD0435
:108C00000600B7040600B1040500AC040600A60483
:108C10000600A00405009B040600950405009004CE
:108C200006008A04050085040500800406007A0415
:108C3000050075040500700405006B04050066045A
:108C40000500610405005C0405005704050052049A
:108C500005004D04050048040500430405003E04DA
:108C600004003A04050035040500300404002C0417
:108C7000050027040400230405001E0404001A0450
:108C8000040016040500110404000D040400090486
:108C900005000404040000040400FC030400F803BD
:108CA0000400F4030400F0030400EC030400E803F0
:108CB0000400E4030400E0030400DC030400D80320
:108CC0000400D4030400D0030400CC030400C80350
:108CD0000300C503030024F404D9201BC40C5C0E5C
:108CE0009804C4095F0265077101F405F900FB04EB
:108CF000B30048048700C10369005803550003030B
:108D00004500BE023A008402310053022A002902C3
:108D1000250004022000E4011C00C8011900AF0175
:108D20001700980114008401130071011000610103
:108D3000100051010E0043010D0036010B002B0104
:108D40000B0020010B00150109000C0109000301B3
:108D50000800FB000800F3000800EB000700E40037
:108D60000600DE000600D8000600D2000600CC0097
:108D70000500C7000500C2000500BD000400B900E1
:108D80000400B5000400B1000400AD000400A90017
:108D90000400A5000300A20003009F0004009B0044
:108DA0000300980003009500020093000300900068
:108DB00003008D0002008B00030088000200860083
:108DC000020084000300810002007F0002007D0099
:108DD00002007B00020079000200770001007600AB
:108DE00002007400020072000100710002006F00B6
:108DF00002006D0001006C0002006A0001006900C1
:108E000002006700010066000100650001006400C7
:108E100002006200010061000100600001005F00CB
:108E200002005D0001005C0001005B0001005A00CF
:108E300001005900010058000100570001005600D0
:108E400001005500010054000100530000005300D0
:108E500001005200010051000100500001004F00CC
:108E600001004E0000004E0001004D0001004C00CA
:108E700001004B0000004B0001004A0001004900C6
:108E800001004800000048000100470001004600C2
:108E900000004600010045000000450001004400BC
:108EA00001004300000043000100420000004200B6
:108EB00001004100000041000100400001003F00AE
:108EC00000003F0001003E0000003E0001003D00A8
:108ED00000003D0001003C0000003C0000003C00A0
:108EE00001003B0000003B0001003A0000003A0096
:108EF000010039000000390001003800000038008E
:108F00000000380001003700000037000100360083
:108F1000000036000000360001003500000035007A
:108F2000000035000100340000003400000034006F
:108F30000100330000003300000033000100320064
:108F4000000032000000320001003100000031005A
:108F5000000031000100300000003000000030004F
:108F600001002F0000002F0000002F0000002F0044
:108F700001002E0000002E0000002E0001002D0038
:108F800000002D0000002D0000002D0001002C002D
:108F900000002C0000002C0000002C0001002B0021
:108FA00000002B0000002B0000002B0001002A0015
:108FB00000002A0000002A0000002A000100290009
:108FC00000002900000029000000290000002900FD
:108FD00001002800000028000000280000002800F0
:108FE00000002800010027000000270000002700E3
:108FF00000002700000027000100260000002600D6
:1090000000002600000026000000260001002500C8
:1090100000002500000025000000250000002500BC
:1090200000002500010024000000240000002400AE
:1090300000002400000024000100230000002300A1
:109040000000230000002300000023000000230094
:109050000000230001002200000022000000220086
:109060000000220000002200000022000100210078
:10907000000021000000210000002100000021006C
:10908000000021000000210001002000000020005D
:109090000000200000002000000020000000200050
:1090A000000020000000200001001F0000001F0041
:1090B00000001F0000001F0000001F0000001F0034
:1090C00000001F0001001E0000001E0000001E0026
:1090D00000001E00000045303A20005A3A20005996
:1090E0003A2000583A20004D53312C4D5332205035
:1090F000696E7300504944204175746F74756E65D4
:109100002066696E697368656421205075742074E7
:109110006865206C617374204B702C204B69206152
:109120006E64204B6420636F6E7374616E74732081
:1091300066726F6D2061626F766520696E746F2054
:10914000436F6E66696775726174696F6E2E680031
:10915000504944204175746F74756E65206661696D
:109160006C6564212074696D656F75740020403AE8
:1091700000543A00423A00504944204175746F74DB
:10918000756E65206661696C6564212054656D703B
:109190006572617475726520746F6F2068696768A5
:1091A00000204B643A2000204B693A2000204B708D
:1091B0003A200020436C6173736963205049442056
:1091C000002054753A2000204B753A2000206D6134
:1091D000783A2000206D696E3A200020643A200021
:1091E00020626961733A2000504944204175746FD0
:1091F00074756E6520737461727400504944204127
:1092000075746F74756E65206661696C65642E2077
:10921000426164206578747275646572206E756D44
:109220006265722E00486F74656E642066616E2000
:109230007370656564206973206C6F776572207444
:1092400068616E206578706563746564005072694A
:109250006E742066616E207370656564206973208A
:109260006C6F776572207468616E206578706563D5
:10927000746564004D494E54454D502042454400AC
:109280004D494E54454D50004D415854454D5000A8
:109290004D415854454D50204245440070012C0129
:1092A00090012701B0012201C0011D01F001180148
:1092B0001002130130020E01600209019002040144
:1092C000C002FF000003FA004003F5008003F00035
:1092D000D003EB002004E6007004E100E004DC00B1
:1092E0004005D700C005D2004006CD00D006C8001A
:1092F0008007C3003008BE00F008B900C009B40000
:10930000B00AAF00B00BAA00D00CA500000EA00060
:10931000500F9B00C01096005012910000148C005A
:10932000C0158700B0178200B0197D00D01B7800EF
:10933000001E730040206E0090226900F02464003B
:1093400040275F0090295A00E02B5500102E500056
:1093500020304B0010324600E033410090353C0095
:109360001037370070383200A0392D00B03A28008D
:10937000A03B2300603C1E00103D1900903D1400EE
:10938000103E0F00703E0A00C03E0500003F000086
:1093900020484F54454E4420544845524D414C209E
:1093A00052554E4157415900204845415442454489
:1093B00020544845524D414C2052554E4157415939
:1093C00000544845524D414C2052554E4157415949
:1093D0000042454420544845524D414C2052554E80
:1093E000415741590020544845524D414C20525557
:1093F0004E41574159202850524548454154204834
:109400004F54454E44290020544845524D414C206C
:1094100052554E41574159202850524548454154D4
:109420002048454154424544290050524548454151
:1094300054204552524F5200424544205052454814
:10944000454154204552524F52002074726967675B
:109450006572656421004865617465727320737775
:10946000697463686564206F66662E20003A200088
:109470004572723A200000FF0102010002FFFFFE68
:109480000001FE01FF00506C656173652072657319
:1094900074617274005553415254322072782046E0
:1094A000756C6C212121003A2000252D31322E319E
:1094B0003253252D642F36002533642F252D336438
:1094C00000203A200025335300252D377300252D29
:1094D00031352E313553252D35640A252D31352E64
:1094E000313553252D35640A0025530A20252D31A9
:1094F000362E313653252D33640A20252D31362E54
:10950000313653252D33640025530A20252D31365D
:109510002E313653252D33640A20252D31362E3138
:109520003653252D33640A20252D31362E313653FE
:10953000252D33640025530A20252D31362E313652
:1095400053252D33640A25530A20252D31362E311B
:109550003653252D33640A0020257325336481207A
:109560000A0025752E25752E25752E2575002000DF
:109570002000466C61736841697220495020416443
:1095800064723A004D4D5520202020202020204E8E
:109590002F410025642E25642E2564002046573A6D
:1095A00000323032352D30342D323200453344769E
:1095B0003666756C6C0052414D426F31306100313E
:1095C0005F37356D6D5F4D4B323553002048617309
:1095D000683A373733313032346564002052657071
:1095E0006F3A707275736133640020332E31342EFC
:1095F000312D38323739004669726D776172653ABC
:10960000003E00464C4558202D20203234302F3566
:109610003000464C4558202D202032343000505028
:109620002020202D20203235342F31303000505072
:109630002020202D20203235340048495053202D41
:1096400020203232302F3130300048495053202D05
:1096500020203232300041425320202D202032354C
:10966000352F3130300041425320202D202032351B
:10967000350050412020202D20203237352F393021
:109680000050412020202D202032373500505642F6
:1096900020202D20203231352F37350050564220E2
:1096A000202D20203231350050432020202D202035
:1096B0003237352F3130350050432020202D2020E7
:1096C0003237350041534120202D20203236302FB3
:1096D0003130350041534120202D202032363000DA
:1096E00050455420202D20203233302F3835005063
:1096F000455420202D202032333000504C41202072
:109700002D20203231352F363000504C4120202D75
:109710002020323135006E6F7A7A6C65202D202042
:109720003235302F30006661726D2020202D2020D0
:109730003235302F383000252D31322E313253253D
:109740002B382E31660045787472756465723A0064
:1097500025632531372E32666D6D00583A00593A2F
:10976000005A3A002563252D31332E313353252BF2
:10977000352E3366002533750050494E4441206331
:10978000616C6962726174696F6E206661696C6593
:10979000642E20436F6E74696E75652077697468F6
:1097A000207072657373696E6720746865206B6ED4
:1097B0006F622E0050494E44412063616C696272B1
:1097C0006174696F6E20646F6E652E20436F6E74D6
:1097D000696E756520776974682070726573736946
:1097E0006E6720746865206B6E6F622E005A3000C1
:1097F0005A31005930005931005830005831004575
:109800006E642073746F70732064696167004738F9
:1098100030004D3435004D3435205A00473736007E
:109820004D3730312050300057697A6172642073AF
:10983000746174653A2025640A0078797A63616CF2
:109840005F73706972616C322063783D25642063B8
:10985000793D2564207A303D256420647A3D256475
:10986000207261646975733D25642061643D2564DF
:109870000A000A00436F756E74646F776E3A202594
:1098800064200025640A005363616E20636F756E67
:1098900074646F776E3A20005061747465726E2044
:1098A00063656E746572205B25662025665D2C20DD
:1098B0006D6174636820256625250A00205B256696
:1098C0002C2025665D5B25665D2066696E616C20D7
:1098D000636972636C650A000000A0400000A0404C
:1098E0000000004000007A43000056439AD95143DB
:1098F000FFFFFFE02D903E8988B24111369C3E77F4
:1099000077C14129CBB03EEFEEDA41BA49CC3EEF08
:10991000EEFC4161C3F33EEFEE16429CA2133FCD35
:10992000CC36428AB0113FABAA56428863DD3DABCC
:10993000AA5642B8AF433F555572421826533F339B
:10994000B38242302A593FEF6E8642000070C10058
:1099500000C8420000C4C10000A0410000E0C000F7
:10996000002041000060C00000C0400000A0412273
:1099700022F2400000A0C19A99A14000000CC255FB
:10998000550542436F6F6C696E672074696D65722F
:109990002073746F7070656400486561746572202F
:1099A000636F6F6C646F776E00436F6F6C696E6787
:1099B0002054696D656F7574207374617274656489
:1099C00000536176696E6720616E64207061726B0E
:1099D000696E670048656174657220636F6F6C64BF
:1099E0006F776E2070656E64696E6700526573757F
:1099F0006D696E672058595A0057726974696E67AD
:109A000020746F2066696C653A200046696C652099
:109A1000616C7265616479206F70656E6564006F5A
:109A2000575E574A5735571F570C57F656E256D1CF
:109A300056BB564A575E57A7569856845673565E7D
:109A400056025A4856365623561256FD55EA55D6F2
:109A500055C155B855A65591554D36303020415514
:109A6000544F0046494E44412066696C616D656EF5
:109A7000742072756E6F75742100436F6D6D756E15
:109A800069636174696F6E2074696D656F757400C8
:109A900050726F746F636F6C204572726F72000347
:109AA000000356657273696F6E206D69736D617422
:109AB000636800436F6D6D616E64204572726F72F2
:109AC00000436F6D6D616E642072656A65637465D5
:109AD00064004D4D5520427574746F6E207075731F
:109AE000686564005265747279427574746F6E5063
:109AF00072657373656400CC59B759A0598B597658
:109B000059625952593B5924590D59F958E558CFC2
:109B100058CF58CF58BA58BA58BA58A758A758A7C4
:109B2000589458945894587D587D587D5868586872
:109B300058685852585258525842582D5817580180
:109B400058F257E557CE57BB57A9579657845774C5
:109B500057427574746F6E00436865636B55736527
:109B600072496E7075742D62746E4C4D52200052A5
:109B7000657365745265747279417474656D70743F
:109B8000730046493A202046533A202020203E20A8
:109B900020822020208100486F74656E64207465E7
:109BA0006D70657261747572652072656163686558
:109BB0006400526573756D696E672054656D700041
:109BC000436F6F6C646F776E20666C616720636CA7
:109BD00065617265640020573A0020453A00543AA6
:109BE000004E6F2030784646207265636569766561
:109BF000640053656E64696E67203078464600469F
:109C0000696C652073656C656374656400205369D5
:109C10007A653A200046696C65206F70656E6564F0
:109C20003A20004E6F772066726573682066696C13
:109C3000653A20004E6F7720646F696E6720666911
:109C40006C653A20002220706F73002220706172D0
:109C5000656E743A2200535542524F5554494E4551
:109C60002043414C4C207461726765743A22007441
:109C70007279696E6720746F2063616C6C207375F4
:109C8000622D67636F64652066696C657320776910
:109C9000746820746F6F206D616E79206C657665D5
:109CA0006C732E002022257322002025236C78005F
:109CB0004449525F45584954004449525F454E5407
:109CC00045523A20257320222573220A00617574BB
:109CD0006F25692E6700041A44656372656D656EB1
:109CE000745265747279417474656D707473000890
:109CF0001B1C0B14525354436F6D6D54696D656F8B
:109D00007574002C206C6173742062797465733AE9
:109D1000200022206661696C65643A20427566669F
:109D200065722066756C6C21002200456E71756548
:109D3000696E6720746F207468652066726F6E7438
:109D40003A2022004572726F723A004D4D553274BE
:109D50006F6F6C3D004D4D55323A004D4D55323AC6
:109D6000006563686F3A003E53302A63362E004D1B
:109D70004D552069732000252E31305320002534A5
:109D80006400457872656D65207370616E206F6642
:109D900020746865205A2076616C756573210025F2
:109DA000642F39004D4D55323A00253364001801B7
:109DB0000419020A92611C61A2603560EC5F5A5F6F
:109DC000E25E7A5E2B5E0B5EBF5D0B5EA85DA85DFA
:109DD000A85DA85DA85DA85DA85DA85DA85DA85D5B
:109DE000A85DA85DA85DA85DA85DA85DA85DA85D4B
:109DF000A85DA85DA85DA85D715D305DE65C735CE3
:109E00003E5CF45BAA5B4C5B135BD15AB45A010114
:109E100001010101010271017101323232030303B8
:109E20000303030303030303030303030303030302
:109E30009393243803930301025603650066006779
:109E400000680069006A006B006C00730074007D9C
:109E5000007E00C900D300DD00CA00D400DE002D62
:109E600001370141012E01380142012F013901431F
:109E70000130013A01440131013B014501320191B8
:109E8000019201F501F601F701F801F901FA01FB70
:109E900001FC0184031F62886214620B6204628AFF
:109EA0004AFF3CFD61F361252E3230530A70727512
:109EB00073612E696F2F3034256875007B5B4552C6
:109EC000523A00332E31342E31005D5B4657523A00
:109ED000005D5B54494D3A005D5B464E4D3A005D76
:109EE0005B46454D3A005D5B5043443A005B544647
:109EF000553A005B50524E3A005B50464E3A305D48
:109F0000005B4449413A005D5B4154423A005D5B6D
:109F10004154303A005D5B5354423A005B53543035
:109F20003A007B5B50524E3A355D007B5B50524E9F
:109F30003A305D007B5B50524E3A395D007B5B509E
:109F4000524E3A385D007B5B5245533A305D5B467A
:109F5000494C3A007B5B5245533A315D5B46494C74
:109F60003A0000002110422063308440A550C660B2
:109F7000E770088129914AA16BB18CC1ADD1CEE1C6
:109F8000EFF13112100273325222B5529442F7723D
:109F9000D662399318837BB35AA3BDD39CC3FFF316
:109FA000DEE36224433420040114E664C774A4444D
:109FB00085546AA54BB528850995EEE5CFF5ACC566
:109FC0008DD55336722611163006D776F66695561D
:109FD000B4465BB77AA719973887DFF7FEE79DD7B6
:109FE000BCC7C448E5588668A778400861180228AD
:109FF0002338CCC9EDD98EE9AFF9488969990AA906
:10A000002BB9F55AD44AB77A966A711A500A333A7C
:10A01000122AFDDBDCCBBFFB9EEB799B588B3BBB55
:10A020001AABA66C877CE44CC55C222C033C600C0C
:10A03000411CAEED8FFDECCDCDDD2AAD0BBD688DA5
:10A04000499D977EB66ED55EF44E133E322E511E5C
:10A05000700E9FFFBEEFDDDFFCCF1BBF3AAF599FF5
:10A06000788F8891A981CAB1EBA10CD12DC14EF195
:10A070006FE18010A100C230E320045025404670FB
:10A080006760B9839893FBA3DAB33DC31CD37FE326
:10A090005EF3B1029012F322D2323542145277624B
:10A0A0005672EAB5CBA5A89589856EF54FE52CD5F6
:10A0B0000DC5E234C324A01481046674476424549B
:10A0C0000544DBA7FAB79987B8975FE77EF71DC706
:10A0D0003CD7D326F2369106B016576676761546EB
:10A0E00034564CD96DC90EF92FE9C899E9898AB956
:10A0F000ABA94458654806782768C018E10882383B
:10A10000A3287DCB5CDB3FEB1EFBF98BD89BBBAB65
:10A110009ABB754A545A376A167AF10AD01AB32A8A
:10A12000923A2EFD0FED6CDD4DCDAABD8BADE89DB5
:10A13000C98D267C076C645C454CA23C832CE01CDA
:10A14000C10C1FEF3EFF5DCF7CDF9BAFBABFD98F45
:10A15000F89F176E367E554E745E932EB23ED10E2A
:10A16000F01E7C3C3E3F2F2A225C0000C536575E25
:10A1700011241FBECFEFD1E2DEBFCDBF00E00CBF88
:10A1800013E0A0E0B2E0E0E5FDE403E00BBF02C0B5
:10A1900007900D92A430B107D9F727E1A4E0B3E00E
:10A1A00001C01D92A430B207E1F710E5C7EBD0E57E
:10A1B00000E006C021970109802FFE010F94ECA05A
:10A1C000C63BD10780E00807A9F70E949FD80D94ED
:10A1D00096A60C94BB742F923F924F925F926F920F
:10A1E0007F928F929F92AF92BF92CF92DF92EF9227
:10A1F000FF920F931F93CF93DF93CDB7DEB72F97C7
:10A200000FB6F894DEBF0FBECDBF6C011B015A0123
:10A21000FC011782168283819E012F5F3F4F490107
:10A2200081FDD2C08FEF9FEFEEC2F12C512C00E0E8
:10A23000003238F48B3209F190F48032F9F0833235
:10A2400009F107FD34C020ED280F2A3020F506FF64
:10A250001BC0FAE0FF9E200D1124F22E05C08D32A6
:10A2600079F0803371F70160F10193FD859193FFDF
:10A2700081911F018111DCCF1AC002600460F4CF0C
:10A280000860F2CF0061F0CF3AE0539E200D112418
:10A29000522E0062E9CF8E3221F406FDB1C2006475
:10A2A000E3CF8C3611F40068DFCF8836E9F29BEB00
:10A2B000980F933008F05FC00061805E06FD02C019
:10A2C00046E0F42E102F1F73853609F05BC0106432
:10A2D00017FF61C08F2D9BE39F1508F48BE3442487
:10A2E0004394480E27E03501F4E06F0E711CF50130
:10A2F0006081718182819381042DA4010F94959CCA
:10A300005C01F981FC87F0FF03C00DE2F3FF07C099
:10A310000BE211FD04C0012F047012FD00E22C8538
:10A320002C70E22E09F46BC00111D8C2F3E0E12CCD
:10A33000F515A0F483E0E52CE81A13FD08C0B6017A
:10A3400080E290E00F94449EEA94E110F8CF00235D
:10A3500029F0B601802F90E00F94449E3C852EE3B7
:10A36000A22E21E7B22E33FD04C092E4A92E91E77C
:10A37000B92E107122C09BE9980F933008F047C1A5
:10A380000F7E9CCF863611F41068A2CFFF2009F40F
:10A390009FCFFA949DCFE7E02F2DEF1518F427E01B
:10A3A00037E0F32E412C9FCF11118052B60190E07F
:10A3B0000F94449E8FEFA81AB80AF5018491811179
:10A3C000F3CFE11084C25301F6019381F10193FDB3
:10A3D000859193FF81911F01882309F411C2853271
:10A3E00041F493FD859193FF81911F01853209F01E
:10A3F0001CCFB60190E00F94449E3501E4CF17FFC7
:10A400006FC04A0CFC85F4FF04C08A81813309F4D3
:10A410004A9414140CF086C028E0241510F488E047
:10A42000482E85E090E017FF06C0C501B7FE02C0C8
:10A4300090E080E0019601110196FF2031F02F2D70
:10A4400030E02F5F3F4F820F931F5816190619F007
:10A4500014F0E52CE81A812F897011F4E11067C01F
:10A46000002329F0B601802F90E00F94449E13FD45
:10A4700002C0E11063C017FF7CC08501B7FE02C0B7
:10A4800010E000E0C501841991092C016F2D70E0E6
:10A49000EE27FF27E61BF70BFF87EE870F3F10071E
:10A4A00029F4B6018EE290E00F94449EA016B10606
:10A4B0000CF44BC0401651060CF047C0F501E01BF0
:10A4C000F10BE80DF91D8181015011092E853F85A1
:10A4D00002171307E4F1B60190E00F94449EDECF1B
:10A4E00016FD9FCFEF2DF0E0EA15FB0534F03CEFB1
:10A4F000A3163FEFB3060CF010683296E80DF91D75
:10A5000001C0FA94FF2019F082918033D1F317FF34
:10A5100088CF442443944F0CFA141B0431F02CF0E0
:10A52000FA187FCF442443947CCFF12C7ACFB60124
:10A5300080E290E00F94449EEA9490CFB60180E3CD
:10A5400090E00F94449EEA9494CF80E3BDCFA01690
:10A55000B10641F49A81963350F4953319F43C8551
:10A5600034FF05C0B60190E00F94449E2ACF81E3EA
:10A57000F9CF8A81813319F09C859F7E9C87B60133
:10A5800090E00F94449EFF20A9F0B6018EE290E087
:10A590000F94449EF394F394E2E001E00E0FE80D73
:10A5A000F92DF11D8081B60190E00F94449EE02FBB
:10A5B0000F11F3CF85E690E014FF02C085E490E030
:10A5C000B6010F94449EB7FC06C0A114B104C1F4B7
:10A5D000EC85E4FF15C0B194A194B1088DE2B601F9
:10A5E00090E00F94449E80E32AE0A216B10454F454
:10A5F000B60190E00F94449EB601C501C096B4CF59
:10A600008BE2EDCF8F5FFAE0AF1AB108EDCF833662
:10A61000C9F0833771F1833509F05BC03501F2E091
:10A620006F0E711CF501A080B1806F2D70E006FDEA
:10A6300002C06FEF7FEFC5010F94D89D9D878C8777
:10A6400000680DC0350132E0630E711CF501808198
:10A65000898321E030E03D872C8754010F7703FD8B
:10A6600006C02C853D855216130609F0A8F4E52C8A
:10A670002BC0350132E0630E711CF501A080B18062
:10A680006F2D70E006FD02C06FEF7FEFC5010F94E4
:10A69000FD9D9D878C87E2CFB60180E290E00F940C
:10A6A000449E5A94DECFF50107FD859107FF819105
:10A6B0005F01B60190E00F94449EE110EA948C850E
:10A6C0009D8501979D878C87EC85FD85EF2B59F73C
:10A6D00078CE843619F0893609F074C0350107FF49
:10A6E00066C0F4E06F0E711CF5016081718182819A
:10A6F0009381102F1F7697FF08C0909580957095D5
:10A7000061957F4F8F4F9F4F10682AE030E0A40182
:10A710000F946B9FA82EA818BA2C012F16FF0AC001
:10A720000E7FAF1438F414FF04C012FD02C0012FD5
:10A730000E7EBF2C04FFA3C0FE01EA0DF11D808137
:10A74000803309F095C0097EF02FF870EF2E03FDDD
:10A75000A5C000FF9FC0FA2CB51410F4F50CFB182F
:10A7600004FFA2C0B60180E390E00F94449E02FF74
:10A7700009C088E790E001FF02C088E590E0B601DB
:10A780000F94449EAF1408F49BC0AA940A2D10E0C5
:10A790000F5F1F4F080D191DF80182918F01B6013F
:10A7A00090E00F94449E80169106B1F70ACEF2E035
:10A7B0006F0E711CF50160817181072E000C880BF2
:10A7C000990B97CF102F8537A9F41F7E2AE030E030
:10A7D000350117FF44C0F4E06F0E711CF501608174
:10A7E000718182819381A4010F946B9FA82EA81878
:10A7F0001F7792CF197F8F3679F1F0F4883539F1D0
:10A80000F601868197812F960FB6F894DEBF0FBEB2
:10A81000CDBFDF91CF911F910F91FF90EF90DF900F
:10A82000CF90BF90AF909F908F907F906F905F90F0
:10A830004F903F902F900895803739F0883701F777
:10A8400014FD146020E130E0C3CF1061F9CF04FDA6
:10A85000166020E132E0BCCF28E030E0B9CFF2E072
:10A860006F0E711CF5016081718190E080E0BBCFBB
:10A8700002FD02C0B39468CFB394B39465CF802F28
:10A88000867809F461CFF6CFB60180E290E00F94AC
:10A89000449EB394B514C0F3E12C62CFE52CEB18C1
:10A8A000B51408F45DCFF8CF802F867809F46ACF0D
:10A8B0008BE201FF80E207FD8DE2B60190E060CF00
:10A8C000B60180E390E00F94449EFA945BCFB6010A
:10A8D00080E290E00F94449EEA9473CD24E0E12C52
:10A8E000251508F036CD84E026CD20E030E040E8A4
:10A8F0005FEB60917E0270917F0280918002909167
:10A9000081020F94F9A1882321F1E091CB11F091FC
:10A91000CC11E252F04F80818B7F8230D1F480E104
:10A92000EEE7F2E0A5EFB1E101900D928A95E1F733
:10A9300080E090E0A0E8BFEB80937E0290937F02DE
:10A94000A0938002B09381028091E0119091E11177
:10A95000089581E090E0089580E1E3E9F6E0A5EF55
:10A96000B1E101900D928A95E1F70895E6E1F6E7ED
:10A97000833021F0E82FF0E0ED5EF94884910895EE
:10A980008091AF059091B0052091B1053091B2054D
:10A99000821B930B8F7799270895982F9F7083FFC1
:10A9A0000DC080917B00886080937B0080917C004B
:10A9B000887F9770892B80937C00089580917B001D
:10A9C000877FF2CF8091B1059091B2059093B00549
:10A9D0008093AF0581E399E69F938F938091D11186
:10A9E0009091D211A091D311B091D4110196A11DD3
:10A9F000B11DBF93AF939F938F938BE394E69F9387
:10AA00008F9382E494E69F938F930F949E9E8DB7CD
:10AA10009EB70A960FB6F8949EBF0FBE8DBF0895DD
:10AA20000F931F93CF93DF93EC01C60FD71F8C17A3
:10AA30009D0779F08C010F5F1F4F0F94DC9F8F3FB4
:10AA400031F081E0DF91CF911F910F910895C801FE
:10AA5000EECF80E0F7CF682F880F770B8091CB1176
:10AA60009091CC118F51904F0F9433A69C019093ED
:10AA7000F6168093F51681E0232B09F480E0089503
:10AA80008091F5169091F6164AE050E070E060E093
:10AA900001960F94679B862F08958091F5169091EB
:10AAA000F6164AE050E070E060E001960F94679B74
:10AAB000CB0108950F931F93CF93DF938C01862FC3
:10AAC000EA010E942B55882319F10E944D559C01E3
:10AAD00097FF03C0319521953109253631059CF04A
:10AAE0009F938F9384E49DE99F938F9383E996E7E7
:10AAF0009F938F930F949E9E0F900F900F900F90A7
:10AB00000F900F9080E0DF91CF911F910F910895EA
:10AB1000F80180818823B1F3CE01DF91CF911F919D
:10AB20000F910D94DC9F8091F5169091F6164AE0F6
:10AB300050E070E060E001960D94679B60E086E66F
:10AB40009FE00F9400A060E088E69FE00F9400A0D3
:10AB500060E085E69FE00F9400A060E084E69FE05F
:10AB60000F9400A060E082ED9EE00F9400A060E0F2
:10AB70008FEC9EE00D9400A080369105F8F4409192
:10AB8000CB115091CC112091DC0F3091DD0F421789
:10AB9000530739F46091CF117091D0111616170632
:10ABA0006CF0B901680F791FFB01E359FF4F2417BF
:10ABB000350730F481E04E175F0708F480E0089510
:10ABC000EE3EF140F8F06C5F7F4F6E3E714018F43E
:10ABD00049365105B8F483599F4F4817590770F308
:10ABE0004DEE51E0421B530B70E060E0C901825210
:10ABF000904F0F940EA68FB7F8941092DD0F10921D
:10AC0000DC0F8FBF81E008952F923F924F925F92A9
:10AC10006F927F928F929F92AF92BF92CF92DF926C
:10AC2000EF92FF920F931F93CF93DF93CDB7DEB7D1
:10AC3000CC58D2400FB6F894DEBF0FBECDBFCB5874
:10AC4000DD4F688379838A839B83C557D240FE0199
:10AC5000E754FE4F88E2DF011D928A95E9F7E85B31
:10AC6000F1401F0180E991E0DF01FC011D92319765
:10AC7000E9F7C75ADD4F19821882C955D2409E01A3
:10AC80002F513E4FC159DD4F39832883CF56D240D3
:10AC90008E01075A1D4FCE018F5C9D4FC359DD4F6A
:10ACA00099838883CD56D2403C01490140EBA42EC4
:10ACB0004FE0B42E53E2C52ED12CF12CE12CB6017D
:10ACC0000D2C000C880B990B0F946A9AD4016D938C
:10ACD0007D938D939D934D01F801619171918F0149
:10ACE000072E000C880B990B0F946A9AD3016D9371
:10ACF0007D938D939D933D01BFEFEB1AFB0AE6E038
:10AD0000EE16F10409F038C3CB58DD4F28813981A4
:10AD10004A815B81C557D240C159DD4FA881B981B5
:10AD2000CF56D2406D917D918D919C910F948DA3C2
:10AD3000412C512C320118160CF402C3C359DD4FBB
:10AD400008811981CD56D2400C5E1F4FC159DD4F8D
:10AD5000E880F980CF56D240B4E1EB0EF11C6E01D1
:10AD6000EFEDCE1AEDEFDE0A9E012B553E4FCF5888
:10AD7000DD4F39832883C157D240D8014D905D9073
:10AD80006D907C90F7016081718182819381D70100
:10AD90005E914E913E912E917D010F9403A14B0146
:10ADA0005C01F80152914291329122918F01C301CD
:10ADB000B2010F9403A1A50194010F9403A2D6013F
:10ADC0009E938E937E936E936D01CF58DD4FE881F5
:10ADD000F981C157D240B292A29292928292CF58F8
:10ADE000DD4FF983E883C157D240C359DD4F288135
:10ADF0003981CD56D2400217130709F0BECF4E015C
:10AE00003FE6831A3EEF930A5E0183EFA81A8DEFA7
:10AE1000B80A61018101EE24E394F12CD4014D9034
:10AE20005D906D907D904D012D913D914D915C9186
:10AE3000C301B2010F9404A19B01AC010F9404A1C2
:10AE4000F80164A775A786A797A7F1E0EF16F104AC
:10AE500061F0D80198964D925D926D927C929B978D
:10AE6000F8014482558266827782FFEFEF1AFF0A6B
:10AE7000F501208131814281538184E0A80EB11C0B
:10AE800064817581868197810F9403A120E030E071
:10AE900040EC50E40F94A99AD601DC966D937D9313
:10AEA0008D939C93DF97045D1F4FB8E2CB0ED11CAE
:10AEB000E5E0EE16F10409F0B1CF7E01FDE2EF0E00
:10AEC000F11C28E2A22EB12C00EB1FEF24E0220E91
:10AED000311CD7012D913D914D915C91139798961E
:10AEE0006D917D918D919C919B970F9403A22B0165
:10AEF0003C016101C01AD10A88248394912CF60187
:10AF0000E00FF11FEA0DFB1D208131814281538149
:10AF1000C301B2010F94A99A9B01AC01F6016081B3
:10AF20007181828193810F9403A1D6016D937D93EA
:10AF30008D939D936D01BFEF8B1A9B0AE6E08E16F1
:10AF40009104E9F63CE2E30EF11C0852110988E293
:10AF5000A80EB11C08339FEF190709F0BACF1E01E4
:10AF6000F5EB2F0E311C6E0121EBC20ED11C7E01C0
:10AF700037E3E31A3EEFF30A04E010E04801B12C96
:10AF8000A12C412C512C3201F601EA0DFB1DD701F9
:10AF9000AA0DBB1D2D913D914D915C9160817181F8
:10AFA000828193810F94A99A9B01AC01C301B201E4
:10AFB0000F9404A12B013C018FEF881A980A94E0AA
:10AFC000A90EB11CA5E08A169104F1F6A301920125
:10AFD000F10160817181828193810F9403A1D60177
:10AFE0002D913D914D915C910F9403A2F7016083E7
:10AFF00071838283938301501109F8E22F1A31087B
:10B000002CE2C21AD10834E0E31AF1080115110547
:10B0100009F0B4CFCB50DE4F88819981AA81BB81E2
:10B02000C55FD140CF57DD4F88839983AA83BB8307
:10B03000C158D2401E0197E4291A9EEF390A10E048
:10B0400000E0C159DD4FA881B981CF56D240CD90E3
:10B05000DD90ED90FD90C159DD4FB983A883CF56A7
:10B06000D240CB58DD4F288139814A815B81C55759
:10B07000D240C701B6010F94F9A11816B4F0CB580D
:10B08000DD4F288139814A815B81C557D240C15942
:10B09000DD4FE881F981CF56D24060817181828194
:10B0A00093810F948DA387FF18C00430110509F018
:10B0B00030C1CB58DD4F288139814A815B81C5572A
:10B0C000D240CF57DD4F688179818A819B81C158F9
:10B0D000D2400F94F9A187FF1CC1D10114968D9025
:10B0E0009D90AD90BC9017978D919D910D90BC91C6
:10B0F000A02DCF58DD4F88839983AA83BB83C15786
:10B10000D240F801EE0FFF1FEE0FFF1F21E931E0E3
:10B110002C0F3D1FE20FF31F40805180628073802F
:10B12000C359DD4FA881B981CD56D2408D919D91F3
:10B130000D90BC91A02DC358DD4F88839983AA83BD
:10B14000BB83CD57D240A7019601CB58DD4F688114
:10B1500079818A819B81C557D2400F9403A16B01ED
:10B160007C0120E030E040E450E40F9474A4CB571D
:10B17000DD4F688379838A839B83C558D240C35847
:10B18000DD4F288139814A815B81CD57D240C35937
:10B19000DD4FE881F981CD56D24064817581868189
:10B1A00097810F9403A1A30192010F9403A2C758A2
:10B1B000DD4F688379838A839B83C957D240A3017B
:10B1C0009201C301B2010F9404A1CF58DD4F288131
:10B1D00039814A815B81C157D2400F94A99AC757E0
:10B1E000DD4F688379838A839B83C958D240A3014A
:10B1F0009201C501B4010F94A99A9B01AC01C757F4
:10B20000DD4F688179818A819B81C958D2400F9432
:10B2100004A120E030E040EC50E40F9403A29B0135
:10B22000AC01C758DD4F688179818A819B81C957FC
:10B23000D2400F9403A1A70196010F94A99AC75871
:10B24000DD4F688379838A839B83C957D240CF5867
:10B25000DD4F288139814A815B81C157D240C501C8
:10B26000B4010F9403A14B015C0120E030E040ECFD
:10B2700050E4C301B2010F94A99A9B01AC01C5012E
:10B28000B4010F9403A2CB57DD4F288139814A8145
:10B290005B81C558D2400F94A99A4B015C0120E014
:10B2A00030E040E05FE3CF58DD4F688179818A81EB
:10B2B0009B81C157D2400F94A99A2B013C01A70151
:10B2C0009601C701B6010F94A99A9B01AC01C30175
:10B2D000B2010F94A99A9B01AC01C501B4010F946E
:10B2E00004A19B01AC01C758DD4F688179818A8137
:10B2F0009B81C957D2400F9404A1C358DD4F2881C8
:10B3000039814A815B81CD57D2400F9404A12B0132
:10B310003C010F5F1F4FF4E02F0E311CC359DD4F6E
:10B3200028813981CD56D2402C5F3F4FC359DD4F24
:10B3300039832883CD56D2400530110509F081CEDE
:10B34000C301B201C457DD4F0FB6F894DEBF0FBE84
:10B35000CDBFDF91CF911F910F91FF90EF90DF90C4
:10B36000CF90BF90AF909F908F907F906F905F90A5
:10B370004F903F902F900895C5010F94EA9FD801F8
:10B380008D939C93B5E0CB0ED11CE2E0AE0EB11CC8
:10B3900096CC0F931F93CF9320919412213079F57F
:10B3A0008C0180E50E942B55882349F10E9440556D
:10B3B000C82F853020F5013C82E0180749F0023C97
:10B3C000124069F08C2FCF911F910F910D94AB6AB1
:10B3D00060E08C2FCF911F910F910D94EE6A8EEC4F
:10B3E0009EE00F94DC9F882351F00F94B453882380
:10B3F00031F08C2FCF911F910F910D946B6BCF91EA
:10B400001F910F9108958F929F92AF92BF92CF920A
:10B41000DF92EF92FF920F931F93CF93DF930091F0
:10B42000F5161091F6160F5F1F4F68018FEFC81ABF
:10B43000D80AD801DC918D2F90E00F946D9D7C018E
:10B44000892B01F5DD3201F56801B2E0CB0ED11C8C
:10B45000F801D181C1E086010150110943E050E0BB
:10B460006AE476E7C8010F94A39D892BC1F460E0DC
:10B4700070E080E89FEFC111DBC060E070E080E821
:10B480009FE7D6C08601D1CFDB3239F46801F2E004
:10B49000CF0ED11CD8011196DC91C0E0DCCF43E087
:10B4A00050E067E476E7C8010F94A39D892B09F467
:10B4B000CCC0F60110E000E020E030E0A9016F010F
:10B4C000D053DA3060F5BC2E6894B1F88C2F8870B8
:10B4D000C2FF09C0811102C00F5F1F4F3196D60114
:10B4E000DC91CB2DECCF882311F001501109A5E0A0
:10B4F000B0E00F9471A09B01AC01220F331F441FD9
:10B50000551F2D0F311D411D511D2839B9E93B072C
:10B510004B07B9E15B0710F3C660BC2EDFCFDE3FFF
:10B5200031F4C3FD33C0BC2E6894B3F8D7CFD53304
:10B5300069F580818D3231F4C061BF016E5F7F4F4C
:10B54000818105C0BF018B32C9F36F5F7F4F80538C
:10B550008A30E0F4FB01B0E8EB16BCE0FB065CF4DB
:10B56000B701660F771F660F771FE60EF71EEE0C0A
:10B57000FF1CE80EF11C819180538A3060F3C4FFF8
:10B5800003C0F194E194F1080E0D1F1DCA01B90129
:10B590000F94689AC370C33009F490584B015C0152
:10B5A00020E030E0A9010F94F9A1882309F43EC0FE
:10B5B000C3E4D6E717FF05C0119501951109CBE249
:10B5C000D6E76E01E8E1CE1AD10880E2E82EF12C30
:10B5D0000DC0FE0125913591459154910E191F0919
:10B5E000C501B4010F94A99A4B015C01D501C401B6
:10B5F0000E151F0574F72497F594E794CC16DD0615
:10B60000A9F78A2F880F8B2F881F8F3F49F020E0E2
:10B6100030E0A901C501B4010F94F9A1811106C060
:10B6200082E290E09093F9168093F816C501B40178
:10B63000DF91CF911F910F91FF90EF90DF90CF900E
:10B64000BF90AF909F908F90089560E070E080EC85
:10B650009FE7EECF2F923F924F925F926F927F9231
:10B660008F929F92AF92BF92CF92DF92EF92FF9212
:10B670000F931F93CF93DF93CDB7DEB7A1970FB68C
:10B68000F894DEBF0FBECDBF84EC92E09D8F8C8F0F
:10B6900085EF282E81E1382E03E916E091E09A8F9C
:10B6A000198EEC8DFD8D8191FD8FEC8F0E942B55B5
:10B6B000E82E882309F454C1F090EB11FA8DFF2293
:10B6C0000E94035A2B013C01F801408251826282A0
:10B6D0007382F98DF33009F045C0DD24D394F11065
:10B6E00001C0D12C8090100290901102A090120203
:10B6F000B090130220E030E040E85FE3C501B40100
:10B700000F94F9A1882359F1F11015C0209101126D
:10B71000309102124091031250910412C301B20100
:10B720000F9403A160939F067093A0068093A106D7
:10B730009093A206DE2CA501940160919F06709162
:10B74000A0068091A1069091A2060F94A99A6093F9
:10B750009F067093A0068093A1069093A206D11035
:10B7600003C05FC0FF2089F0F10120813181428157
:10B770005381F80160817181828193810F9404A1CA
:10B78000F8016083718382839383F98DF230D9F558
:10B7900080918903823009F0EEC08CE0E0EAF2E0AB
:10B7A000DE011D9601900D928A95E1F78CE0ECEA9E
:10B7B000F2E0DE01119601900D928A95E1F7C090BA
:10B7C0009B06D0909C06E0909D06F0909E0620E09F
:10B7D00030E0A901C701B6010F94F9A187FF52C05B
:10B7E000CE0101967C01D12CF7016191719181917B
:10B7F00091917F010F9475A28D2D0F948F21D39479
:10B80000F3E0DF12F1CFF98DFF5FF98F8A8D880F9A
:10B810008A8F94E0290E311C0C5F1F4FF43009F021
:10B8200040CF86E40E942B55882399F00E94035A4A
:10B830006B017C0120E030E0A9010F948DA3181664
:10B8400044F4C0927A02D0927B02E0927C02F092A1
:10B850007D02A1960FB6F894DEBF0FBECDBFDF917B
:10B86000CF911F910F91FF90EF90DF90CF90BF90FD
:10B87000AF909F908F907F906F905F904F903F9090
:10B880002F90089520E030E048E453E4C701B6016A
:10B890000F948DA31816A4F4CE010D967C01D12C23
:10B8A000F70161917191819191917F010F9475A23E
:10B8B0008D2D0F948F21D394F3E0DF12F1CFA3CF1E
:10B8C000CE01019699A388A3FE013D96FF8FEE8FCE
:10B8D0001B8EE8A1F9A1C190D190E190F190F9A35C
:10B8E000E8A3EE8DFF8D6191719181919191FF8F10
:10B8F000EE8FA70196010F9403A120E030E048E409
:10B9000053E40F9403A24B015C0120919B063091FC
:10B910009C0640919D0650919E060F94A99A2B017A
:10B920003C0120E030E0A901C501B4010F94A99ABF
:10B930009B01AC01C701B6010F9403A19B01AC01AF
:10B94000C301B2010F9404A10F9475A28B8D0F94C3
:10B950008F21FB8DFF5FFB8FF33009F0BACF53CF00
:10B96000F10180819181A281B381F801808391836B
:10B97000A283B38348CFEA8DEE0FEA8FF4E02F0E57
:10B98000311C0C5F1F4F83E0898F8BCE60910017B5
:10B990007091011790E08A3020F0895A9F4F0D94E2
:10B9A000449EC096FCCF2FB784FF1EC0F8949091A0
:10B9B00005019260909305012FBF2FB785FF19C035
:10B9C000F894909105019160909305012FBF86FF37
:10B9D00015C0459A87FF14C0469A739A85E08A95E8
:10B9E000F1F7000073980895F894909105019D7FF8
:10B9F000E1CFF894909105019E7FE6CF4598EACF7C
:10BA00004698EBCF0F931F93CF93DF93C82FD62F7A
:10BA10008A0160FF15C05F9A8AE18A95F1F700C03C
:10BA20008C2F0E94D35CD1FD04C08C2F82950E9484
:10BA3000D35CC801DF91CF911F910F910C94DEBFB1
:10BA40005F98EACFCF92DF92EF92FF92CF93DF938E
:10BA5000EC016A017B010F94E49F6F3F7F4F8F4F92
:10BA60009F4F59F4B701A601CE01DF91CF91FF900E
:10BA7000EF90DF90CF900D9432A0DF91CF91FF90A7
:10BA8000EF90DF90CF9008957F928F929F92AF9228
:10BA9000BF92CF92DF92EF92FF920F931F93CF93BB
:10BAA000DF93CDB7DEB760970FB6F894DEBF0FBE59
:10BAB000CDBF5C016B01742E81E0809378021F93EF
:10BAC0000F931F922F938DE793E69F938F930F947D
:10BAD0009E9E81E40E942B550F900F900F900F9027
:10BAE0000F900F90882389F08091F5169091F616AB
:10BAF000FC012181283709F056C040E150E070E098
:10BB000060E002960F94679B5B0183E40E942B55D3
:10BB1000882309F44DC00E9493554B017501CA1446
:10BB2000DB0408F47601C4018E0D9F1DC816D906EA
:10BB300018F08E159F0518F446018E189F0888E5A9
:10BB40000E942B55882309F471C02091F51630917D
:10BB5000F6162F5F3F4FCE0101965C01DC01D12C20
:10BB6000C12CF90180812F5F3F4F8823B9F190E10B
:10BB7000C916D10499F18032A1F38A3079F190EDA0
:10BB8000980F9A30C8F48295807F9F012E5F3F4FB7
:10BB9000918140ED490F4A30B8F4842B8D93EFEF3B
:10BBA000CE1ADE0ADECF0E94035A0F9475A2ACCFE4
:10BBB00088248A94982CB2CF9FE9980F963058F435
:10BBC0008295807F8057E1CF4FE9490F463018F4C6
:10BBD0009755892BE3CFD194C194D108912C812C16
:10BBE000C814D90491F0F50161915F01C4018E0D73
:10BBF0009F1DF1E07F1631F0FC016083FFEF8F1A8B
:10BC00009F0AEECF0F9424A0F9CFFF92EF921F93DB
:10BC10000F939F928F9283E593E69F938F930F9458
:10BC20009E9E0FB6F894DEBF0FBECDBF472DB40168
:10BC3000C70160960FB6F894DEBF0FBECDBFDF918F
:10BC4000CF911F910F91FF90EF90DF90CF90BF9019
:10BC5000AF909F908F907F900D94E55280E1E5EF3B
:10BC6000F1E1A0E9B2E001900D928A95E1F78091AF
:10BC70008E0290918F029093F4118093F311809132
:10BC8000F1119091F2119093F0118093EF11809146
:10BC9000ED118093EC118091EB1183FB882780F9E3
:10BCA0008093EA118091E9118093E8110895CF9370
:10BCB000DF938AEF95E10E943B7088E394E1892B42
:10BCC00051F0CAE0D5E1A397CE010E943B7084E118
:10BCD000C833D807C1F785E194E10E943B7080EF3B
:10BCE00093E1DF91CF910C943B70CF93DF93C5EF3D
:10BCF000D1E120E030E048EC51E46C857D858E8513
:10BD00009F850F9404A16C877D878E879F8763E34F
:10BD100073E383E590E4DF91CF910D94708460E04C
:10BD200085EA9FE00F9400A060E08FE79CE00F940D
:10BD300000A080E090E0A0E8BFEB80937E029093AB
:10BD40007F02A0938002B093810282E08093790207
:10BD50001092E71108958091EF119091F0112091C8
:10BD6000F1113091F2112817390771F09093F21107
:10BD70008093F11181E0809399030F94740F0F94D5
:10BD8000984E82E08093990308958091E71188236B
:10BD900041F080918E0290918F029093F4118093E4
:10BDA000F3110895CF92DF92EF92FF92C090CA04F0
:10BDB000D090CB04E090CC04F090CD048091C904E5
:10BDC000882309F44EC020E030E0A901C701B60184
:10BDD0000F948DA318160CF044C02BED3FE049E4FE
:10BDE00050E4C701B6010F94A99AA70196010F94D8
:10BDF000A99A20E030E040E85EE30F94A99A9B0105
:10BE0000AC0160E070E080E89FE30F9403A26B0157
:10BE10007C016091590270915A0264367105A1F05B
:10BE2000072E000C880B990B0F946A9A2AE037EDC5
:10BE300043E25CE30F94A99A9B01AC01C701B601F0
:10BE40000F94A99A6B017C01C0921002D09211024A
:10BE5000E0921202F0921302FF90EF90DF90CF90E9
:10BE60000895C12CD12C80E8E82E8FE3F82ED1CF95
:10BE70008F929F92AF92BF92CF92DF92EF92FF92FA
:10BE800081EF9FE00F94B7486B017C018DEE9FE03E
:10BE90000F94B7484B015C010F94661C2CE330E013
:10BEA00040E050E00F944FA0BA01A901480D591D80
:10BEB0006A1D7B1D8DEE9FE00F9412A06091840699
:10BEC00070918506809186069091870628EE33E072
:10BED00040E050E00F944FA0BA01A9014C0D5D1D48
:10BEE0006E1D7F1D81EF9FE00F9412A00F943B20E9
:10BEF000109284061092850610928606109287068C
:10BF000080919412813081F460919812709199120D
:10BF100090E080E00F949F4810929912109298122E
:10BF200010929B1210929A12FF90EF90DF90CF9098
:10BF3000BF90AF909F908F9008958091E9111F92CC
:10BF40008F93809140031F928F93E5E8F3E0428145
:10BF500053812CE3249FC001259F900D11249F93B2
:10BF60008F9340815181249FC001259F900D112402
:10BF70009F938F9384E194E69F938F930F949E9E5B
:10BF80008DB79EB70A960FB6F8949EBF0FBE8DBFB1
:10BF900008958AE493E00D94A11120E030E040E799
:10BFA00052E40F9403A208951092770240913B034C
:10BFB00050913C0360913D0370913E0340937A029F
:10BFC00050937B0260937C0270937D0290938F026A
:10BFD00080938E028AE493E00D94A1111F93CF9376
:10BFE000DF93182F80917A0290917B02A0917C02BE
:10BFF000B0917D0280933B0390933C03A0933D035B
:10C00000B0933E03C0918E02D0918F0284E690E0FF
:10C0100090938F0280938E028AE493E00F94A11193
:10C0200010937702CE01DF91CF911F910895CF92A7
:10C03000DF92EF92FF920F931F93CF93DF9390E0E5
:10C04000EC01CC0FDD1FCC0FDD1FFE01EB59F948D1
:10C050002591359145915491FE01E657FB4FC080E3
:10C06000D180E280F3808E010B501E4EC701B601D5
:10C070000F9404A1F8016083718382839383FE018E
:10C08000E75AF94825913591459154918E010C5DFF
:10C090001D4FC701B6010F9404A1F801608371839D
:10C0A00082839383FE01E35BF948259135914591A5
:10C0B0005491C85EDD4FC701B6010F9404A1688397
:10C0C00079838A839B83DF91CF911F910F91FF909A
:10C0D000EF90DF90CF90089540E050E0BA018DEEF0
:10C0E0009FE00F9412A040E050E0BA0181EF9FE082
:10C0F0000F9412A00E949E5570E060E085E09FE0E2
:10C100000F941EA070E060E083E09FE00F941EA0FB
:10C1100070E060E081E09FE00F941EA070E060E0BE
:10C120008FEF9EE00F941EA070E060E083ED9EE034
:10C130000F941EA070E060E080ED9EE00F941EA0C2
:10C1400040E050E0BA0188EA9CE00D9412A0F89417
:10C1500088E19FE00FB6F894A895809360000FBE29
:10C1600090936000FFCF85EA9FE00F94DC9F91E001
:10C17000811101C090E0892F089580919B03811166
:10C1800006C081E090915903923009F080E0089553
:10C1900080916A1381110AC08091D511811106C066
:10C1A00081E090915903913009F080E00895CF9398
:10C1B000DF93C0910512C1111FC080910612811139
:10C1C0001CC00E94BD60811118C0D091C80DD43030
:10C1D00061F48091F1119091F211892B91F4809189
:10C1E000ED119091EE11892B61F40E94C860C82F67
:10C1F000811103C0C1E0D111C0E08C2FDF91CF913C
:10C200000895C1E0FACF0E94D760882389F020E02A
:10C2100030E040E050E46091FD117091FE1180919A
:10C22000FF11909100120F94F9A1881F8827881F91
:10C2300008950E94C860811118C00E94BD608111DC
:10C2400014C08091E711811110C08091C80D811137
:10C250000BC080919512811107C080910512811148
:10C2600004C080910612089581E0089580E1E5EF11
:10C27000F1E1A3E9B6E001900D928A95E1F7089506
:10C280004F925F926F927F928F929F92AF92BF92E6
:10C29000CF92DF92EF92FF920F931F93CF93DF9392
:10C2A00000D000D01F921F92CDB7DEB72091E711CA
:10C2B000222309F473C120919C03223009F46EC13A
:10C2C00020919C03213011F410929C032B013C011E
:10C2D0001092E9111091EC1160918A0370918B0317
:10C2E00080918C0390918D030F947CA2611731F0A3
:10C2F000812F90E09093EE118093ED110E94AB5E40
:10C300008091E8118093E9119091EB118091EA11ED
:10C3100081958927887089278093EB11A301920169
:10C3200060919C0270919D0280919E0290919F026B
:10C330000F9403A16D837E838F839887CE0105962A
:10C340000F94C8741092400220E030E040E85FEBA8
:10C35000609190027091910280919202909193026B
:10C360000F94F9A1811120C08091F5119091F611DF
:10C37000A091F711B091F8118093900290939102DF
:10C38000A0939202B09393028091F9119091FA11C7
:10C39000A091FB11B091FC118093940290939502AF
:10C3A000A0939602B0939702A301920160919C0220
:10C3B00070919D0280919E0290919F020F9403A123
:10C3C00069837A838B839C83E090FD11F090FE114A
:10C3D0000091FF111091001220919402309195026A
:10C3E0004091960250919702609190027091910253
:10C3F00080919202909193021F921F921F921F921E
:10C40000E2E68E2EE7E29E2EE6E7AE2EE2E4BE2EB8
:10C41000FE0131966F010F942275A3019201609184
:10C420009C0270919D0280919E0290919F020F94B8
:10C4300003A169837A838B839C83E0909802F090B8
:10C44000990200919A0210919B02209194023091DE
:10C4500095024091960250919702609190027091DE
:10C46000910280919202909193021F921F921F92CB
:10C470001F920F942275E0909802F090990200911B
:10C480009A0210919B022091940230919502409162
:10C490009602509197026091900270919102809162
:10C4A0009202909193021F921F921F921F92812CD1
:10C4B000912CF8EEAF2EF2E4BF2EACE9CA2EA2E02A
:10C4C000DA2E0F9422750F94422211E0109340024D
:10C4D0006091E2117091E31190E080E00F94689A0E
:10C4E00060937A0270937B0280937C0290937D022A
:10C4F0008091F3119091F41190938F0280938E02AA
:10C5000080E1E0E9F2E0A5EFB1E101900D928A95BA
:10C51000E1F70E943661809179020FB6F894DEBF90
:10C520000FBECDBF811151C06091D8117091D9114A
:10C530008091DA119091DB1160937E1670937F16D3
:10C5400080938016909381160F94F6438091D811B2
:10C550009091D911A091DA11B091DB118093DC1187
:10C560009093DD11A093DE11B093DF1110936A1345
:10C5700060E085EA9FE00F9400A060E08FE79CE018
:10C580000F9400A087E69BE60E9465E682E0809318
:10C5900079021092E71181E08093AC0D28960FB6D6
:10C5A000F894DEBF0FBECDBFDF91CF911F910F91E9
:10C5B000FF90EF90DF90CF90BF90AF909F908F90C3
:10C5C0007F906F905F904F900895813089F68091B1
:10C5D000D8119091D911A091DA11B091DB1180930B
:10C5E000D1119093D211A093D311B093D411109282
:10C5F000DB0F1092DA0F0E94E254BACF3F924F92B3
:10C600005F926F927F928F929F92AF92BF92CF92E2
:10C61000DF92EF92FF920F931F93CF93DF933090AF
:10C62000DC16332009F480C08B01EC0131FE54C0CC
:10C6300088809980AA80BB80FB01C080D180E28085
:10C64000F3802091B1163091B2164091B3165091FB
:10C65000B416C501B4010F94A99A2B013C01209195
:10C66000B5163091B6164091B7165091B816C7015D
:10C67000B6010F94A99A9B01AC01C301B2010F94BA
:10C6800004A12B013C012091A9163091AA164091DA
:10C69000AB165091AC16C501B4010F94A99A4B0189
:10C6A0005C012091AD163091AE164091AF165091BD
:10C6B000B016C701B6010F94A99A9B01AC01C50140
:10C6C000B4010F9404A1688379838A839B83F80162
:10C6D000408251826282738230FE26C02091D4163D
:10C6E0003091D5164091D6165091D7166881798130
:10C6F0008A819B810F9404A1688379838A839B83B9
:10C700002091D8163091D9164091DA165091DB1647
:10C71000F80160817181828193810F9404A1F801F5
:10C720006083718382839383DF91CF911F910F91F7
:10C73000FF90EF90DF90CF90BF90AF909F908F9041
:10C740007F906F905F904F903F9008952F923F920F
:10C750004F925F926F927F928F929F92AF92BF9211
:10C76000CF92DF92EF92FF920F931F93CF93DF93BD
:10C7700000D000D01F921F92CDB7DEB78C011B01F5
:10C78000FC0180819181A281B38189839A83AB83EB
:10C79000BC83FB0180819181A281B3818D839E83C3
:10C7A000AF83B887BE016B5F7F4FCE0101960E94B9
:10C7B000FE62C980DA80EB80FC8020E030E0A901D5
:10C7C000C701B6010F94F9A187FF35C019821A82FB
:10C7D0001B821C82FF24F3948D809E80AF80B884DE
:10C7E00020E030E040E850ECC501B4010F94F9A11D
:10C7F00087FF35C080E090E0A0E8B0EC8D839E8399
:10C80000AF83B887CD80DE80EF80F88489809A80FE
:10C81000AB80BC807090DC1671104CC0F801808237
:10C820009182A282B382F101C082D182E282F3823C
:10C83000FF24F39425C020E030E04AE753E4C70129
:10C84000B6010F948DA3F12C181634F680E090E019
:10C85000AAE7B3E489839A83AB83BC83BBCF20E090
:10C8600030E042E553E4C501B4010F948DA31816DE
:10C870002CF480E090E0A2E5B3E4C0CFF110C2CF89
:10C880008F2D28960FB6F894DEBF0FBECDBFDF9177
:10C89000CF911F910F91FF90EF90DF90CF90BF90BD
:10C8A000AF909F908F907F906F905F904F903F9050
:10C8B0002F90089570FE1CC02091D4163091D5168B
:10C8C0004091D6165091D716C501B4010F9403A11B
:10C8D0004B015C012091D8163091D9164091DA169F
:10C8E0005091DB16C701B6010F9403A16B017C01C7
:10C8F00071FE9ECF2091C4163091C5164091C61688
:10C900005091C716C501B4010F94A99A2B013C019F
:10C910002091C8163091C9164091CA165091CB1675
:10C92000C701B6010F94A99A9B01AC01C301B201E2
:10C930000F9404A1F8016083718382839383209113
:10C94000CC163091CD164091CE165091CF16C50120
:10C95000B4010F94A99A4B015C012091D01630913B
:10C96000D1164091D2165091D316C701B6010F943B
:10C97000A99A9B01AC01C501B4010F9404A1F10176
:10C98000608371838283938353CFCF92DF92EF9240
:10C99000FF92CF93DF93EC01BC016C5F7F4F0E944D
:10C9A000A663C0902C02D0902D02E0902E02F09051
:10C9B0002F02A7019601688579858A859B850F944A
:10C9C000F9A187FF04C0C886D986EA86FB86C09095
:10C9D0002002D0902102E0902202F0902302A701D1
:10C9E0009601688579858A859B850F948DA3181695
:10C9F00024F4C886D986EA86FB86DF91CF91FF9022
:10CA0000EF90DF90CF9008952F923F924F925F92D8
:10CA10006F927F928F929F92AF92BF92CF92DF924E
:10CA2000EF92FF920F931F93CF93DF93CDB7DEB7B3
:10CA3000A2970FB6F894DEBF0FBECDBF1C0183E9ED
:10CA400096E00E94C5648AE493E00F94A11140909F
:10CA5000F5115090F6116090F7117090F811C09098
:10CA60009306D0909406E0909506F0909606A70164
:10CA70009601C301B2010F94F9A181113FC0209129
:10CA80009706309198064091990650919A066091C8
:10CA9000F9117091FA118091FB119091FC110F9492
:10CAA000F9A181112BC020E030E040E752E4609111
:10CAB0007A0270917B0280917C0290917D020F94AA
:10CAC00003A20F943D840E94AC54A2960FB6F89432
:10CAD000DEBF0FBECDBFDF91CF911F910F91FF90B1
:10CAE000EF90DF90CF90BF90AF909F908F907F900E
:10CAF0006F905F904F903F902F90089560918E02BD
:10CB000070918F02072E000C880B990B0F946A9A74
:10CB100020917A0230917B0240917C0250917D02FB
:10CB20000F94A99A2EE333EC4EE259E30F94A99A9D
:10CB30006F83788789879A8780919C12882309F46C
:10CB40000FC1A3019201C701B6010F9403A12B01EC
:10CB50003C012091F9113091FA114091FB11509153
:10CB6000FC116091970670919806809199069091BA
:10CB70009A060F9403A16B877C878D879E87C301DC
:10CB8000B2019F772B853C854D855E855F770F943D
:10CB900004A16B017C0120E030E0A9010F948DA37A
:10CBA00018160CF0DDC020E030E040EF51E4C70182
:10CBB000B6010F9403A20F94E2A10F947CA27E838E
:10CBC0006D836230710508F4CBC02114310409F47F
:10CBD000C7C02091FD113091FE114091FF1150917D
:10CBE000001260919B0670919C0680919D06909129
:10CBF0009E060F9403A16F87788B898B9A8B209167
:10CC0000011230910212409103125091041260916E
:10CC10009F067091A0068091A1069091A2060F94A4
:10CC200003A16B8B7C8B8D8B9E8BAD81BE81CD01E7
:10CC3000B0E0A0E08F8F98A3A9A3BAA32D813E8175
:10CC40002216330608F08CC0B10190E080E00F940A
:10CC5000689A6B017C016F8D78A189A19AA10F94CC
:10CC6000689A9B01AC01C701B6010F9403A26B0146
:10CC70007C01AC019B016B897C898D899E890F9415
:10CC8000A99A9B01AC0160910112709102128091EE
:10CC90000312909104120F9404A169837A838B8309
:10CCA0009C83A70196016F85788989899A890F9459
:10CCB000A99A2091FD113091FE114091FF115091E0
:10CCC00000120F9404A16F8B788F898F9A8FA70120
:10CCD00096016B857C858D859E850F94A99A209100
:10CCE000F9113091FA114091FB115091FC110F9400
:10CCF00004A16B8F7C8F8D8F9E8FA7019601C3013E
:10CD0000B2010F94A99A2091F5113091F61140913A
:10CD1000F7115091F8110F9404A13F922F92A5EFB3
:10CD2000B1E1BF93AF938F809884A984BA84DE0168
:10CD300011966D01EF88F88C098D1A8D2B8D3C8D25
:10CD40004D8D5E8D0F9422750F900F900F900F9068
:10CD50008091AC0D8111B7CEBFEF2B1A3B0A6ECF7D
:10CD6000E0909B06F0909C0600919D0610919E0617
:10CD700020919706309198064091990650919A0615
:10CD80006091930670919406809195069091960615
:10CD90001F921F92E5EFF1E1FF93EF938F8098844C
:10CDA000A984BA84EFE9CE2EE6E0DE2E0F94227538
:10CDB0000F900F900F900F9086CECF92DF92EF9250
:10CDC000FF92CF93C090FD11D090FE11E090FF1123
:10CDD000F0900012A70196010F9404A16093FD1139
:10CDE0007093FE118093FF119093001283B1909184
:10CDF000A506911102C084FF26C085EF91E10E9433
:10CE0000C56460914E0470914F04809150049091DC
:10CE100051040F9470840F944222A70196016091EF
:10CE2000FD117091FE118091FF11909100120F94ED
:10CE300003A16B017C01C701B601CF91FF90EF9078
:10CE4000DF90CF90089515980F94422281E00F94BF
:10CE50007A2CC82F65E575E585E591E40F9470841B
:10CE60000F94422282E00F942E22A70196010F9484
:10CE700003A16B017C018C2F0F947A2CDCCF8F9255
:10CE80009F92AF92BF92CF92DF92EF92FF924B01AF
:10CE90005C01C090FD11D090FE11E090FF11F09068
:10CEA0000012AC019B01C701B6010F948DA387FF4F
:10CEB00011C0A5019401C701B6010F9403A19F778A
:10CEC000FF90EF90DF90CF90BF90AF909F908F90AA
:10CED0000C94DD66FF90EF90DF90CF90BF90AF9005
:10CEE0009F908F9008952F923F924F925F926F92F2
:10CEF0007F928F929F92AF92BF92CF92DF92EF92EA
:10CF0000FF920F931F93CF93DF9300D01F921F9236
:10CF1000CDB7DEB7D82E2A013B01322EE982FA8244
:10CF20000B831C830F94422281E080930512FC2C1A
:10CF3000E32CD31010C0ED2CDC100DC060E070E0CD
:10CF400080EA90E40E943F67FF24F394EE24E39488
:10CF50002224239401C02D2C0F945C8F80919C126D
:10CF60008D8310929C1282E00F942E226093FD110B
:10CF70007093FE118093FF1190930012F1100F94A3
:10CF80000B8B81E00E94EE5F8C010E943661109253
:10CF90007A0210927B0210927C0210927D02222073
:10CFA00019F080E00F94BC53EE2019F081E00F944B
:10CFB000BC53DD20E9F04114510461047104C1F057
:10CFC000C301B2010F946A9A9B01AC0160918A047B
:10CFD00070918B0480918C0490918D040F9404A126
:10CFE0006093F5117093F6118093F7119093F811F7
:10CFF000332001F189819A81AB81BC810097A10521
:10D00000B105C1F0BC01CD010F946A9A9B01AC013E
:10D0100060918E0470918F0480919004909191049E
:10D020000F9404A16093F9117093FA118093FB118E
:10D030009093FC11FF2009F499C060E070E080EA51
:10D0400090E40E943F678091A306811102C00F9473
:10D05000BC538091A406811103C081E00F94BC539E
:10D060000F94C18FE0E5F8E885919591A591B49171
:10D07000ECE4F8E8459155916591749140939306DD
:10D080005093940660939506709396068093970646
:10D0900090939806A0939906B0939A0667E976E074
:10D0A00083E996E00E94FE620F94238F20E030E037
:10D0B00040E850EC6091970670919806809199062F
:10D0C00090919A060F94F9A187FF0CC080E090E040
:10D0D000A0E8B0EC8093970690939806A0939906E9
:10D0E000B0939A0680E090E0A6E1B3E480937A02E0
:10D0F00090937B02A0937C02B0937D021092770202
:10D100000F94308360917A0270917B0280917C024F
:10D1100090917D020F943D840F944222809193065A
:10D1200090919406A0919506B09196068093F51182
:10D130009093F611A093F711B093F8118091970690
:10D1400090919806A0919906B0919A068093F91152
:10D150009093FA11A093FB11B093FC1181E080939E
:10D1600077020F94962C82E00F94BC53CC20E9F008
:10D1700081149104A104B104C1F0C501B4010F945C
:10D180006A9A9B01AC016091920470919304809122
:10D190009404909195040F9404A16093FD117093F1
:10D1A000FE118093FF11909300120F943083C801F9
:10D1B0000E94D45F0F94962C0F94C18F0F945F8DB3
:10D1C000D11007C0311005C08B8D811102C0CC2059
:10D1D00039F1F11025C09D81992311F181E08093EF
:10D1E0009C120F942E226B017C0180E00F942E2262
:10D1F000A70196010F9408609B01AC016091FD119D
:10D200007091FE118091FF11909100120F9403A173
:10D210006093FD117093FE118093FF1190930012A3
:10D2200084E10F94FF970F944222109205120F9001
:10D230000F900F900F900F90DF91CF911F910F9152
:10D24000FF90EF90DF90CF90BF90AF909F908F9026
:10D250007F906F905F904F903F902F900895E3E301
:10D26000F3E09FE781918F3731F0DF01119787FF5E
:10D2700007C08F778C9383E0EB33F80799F7089515
:10D280009C93F9CF90915B02981710F480935B0206
:10D2900080915C02882339F0E091D203F091D303AE
:10D2A000309709F019940895CF93DF93CDB7DEB787
:10D2B000AE014A5F5F4FFA0161917191AF0180EC5D
:10D2C00093E00F94239FDF91CF91089560EC73E07A
:10D2D0000D94749E60EC73E0082E000C990B0D9475
:10D2E000449ECF93C82FC15020F080E20E946A690B
:10D2F000FACFCF910895CF93C82F862F643008F0CE
:10D3000083E0809332030E94B6548C0F80933103E4
:10D3100044E650E060E08068CF910C94025DCF93CA
:10D32000DF93EA010E947B6960EC73E0CE01DF913C
:10D33000CF910D94749ECF93C42F0E947B6960ECB3
:10D3400073E08C2FCC0F990BCF910D94449E60E02D
:10D3500080E00E947B6910923103089540E456E01A
:10D3600060E081E00E94025D10923203109231036E
:10D3700048E050E06FE770E083E393E00D940EA681
:10D3800090915C02981709F180935C028823E9F080
:10D3900010920705109206051092110681EB93E09A
:10D3A0000F94A1110F94740F6150710981099109B3
:10D3B00060939303709394038093950390939603E3
:10D3C0000E94AE6982E00C9442690895CF93C82F01
:10D3D000109232031092310348E050E06FE770E0A2
:10D3E00083E393E00F940EA644E951E162E080E309
:10D3F0000E94025D46E950E062E080E30E94025D27
:10D4000046E950E062E080E30E94025D46E950E0B8
:10D4100062E080E20E94025D8091CE0344E650E02B
:10D4200060E080620E94025D84E08093300344E605
:10D4300050E060E08CE00E94025DC1110E94AE6984
:10D4400044E650E060E086E0CF910C94025D81E01C
:10D450000C94E669CF92DF92FF920F931F93CF93C4
:10D46000DF9300D000D01F921F92CDB7DEB78A3075
:10D47000D9F480913203843018F08FEF8093320317
:10D48000609132036F5F80E00E947B6928960FB63F
:10D49000F894DEBF0FBECDBFDF91CF911F910F91EA
:10D4A000FF90DF90CF90089590E8980F44E650E009
:10D4B00061E09A3408F5482F4058550B9A0196E0E0
:10D4C000929FA001939F500D1124FA01E45AFB484A
:10D4D000F490E3E3F3E030E020E09FEF6191782FF8
:10D4E00076277F7789F4F901ED5CFC4F8083F22E7B
:10D4F00044E650E061E08F2D0E94025D809131038F
:10D500008F5F80933103C2CF6F3709F03CC0F901C0
:10D51000ED5CFC4F8083922FF92EFA01E95AFB480B
:10D520008E010F5F1F4FD801959188E0182E10FED5
:10D5300005900294802D9795881F8D931A94B9F7C2
:10D54000BF2DE8E0BE02C001112444E650E060E0D7
:10D5500080640E94025D6E01F9E0CF0ED11C44E6AA
:10D5600050E061E0D8018D918D010E94025DC016EE
:10D57000D106A9F78091310344E650E060E080686D
:10D580000E94025DB5CF67FF922F2F5F3F4F28307B
:10D59000310509F0A3CF9F3F09F0BECFA9CF8F92ED
:10D5A0009F92AF92BF92EF92FF920F931F93CF93F0
:10D5B000DF93CDB7DEB7A0970FB6F894DEBF0FBEEE
:10D5C000CDBF611571058105910599F480E3A096A1
:10D5D0000FB6F894DEBF0FBECDBFDF91CF911F9184
:10D5E0000F91FF90EF90BF90AF909F908F900C9411
:10D5F0002A6A00E0842E912CB12CA12C9E012F5F71
:10D600003F4F7901A50194010F944FA0F701E00F5E
:10D61000F11D6083B901CA010F5F611571058105B4
:10D62000910581F70E0D1F2D111DE016F10659F021
:10D63000F80182918F018A3020F4805D0E942A6A6D
:10D64000F4CF895CFBCFA0960FB6F894DEBF0FBE77
:10D65000CDBFDF91CF911F910F91FF90EF90BF90C1
:10D66000AF909F908F900895CF92DF92EF92FF92AC
:10D670006B017C01F7FE0BC08DE20E942A6AF094D8
:10D68000E094D094C094C11CD11CE11CF11C4AE070
:10D69000C701B601FF90EF90DF90CF900C94CF6A56
:10D6A0000F931F93CF938C01C62FCC2359F0F80111
:10D6B0002491222339F00F5F1F4F84910E942A6A20
:10D6C000C150F3CF8C2F0E9471698C2FCF911F9185
:10D6D0000F9108950F931F93CF938C01C62FCC23E6
:10D6E00049F0F80181918F01882321F00E942A6A74
:10D6F000C150F5CF8C2F0E9471698C2FCF911F9153
:10D700000F910895CF93DF93EC018991882319F04D
:10D710000E942A6AFACFDF91CF9108950E942A6A67
:10D7200090E080E00895109263031092140608952B
:10D73000CF9380916303C1E0811104C0C0E08C2FBE
:10D74000CF9108950E94936BFACF8EEF9FE00F94D4
:10D75000DC9F8E3F39F091E020912F03281390E059
:10D76000892F089580E0089510922F036EEF8EEFB9
:10D770009FE00D9400A0853728E6920709F459C070
:10D78000F8F48E3625E6920709F459C050F4833731
:10D7900023E69207B1F185369446B1F182E993E62A
:10D7A0000895823726E6920791F1823728E692079C
:10D7B00009F442C08337954689F789EE93E60895C8
:10D7C0008C3620E7920731F170F48C362EE6920702
:10D7D00021F18F362EE6920731F184379946F1F622
:10D7E00087ED93E608958B3623E79207F9F08637A5
:10D7F00023E79207A9F08F36924781F685E993E6F1
:10D80000089589EF93E6089581EF93E6089580EEF9
:10D8100093E6089580ED93E6089585EC93E60895E8
:10D820008DEB93E6089587EB93E608958CEA93E6F3
:10D83000089585EA93E608958CE993E6089581E0DA
:10D8400094E60895E3E5F4E785919591A591B49167
:10D850008F3F9F4FAF4FBF4FB1F020E031E081E0ED
:10D86000F9014591559165917491453A5A45644B3A
:10D870007B4409F00895F901349645915491240FA1
:10D88000351F8F5FEDCF81E008950F931F938111B6
:10D8900013C010922E0310922D0310922F0390911B
:10D8A0002F0398135CC0682F8EEF9FE00F9400A0A9
:10D8B00081E01F910F910895813089F7E0E0F1E058
:10D8C0004591559165917491453A5A45644B7B4415
:10D8D00031F7E4E0F1E0A591B491E8E0F1E0659181
:10D8E000749150E040E030E020E0A417B50729F53E
:10D8F000261B370B3227232732276217730709F0BD
:10D90000CECFECE0F1E00591159125913491E3E55E
:10D91000F4E7459155916591749104171507260711
:10D92000370709F0BCCF20E031E030932E0320937D
:10D930002D0391E090932F03B2CFFA01E050FF4FF7
:10D94000E491F0E098E040FD90E002C0EE0FFF1F90
:10D950009A95E2F72E0F3F1F4F5F5F4FC6CF80E0D3
:10D96000A8CF20912F03211104C0FC013296CF01D2
:10D97000089540912D0350912E0341155105A9F3AF
:10D98000FC01259134912F3F320779F3F901389644
:10D99000EE0FFF1FE40FF51F25913491FA01E20FFE
:10D9A000F31F2491222309F3E2CFCF93DF93EC01FD
:10D9B00020E030E04CE852E46091011270910212D4
:10D9C00080910312909104120F9404A160930112AC
:10D9D00070930212809303129093041260E070E03F
:10D9E00080EA91E40F9470840E94755E0E94AE6993
:10D9F00082E09AE50E94B16CAC0160E080E00E9498
:10DA00008F698881882339F061E080E00E947B691A
:10DA1000CE010E94826B85E699E30E94B16CAC0155
:10DA200062E080E00E948F6983E49BE20F940B0C1C
:10DA3000DF91CF910D9442220F9492418F3F11F1CB
:10DA400080E00E94C0690E94AE698EE596E50E9462
:10DA5000B16CAC0161E080E00E948F6980E20E94BD
:10DA60002A6A0F949241682F70E06F5F7F4F072EF4
:10DA7000000C880B990B0E94346B0F94936A81E021
:10DA80000C94C06908951F920F920FB60F92112443
:10DA90000BB60F922F938F939F93EF93FF93E09189
:10DAA0002803E830E8F4F0E08827E65AF2498F4F7F
:10DAB0000D94ECA0626D7C6D876D956DAB6DB46D52
:10DAC000D76DE96D8091920681110AC080915B0645
:10DAD000880F80932703882319F081E0809328031F
:10DAE000FF91EF919F918F912F910F900BBE0F900F
:10DAF0000FBE0F901F901895809126038F5F809323
:10DB0000260390912703981758F382E0E7CF83E02C
:10DB1000809328038FE0809325038FEF86BD81E0FB
:10DB200085BD84B58F7E84BDDBCF80912503829532
:10DB3000807F819588BD80912503882321F08150C5
:10DB400080932503CDCF84E0809328038FEF88BD99
:10DB50008EEF86BDC5CF85E0809328038FEF88BD0B
:10DB600086BD82E085BDBCCF2FEF28BD8091920697
:10DB70008111B6CF809126038F5F80932603909109
:10DB80002703891708F4ACCF80915B0690E08F37AC
:10DB900091050CF0A5CF86E0809328038FE0809359
:10DBA000250326BD81E085BD84B58061BCCF809111
:10DBB00025038295807F819588BD80912503811101
:10DBC000BECF87E08093280380E886BD8FEF88BDB5
:10DBD00087CF1092280380E886BD8FEF88BDC1CF24
:10DBE000CF93DF93EC0187E69FE00F94DC9F91E0F9
:10DBF000811101C090E081E02881211101C080E005
:10DC00008913988387E09FE00F94DC9F91E0811156
:10DC100001C090E0998385ED9EE00F94DC9F91E038
:10DC2000811101C090E09A8387E49DE00F94DC9F0E
:10DC30008F3F21F08887DF91CF9108951886FBCF21
:10DC4000CF93C82F682F87E69FE00F9400A0CC23C6
:10DC500019F0CF910D943E53519859981092841613
:10DC6000CF910895109284030F94740F60938D16D2
:10DC700070938E1680938F169093901608958093CC
:10DC8000240380FD1CC010924003209140038FEFBD
:10DC9000820F8E3FE8F08091A000877F8093A000E4
:10DCA0001092AD001092AC009FB7222361F0F8945F
:10DCB000809102018062809302019FBF08958FEFDF
:10DCC00080934003E2CFF894809102018F7DF3CFDF
:10DCD000EFB7F8948091A00088608093A00030E0B6
:10DCE000809172004FEF50E081FF04C04091A80086
:10DCF0005091A900249FC001259F900D349F900D45
:10DD000011246FEF70E00F94A5A07093AD006093A5
:10DD1000AC00EFBF08951F93CF93DF93D0912403FE
:10DD2000D1FD1DC010919A03C1E020E030E048E42D
:10DD300052E46091C40D7091C50D8091C60D909113
:10DD4000C70D0F948DA318160CF0C0E0DE7FCD2B0D
:10DD500081E0111101C080E0C82BC09324038091A1
:10DD60002403DF91CF911F910C943F6EEF92FF92AD
:10DD70000F931F93CF93DF93EC018B017A010E94E5
:10DD8000105581110BC0A801BE01C701DF91CF91D1
:10DD90001F910F91FF90EF900D94F09FDF91CF9125
:10DDA0001F910F91FF90EF9008950F931F93CF93C2
:10DDB000DF938C01D62FC72F0F94EA9F8F3F9807D0
:10DDC00039F46D2F7C2FC8010F943AA08D2F9C2F12
:10DDD000DF91CF911F910F9108950F931F93CF93D0
:10DDE0008C01C62F0F94DC9F8F3F29F46C2FC80144
:10DDF0000F9424A08C2FCF911F910F910895CF9352
:10DE0000DF93EC010F94EA9FBC016F5F7F4FCE015F
:10DE1000DF91CF910D943AA0CF93DF93EC010F9453
:10DE2000DC9F61E0680FCE01DF91CF910D9424A0BB
:10DE30002BE0829FC0011124805B924F0F94EA9FD8
:10DE400021E0019609F420E0822F0895CF93DF931B
:10DE5000C82FD8E0CF5FC8300CF0C0E08C2F0E94F4
:10DE6000186F811103C0D150A9F7CFEF8C2FDF912C
:10DE7000CF91089581EA9DE00F94DC9F0E94266F68
:10DE800087FD05C0682F81EA9DE00D9400A00895EC
:10DE90000F931F93CF93C82F8B0166E074E78230F6
:10DEA00070F06FEF73E7843050F067EF73E7843002
:10DEB00031F06FEE73E7853011F068EE73E7C8015B
:10DEC0000F94939D8CEF8C0F823028F0C170CF5C43
:10DED000F801C6831782CF911F910F91089561E0D9
:10DEE00080EC9FE00F9400A060E08FEB9FE00F9428
:10DEF00000A060E08EEB9FE00F9400A060E08DEB4F
:10DF00009FE00F9400A060E08CEB9FE00D9400A0D8
:10DF1000CF93C82F82958F700E94C65C8C2F8F7014
:10DF2000CF910C94C65C4091CF115091D01190E0EC
:10DF300080E041155105B1F12091CB113091CC1108
:10DF400090E080E0F901E252F04FA081A23021F48C
:10DF500061817281860F971F4150510919F1F901B2
:10DF6000EF51F04FA1919F012E5D3F40A111FACFDB
:10DF7000F901E252F04F2D3EA1E03A0730F4A191B1
:10DF8000A111E0CF2F5F3F4FF6CF2D3EE1E03E07DE
:10DF9000C9F6EEEDFFE09F012E5D3F40A191AA235F
:10DFA000D1F3D0CF08958091CF119091D011181650
:10DFB00019060CF043C001979093D0118093CF11B4
:10DFC000892BA1F48091DA0F9091DB0F892B21F43A
:10DFD0001092DD0F1092DC0F8091DC0F9091DD0F1D
:10DFE0009093CC118093CB1181E008958091CB1157
:10DFF0009091CC110396FC01E252F04F20810196E2
:10E000002111F9CFFC01E252F04F8D3E21E0920741
:10E0100040F441919C012F5F3F4F4111E1CFC90175
:10E02000F4CFEEEDFFE08D3E21E09207C9F6CF017F
:10E030008E5D9F4021912223D1F3D2CF80E00895BD
:10E04000FC0120E03EE2DB014D91BD01403249F090
:10E05000283011F430833196DB0111974C914083C5
:10E0600031962F5F2B3079F71082089540E050E011
:10E07000BA010D943F39FC01238121110D94926E58
:10E08000089590910405911107C09091C00095FFEB
:10E09000FCCF8093C6000895913031F49091C80070
:10E0A00095FFFCCF8093CE0008950E94417090E0D0
:10E0B00080E00895CF93DF93EC01FE0184918823E3
:10E0C00021F00E9441702196F8CFDF91CF91089501
:10E0D000CF92DF92EF92FF92C090C40DD090C50D09
:10E0E000E090C60DF090C70D89E598E70E945A7040
:10E0F00042E0C701B6010F94499781E598E70E9475
:10E100005A7060918A0370918B0380918C03909177
:10E110008D0341E00F944997FF90EF90DF90CF90EF
:10E120000D94FC974F925F926F927F928F929F9285
:10E13000AF92BF92CF92DF92EF92FF920F931F9315
:10E14000CF93DF93CC24CA94DC2C76010EEA1FE037
:10E1500093E2892E912CA12CB12C412C512C32010F
:10E16000D0E0C0E08FEFC81609F45DC0C8010F947D
:10E17000EA9FEC01BC01990F880B990B0F946A9AE6
:10E1800020913E0430913F0440914004509141045D
:10E190000F9403A22B013C01C701B6010F94A29674
:10E1A0008DEA97E70E945A70C501B4010F94A296B8
:10E1B0008DEA97E70E945A70BE010D2E000C880B65
:10E1C000990B0F94A2968DEA97E70E945A7020E06F
:10E1D00030E04AE754E4C301B2010F94A99A0F94C6
:10E1E0008D4185E0880E911CA11CB11C0E5F1F4F54
:10E1F0008FEFC81AD80AE80AF80A0A3B8FE0180716
:10E2000009F0B0CFDF91CF911F910F91FF90EF9068
:10E21000DF90CF90BF90AF909F908F907F906F9046
:10E220005F904F9008958CE89DE30E945A70B8CF9C
:10E23000882371F181EA97E70E945A706091231256
:10E2400070E090E080E00F94A296809123128430D9
:10E25000D8F0109223128CE997E70E945A708091AF
:10E26000231290E00F94AA41809123122091EF1184
:10E270003091F0113093F2112093F1110E94F9F6D0
:10E280000E94755E0D9442228F5F80932312E3CF2C
:10E2900084E29EE30E94B16C70E060E00E94EABC00
:10E2A000E5CFCF93DF9389E997E70E945A70C5EFD6
:10E2B000D1E1688179818A819B8142E00F944997FD
:10E2C00085E997E70E945A706C817D818E819F81DC
:10E2D00042E00F94499781E997E70E945A70688558
:10E2E00079858A859B8542E00F9449978DE897E769
:10E2F0000E945A706C857D858E859F8542E00F94C3
:10E30000499789E094E60E945A7080E00F94202299
:10E310000F946A9AC2E3D4E02C813D814E815F81E3
:10E320000F9403A242E00F94499789E897E70E946F
:10E330005A7081E00F9420220F946A9A28853985BB
:10E340004A855B850F9403A242E00F94499785E8C4
:10E3500097E70E945A7082E00F9420220F946A9AE5
:10E360002C853D854E855F850F9403A242E00F9476
:10E37000499781E897E70E945A7083E00F94202222
:10E380000F946A9A288939894A895B890F9403A274
:10E39000DF91CF910D948D4180E996E70E945A70EC
:10E3A0006091C40D7091C50D8091C60D9091C70DFF
:10E3B00041E00F9449978DE896E70E945A7060916A
:10E3C000F1117091F211072E000C880B990B0F942C
:10E3D0006A9A41E00F94499789E896E70E945A703B
:10E3E00060918A0370918B0380918C0390918D03CF
:10E3F00041E00F94499786E896E70E945A70609131
:10E40000ED117091EE11072E000C880B990B0F94F3
:10E410006A9A41E00F94499781E896E70E945A7002
:10E420006091C40D7091C50D8091C60D9091C70D7E
:10E4300041E00F9449978EE796E70E945A706091E9
:10E44000F1117091F211072E000C880B990B0F94AB
:10E450006A9A41E00F9449978AE796E70E945A70BA
:10E460006091620670E090E080E00F94A29685E7EC
:10E4700096E70E945A7060915B0670E090E080E041
:10E480000F94A29681E796E70E945A7060918E06DB
:10E4900070918F06809190069091910641E00F94C3
:10E4A00049970D94FC970E945A700D94FC978F9297
:10E4B0009F92AF92BF92CF92DF92EF92FF920F9412
:10E4C000740F6B017C0120913202222309F14091EB
:10E4D00078024130E9F08091140290911502A091E8
:10E4E0001602B091170246015701881A990AAA0A22
:10E4F000BB0A30E0A8EEB3E00F947CA08616970626
:10E50000A806B9066CF0443031F19CF44230D4F4E2
:10E51000C0921402D0921502E0921602F0921702F5
:10E52000FF90EF90DF90CF90BF90AF909F908F9033
:10E530000895453069F781E69DE90E945A708CE59F
:10E5400098E706C081E69DE90E945A7089E898E73D
:10E550000E945372DDCF81E69DE90E945A7083E7E5
:10E5600098E7F6CFCF9381EA9DE00F94DC9FCBE054
:10E570008C9FC0011124805B924F0F94EA9F8156BB
:10E58000904F803A9F40C8F088E298E70E9453720B
:10E5900081EA9DE00F94DC9F8C9FC001112470E004
:10E5A00060E0805B924F0F943AA08BEE97E70F9458
:10E5B000470B81E0CF910C94C069CF910895EC0195
:10E5C000F8940F945F12179A1092A306169A10925D
:10E5D000A406149A84E49DE90E945A708CEC97E793
:10E5E0000E945372209779F0CE010E945372BE01AF
:10E5F00085E99CE00F943AA062E484E99CE00F94E2
:10E6000024A00E94A760C4ECD7E7F1CF8AE493E08E
:10E610000F94A1118091CF119091D011892B79F095
:10E62000E091CB11F091CC11E252F04F808181301A
:10E6300011F0863021F481E399E60C945372089529
:10E640008091CF119091D011892B29F00E940673EF
:10E650000E94D36FF5CF1092CC111092CB11109273
:10E66000DD0F1092DC0F81E08093E6110895EF92A8
:10E67000FF920F931F93CF93DF9380919C12882377
:10E6800089F186E597E70E94537280E497E70E943C
:10E6900053728FE297E70E945372C7E0DCE1C150EA
:10E6A00058F1CD9F7001112401E010E08CE297E752
:10E6B0000E945A70F801EE0FFF1FEE0FFF1FEE0DC4
:10E6C000FF1DE756FD4E608171818281938145E097
:10E6D0000F9449970F5F1F4F0830110539F70F94BA
:10E6E000FC97DDCF83E697E7DF91CF911F910F91E4
:10E6F000FF90EF900C945372DF91CF911F910F9187
:10E70000FF90EF900895CF92DF92EF92FF926B010E
:10E710007C01C0922903D0922A03E0922B03F0924D
:10E720002C03809145038230B1F420E030E040E9D1
:10E7300050E4C7010F94F9A187FF14C080916204CF
:10E7400090916304A0916404B0916504803D97406A
:10E75000A105B10520F5C701B601FF90EF90DF904C
:10E76000CF9008952AE939E949E95EE3C701B60186
:10E770000F94F9A187FF0AC020E030E048E351E49C
:10E78000C701B6010F94A99A6B017C018AE394E753
:10E790000E945A70C701B6010F948D41DCCF2AE95F
:10E7A00039E949E95EE3C701B6010F94F9A187FD94
:10E7B000E3CF20E030E040E85EE3C701B6010F940C
:10E7C000A99A20E030E048E550E40F9404A1DCCFA2
:10E7D000CF92DF92EF92FF92CF93909145039817DB
:10E7E000B9F1C82FC0902903D0902A03E0902B03E1
:10E7F000F0902C0320E030E0A901C701B6010F948E
:10E80000F9A1882341F0C0928604D0928704E09257
:10E810008804F09289048DE194E70E945A70C13017
:10E8200011F1E0F0C23011F1C0934503609186040C
:10E830007091870480918804909189040E94837369
:10E84000609386047093870480938804909389046E
:10E85000CF91FF90EF90DF90CF90089585E194E7FE
:10E860000E945372E1CF81E194E7FACF8DE094E703
:10E87000F7CF0F944222179AE3EAF6E01082169A35
:10E880001182149A80E00E94E8738FEF9FEF9093BB
:10E890007502809374022FEF2093710290933E02D1
:10E8A00080933D0220933F02909373028093720203
:10E8B00090933C0280933B020895182FF894CDB7B3
:10E8C000DEB700D0CF90DF90EF9088E199E20FB6ED
:10E8D000F894A895809360000FBE909360009FB756
:10E8E000F894E2E0F1E08081886080839FBF0F941C
:10E8F0005F128CEC93E70E94537284EC93E70E94C2
:10E900005A70612F70E090E080E04AE00F942C96FE
:10E9100080EC93E70E945A708E2DB60190E040E1A2
:10E920000F942C968CEB93E70E945A70BE0190E0F6
:10E9300080E040E10F942C960F94FC9740E060E05B
:10E9400072E290E080E00F94E55281E399E60E9444
:10E9500053720E94A760C82F729A682F83E09DE0CF
:10E960000F9400A080917C06882319F08C2F0E94C0
:10E970005D740E94A7601F920F920FB60F92112430
:10E9800083E00E94AB741F920F920FB60F92112476
:10E9900082E00E94AB7441ED50E06BEE72E782E3DF
:10E9A00094E00F94769D0F9495740F9496180E949E
:10E9B000D25E81E69DE90E945A7089EC92E70C9440
:10E9C000537244E050E064E170E082E394E00F941D
:10E9D000CC9F43E050E06BEE72E782E394E00F944B
:10E9E000BB9D892B09F05DC0EFEAF3E74591559196
:10E9F0006591749188ED90E00E94225DE3EBF3E76E
:10EA000045915591659174918CED90E00E94225D45
:10EA1000E7EBF3E7649180EE90E00E94ED6EE8EBA7
:10EA2000F3E76591749181EE90E00E94D56EEAEB78
:10EA3000F3E76591749183EE90E00E94D56EEBEA66
:10EA4000F3E7459155916591749184ED90E00E94B2
:10EA5000225D47E853E760E170E080EB90E00E94C0
:10EA6000B66E47E953E760E170E080EC90E00E9409
:10EA7000B66E41ED50E064E170E082E394E00F9403
:10EA8000CC9F0E94D25E0F9495740F94961881E6E5
:10EA90009DE90E945A708FEA92E70E94537281E0CA
:10EAA00008950E94CB7464E070E084E190E00E94DD
:10EAB000105591E0892708956BEE72E782E394E0A8
:10EAC0000F94939D41ED50E064E170E082E394E0A7
:10EAD0000F94F09F81E69DE90E945A708FE992E7BA
:10EAE0000C9453722F923F924F925F926F927F924B
:10EAF0008F929F92AF92BF92CF92DF92EF92FF924E
:10EB00000F931F93CF93DF93CDB7DEB7A0970FB6C8
:10EB1000F894DEBF0FBECDBF8FE590E00E94BC55DC
:10EB2000882309F4A1C00E94C0548F37910561F475
:10EB30008091B1059091B2059093B0058093AF0597
:10EB400080E992E70E9453726E014FE1C40ED11C1E
:10EB5000992493940E94C054181619060CF078C09A
:10EB60008091E711882329F00E94BD60882309F471
:10EB70006FC08091610381116BC02091B10530910C
:10EB8000B2058091AF059091B0058217930711F3FC
:10EB9000F901E15DFA4F80812F5F3F4F2F773327D7
:10EBA0003093B2052093B1058F3F09F079C0809171
:10EBB0001B03882309F471C090921A0310921B035F
:10EBC0001F8E18A280901E03882021F280911C03C2
:10EBD0008F8FF1E0F81518F480911D0388A310922F
:10EBE0001E031601822D8C19881508F0B3CFF10190
:10EBF00011911F0181E293E00F94D60F17FDF2CF20
:10EC00008091DA0F9091DB0F1A3009F44BC11D305F
:10EC100009F448C18F3591050CF049C11B3311F43B
:10EC200090922003209120032111DCCF9C012F5FC3
:10EC30003F4F3093DB0F2093DA0F2091DC0F3091A0
:10EC4000DD0F2252304F820F931FFC011383CACF76
:10EC50008091DA0F9091DB0F181619060CF451C24F
:10EC600080916A13811167C2A0960FB6F894DEBF37
:10EC70000FBECDBFDF91CF911F910F91FF90EF900D
:10EC8000DF90CF90BF90AF909F908F907F906F90CC
:10EC90005F904F903F902F90089590921B0390CFDC
:10ECA00090911A03992309F458C0893FE9F170F54E
:10ECB000863F09F44AC0873F09F443C08BE592E7D9
:10ECC0000E945A7086E592E70E945A7010911903CB
:10ECD00082E592E710FD02C08DE492E70E945A702F
:10ECE000012F027088E492E711FD02C083E492E7ED
:10ECF0000E945A7082E492E70E945372002349F105
:10ED000085E480930B0210921A035ACF8A3F41F098
:10ED10008B3FA1F680911903816080931903CECFB8
:10ED2000809119038E7FF9CF10921E0310921A035F
:10ED3000109219031092180310921B0310921703DC
:10ED4000BDCF809119038260E8CF809119038D7F38
:10ED5000E4CF90E290930B02D6CF90911B033091B9
:10ED60001903992331F1E0911E0330FF49C020912E
:10ED70001703222309F440C091E09E0F90931E03D5
:10ED8000AE2FB0E0A45EBC4FFFEFFC9340911803A0
:10ED9000442351F0EE5FE0931E03E92FF0E0E45EC0
:10EDA000FC4F4083109218032150209317031092B8
:10EDB0001B03E0911E0330FF6CC090911703992351
:10EDC00049F121E02E0F20931E03AE2FB0E0A45E88
:10EDD000BC4F8C9380911803882351F0EE5FE09331
:10EDE0001E03E22FF0E0E45EFC4F808310921803D4
:10EDF000915090931703E4CE42E040931703D7CF8E
:10EE000091E09E0F90931E03F0E0E45EFC4F9FEFB5
:10EE10009083CDCFA82FAF7030E021E0AF3029F044
:10EE2000B0E0A050BE4F3C9120E0482F407F403FD3
:10EE300059F4226020FF13C09092170321FF0CC0E9
:10EE4000E2E0E0931703BCCE82958F70A82FB0E06C
:10EE5000A050BE4F9C91EECF90931803B1CE81E0AD
:10EE60008E0F80931E03AE2FB0E0A45EBC4F3C9388
:10EE70003A3009F4A5CE21FF03C090921703A0CE2B
:10EE8000EE5FE0931E03E82FF0E0E45EFC4F90831A
:10EE900097CE91E09E0F90931E03F0E0E45EFC4F4E
:10EEA00080838ECE009719F410922003DDCE00915E
:10EEB000DC0F1091DD0F0F51104F800F911FFC01DF
:10EEC00010821A830983809120038111FDC0F8010B
:10EED00080818E3409F084C04AE050E0BE016F5F4B
:10EEE0007F4FC80101960F94679B2B013C01E9807D
:10EEF000FA80F7018081803231F4FFEFEF1AFF0AC8
:10EF0000FA82E982F4CF8091D1119091D211A0912F
:10EF1000D311B091D4110196A11DB11D8415950591
:10EF2000A605B70549F044E050E06BE872E7C70179
:10EF30000F94BB9D892BA1F46AE270E0C7010F9486
:10EF400033A69093F6168093F516009709F441C006
:10EF5000F801F12C8E179F07F1F02191F226FACFDC
:10EF600084E49DE90E945A7080E293E60E945A7000
:10EF70006091D1117091D2118091D3119091D411DF
:10EF80000F94A2960F94FC970E94E2541092DB0F0C
:10EF90001092DA0F69CE0E944D55F816190639F015
:10EFA00084E49DE90E945A7081E093E6DFCFE0910E
:10EFB000F516F091F6161082E980FA8066E872E79D
:10EFC000C7010F948A9D892B39F587E695E60E9443
:10EFD000DF7284E49DE90E945A7087ED92E6C6CF05
:10EFE00089819A81FC012081203221F401969A8343
:10EFF0008983F6CF6AE270E00F9433A6892B39F04B
:10F0000084E49DE90E945A708DEA92E6AFCF4424D1
:10F010004A94542C3201D0CF44E050E061E872E7CA
:10F02000C7010F94BB9D5C01F7018081873481F497
:10F030008091CB0D853061F085ED91E10F94D60F75
:10F04000F6E0F093CB0D60E085EA9FE00F9400A01E
:10F05000AB2821F08091CE11811198CF26E077FC6A
:10F0600021E08091DC0F9091DD0FFC01E252F04F26
:10F07000208349815A81F801DA0140175107A1F52F
:10F0800001900020E9F79F01201B310B0396280F08
:10F09000391F2D3EF1E03F0779F13093DD0F2093CA
:10F0A000DC0F8091CF119091D01101969093D011E7
:10F0B0008093CF1177FC08C04092D1115092D211A9
:10F0C0006092D3117092D4111092DB0F1092DA0F6C
:10F0D0000E94C054892B09F4C7CD8FE590E00E94AF
:10F0E000BC5581117FCDC0CD6D9161939D01241BD5
:10F0F000350B6111F9CFCACF1092DD0F1092DC0FE2
:10F10000D0CF8091CA0D60E273E0811102C060ED42
:10F1100077E081E293E00F94A70F882309F4A0CD54
:10F12000109220031092DB0F1092DA0F86E792E71D
:10F130000E94537299CD8091FD15882309F494CDD6
:10F140008091DA0F9091DB0F892B09F08DCD8091A2
:10F15000CF119091D011892B11F410921F0312E05E
:10F1600001E040917E1650917F166091801670915B
:10F1700081168091771690917816A0917916B091AA
:10F180007A16481759076A077B0708F0C1C08091B3
:10F190001F038111BDC00F94CE48409102165091BB
:10F1A0000316609104167091051640937E165093D5
:10F1B0007F1660938016709381162091DA0F30913C
:10F1C000DB0F8A3061F08D3051F0833209F487C053
:10F1D0002F35310524F48F3F980709F087C021159A
:10F1E000310509F441CD8091FD15811103C040E046
:10F1F00050E0BA018091DC119091DD11481B590B50
:10F20000A091DC0FB091DD0FFD01E252F04F1083B1
:10F210004183528313962252304FF901EA0FFB1FAC
:10F220001082A252B04FFD0101900020E9F7319702
:10F23000EA1BFB0BF8948091CF119091D0110196AD
:10F240009093D0118093CF11EC5F8091DC0F90915F
:10F25000DD0FE80FF92FF11DF093DD0FE093DC0FC8
:10F260008091FD15882309F43DC080917E16909110
:10F270007F16A0918016B09181168093DC11909337
:10F28000DD11A093DE11B093DF11ED3EF14021F4CA
:10F290001092DD0F1092DC0F7894109220031092E0
:10F2A000DB0F1092DA0F40917E1650917F1660911D
:10F2B0008016709181168091771690917816A091A2
:10F2C0007916B0917A16481759076A077B0700F537
:10F2D0008FE590E00E94BC55811143CFC5CC0093CF
:10F2E0001F037DCF80E090E0DC01C7CFA9014F5F15
:10F2F0005F4F5093DB0F4093DA0F4091DC0F50913A
:10F30000DD0F4252504F240F351FF901838329CF5F
:10F3100040917E1650917F166091801670918116F3
:10F320008091771690917816A0917916B0917A16FF
:10F33000481759076A077B0708F496CC0E94936F19
:10F34000892B09F091CC0F94E4418AE992E60E945E
:10F3500053720F94661C6B017C010E94385F8CE332
:10F36000882E912CA12CB12CC701B601A5019401C6
:10F370000F944FA0CA01B901A50194010F944FA0A9
:10F380007F936F93C701B60120E13EE040E050E07B
:10F390000F944FA03F932F9382E692E79F938F9312
:10F3A0008E010F5F1F4F1F930F930F94F39E81E603
:10F3B0009DE90E945A70C8010F94FD98C8010E94EF
:10F3C00081EF0F943E4D109256020FB6F894DEBFB7
:10F3D0000FBECDBF80916B13882359F00F94114459
:10F3E0008091CA0D882309F43FCC86E00F94FF97E3
:10F3F0003BCC81E00F947D4D80916B138111EECF5A
:10F40000EFCF0F931F93CF93DF93D82F8091841664
:10F41000813009F449C0823009F44DC00E9419615D
:10F420008111ECC08091F1119091F211009739F4A3
:10F430002091ED113091EE11232B09F4DFC04091A2
:10F4400033025091340260913502709136024115B9
:10F4500051056105710509F4D1C0892B31F4809102
:10F46000ED119091EE11892B29F080911A068823D5
:10F4700009F42CC18091CA0D882321F040EE52E39B
:10F4800069E270E08AE196E00F94E20F882309F4C4
:10F49000B7C00F945F1280E696E30E94B16C0F94A0
:10F4A000470B0E9417FEACC082E0809384160E9436
:10F4B000FCC3809387161092881680918416823040
:10F4C00009F0ACCF8091891681113DC00E94FCC328
:10F4D000C82F80918716C81709F4A0CFC09387164C
:10F4E00089E896E10F94D60FCC23B1F1809185166F
:10F4F000882311F18091620381111EC080919412C2
:10F500008130D1F08091A80D9091A90D891B8F7049
:10F5100099F40E94C86081110FC08091C80D843099
:10F5200059F08FE59FE00F94DC9F811105C061E0E9
:10F5300083E098E30F94299481E08093881681E01A
:10F5400080935B026BCF64E670E089E896E10F94EC
:10F55000A70F8111BBCF62CF80918616882379F3E4
:10F56000809162038111EBCF8091A80D9091A90D3C
:10F57000891B8F7021F40E94C860882301F3809159
:10F58000E7118111DCCF809194128130C1F280911A
:10F59000C80D8430A1F28FE59FE00F94DC9F8111AC
:10F5A000CECF88E694E69F938F938EE494E69F9364
:10F5B0008F930F949E9E10928616109285160F9030
:10F5C0000F900F900F908091E711811105C060E0BE
:10F5D00070E0CB010F94F14160E070E0CB010E943C
:10F5E000406185E69FE00E940C6F81E09FE00E94F1
:10F5F000FF6E8BE79BE60F945743A1CF10921A063C
:10F600008091CF119091D011039714F40E947275DC
:10F610009091A80D8091A90D981781F08091CB0D44
:10F62000863061F468E873E185ED91E10F94A70FEE
:10F63000882321F085ED91E10F94D60F4091460388
:10F64000509147036091480370914903411551055A
:10F650006105710509F03FC04091370250913802B1
:10F660006091390270913A024115510561057105A9
:10F67000A9F08AE493E00F94E20F882379F0909147
:10F68000A80D8091A90D981309C0D11107C0179A30
:10F690001092A306169A1092A406149AC091E9112A
:10F6A0009091A90D8091A80D981701F18091A90D55
:10F6B0009EE6899FF0011124E25FF84FC08190918E
:10F6C000A80D981799F08F5F8F70F9CF8AE196E0B7
:10F6D0000F94A11195CF8AE493E00F94E20F882351
:10F6E00009F4BACF80EB97E70E94DF72CC2309F4CC
:10F6F000BEC08091410390914203A0914303B09119
:10F700004403892B8A2B8B2B81F40F94740F605E3A
:10F710007C4F8F4F9F4F60934103709342038093C0
:10F72000430390934403CFEF0FC00F94740F0091E5
:10F730004103109142032091430330914403601729
:10F7400071078207930778F380918403882309F473
:10F7500097C0C093670280912D04811107C081E09A
:10F7600080932D040F94526410922D0480911306FF
:10F770008823C9F1109213064FB7F89480911106AF
:10F78000282F082E000C330B37FF03C0319521952D
:10F790003109243031050CF476C0982F87FF02C060
:10F7A00093E0980F95959595209106053091070562
:10F7B000290F311D97FD3A953093070520930605D3
:10F7C000837887FF03C081508C6F8F5F8093110611
:10F7D0004FBF86E00F949F2C80915B02811103C084
:10F7E00081E080935B0280911406882361F00E947F
:10F7F000936BE091D403F091D503309721F0809181
:10F800005C02811119952091621330E0A8EEB3E0FB
:10F810000F947CA0AB01BC0183E693E10F94E20F4F
:10F82000882399F08091611380FD0E94CC718091B2
:10F83000611382FD0E9451718091611381FD0E94CC
:10F840009D5F83E693E10F94A1118091CA0D811110
:10F8500002C00E94577240E355E760E070E08AE51D
:10F8600093E0DF91CF911F910F910D94E20F1092D1
:10F87000410310924203109243031092440364CF59
:10F88000C093050568CF109211064FBF80E0A2CF4C
:10F89000CF93DF93EC010F945B3281E00E94017AF9
:10F8A00080E00E944269209799F0C233D10540F070
:10F8B00062E370E080E090E00F947B0DE297EBCF85
:10F8C000BE0190E080E00F947B0DD0E0C0E0E3CF7C
:10F8D000DF91CF910895CF93DF93C82FDFEF0F947F
:10F8E0005B3281E00E94017A809192128F3FD9F4BD
:10F8F00080912712843021F480912A128111EFCF58
:10F900008091651290916612019749F780918C124F
:10F9100090918D128932904811F360E089E290E86D
:10F920000F94AA4FDCCFD0939212853039F4CF3F99
:10F93000F9F261E08C2F0F94EE6AD1CF8430C1F6DA
:10F94000DF91CF910895CF93DF93EC0189918823C4
:10F9500019F00E944170FACFDF91CF910895FF9284
:10F960000F931F93CF93DF93EC01F62E662309F4D8
:10F970004BC00F949A9D8C01C8010E94BC558823EE
:10F9800009F453C08091DC0F9091DD0FFC01E2522D
:10F99000F04F23E020838F51904FBE01FF20E9F10B
:10F9A0000F94939D81E69DE90E945A708FE892E63C
:10F9B0000E945A708091DC0F9091DD0F8F51904F13
:10F9C0000E94A37C80E492E70E9453728091DC0F36
:10F9D0009091DD0F0496080F191F0D3E81E0180766
:10F9E000F9F01093DD0F0093DC0F8091CF1190910F
:10F9F000D01101969093D0118093CF11DF91CF91C8
:10FA00001F910F91FF900895FC0101900020E9F7EC
:10FA100031978F01081B190BAFCF0F9447A6C2CFA8
:10FA20001092DD0F1092DC0FE0CF84E49DE90E947C
:10FA30005A708FE892E60E945A70CE01FF2059F06A
:10FA40000E945A7082E19DE9DF91CF911F910F9141
:10FA5000FF900C9453720E94A37CF4CF0F931F93DA
:10FA6000CF93DF93D62F8C01C0E0F801859194915C
:10FA700028E68D30920721F420919412213019F458
:10FA800061E00E94AF7CCF5F0E5F1F4FDC13EDCFB4
:10FA9000DF91CF911F910F910895CF93DF93CDB751
:10FAA000DEB76E970FB6F894DEBF0FBECDBF9E01D6
:10FAB0002C5D3F4FF901419151919F016EE170E042
:10FAC000CE0101960F94329F60E0CE0101960E9414
:10FAD000AF7C6E960FB6F894DEBF0FBECDBFDF9140
:10FAE000CF9108951F920F920FB60F9211240BB66B
:10FAF0000F922F933F934F935F936F937F938F93C7
:10FB00009F93AF93BF93EF93FF9320917800309131
:10FB10007900E0911603F0E0EE0FFF1FEA5FFC4F63
:10FB200080819181820F931F91838083809105034F
:10FB30008F5F809305038031E9F5809116038F5F15
:10FB400080931603883071F5809106039091070326
:10FB500090934A068093490680910A0390910B0383
:10FB600090934C0680934B06809108039091090373
:10FB7000909348068093470681E080936306FF9147
:10FB8000EF91BF91AF919F918F917F916F915F9115
:10FB90004F913F912F910F900BBE0F900FBE0F9082
:10FBA0001F901895809104034FE553E08F5F41F457
:10FBB0001092040380917A00806480937A00DFCFF2
:10FBC0009A01082E02C0359527950A94E2F720FF86
:10FBD000EDCF809304030E94CD5410920503EACF29
:10FBE000CF93DF93CAE7D0E088818F7B8883109220
:10FBF0000503109216031092040380E00E94CD5476
:10FC0000E6E0F3E080E1DF011D928A95E9F7888163
:10FC100080648883DF91CF9108952F923F924F9215
:10FC20005F926F927F928F929F92AF92BF92CF928C
:10FC3000DF92EF92FF920F931F93CF93DF93CDB795
:10FC4000DEB7A4970FB6F894DEBF0FBECDBF0F94FA
:10FC500042228091AC0D811117C081E08093061281
:10FC60008091A306882349F08091A406882329F077
:10FC70002091A5062F83211120C081E08093E611F9
:10FC800082E198E60F945743A4960FB6F894DEBF2E
:10FC90000FBECDBFDF91CF911F910F91FF90EF90DD
:10FCA000DF90CF90BF90AF909F908F907F906F909C
:10FCB0005F904F903F902F9008958BEA9DE00F94B6
:10FCC000DC9F182F8EE40E942B55082F0E94405570
:10FCD0008E83002329F0873009F4C9C0833029F0CE
:10FCE000133009F0C3C063E06E8380E090E0A0E8C9
:10FCF000BFE38A839B83AC83BD838AEA9DE00F9434
:10FD0000DC9F888F83E40E942B55182F0E9440555A
:10FD1000112329F0882319F08B3008F4888F88E5A7
:10FD20000E942B55882309F4ABC00E94035A20E09F
:10FD300030E048E052E40F9403A120E030E048EBCB
:10FD400051E40F9403A16A877B878C879D8789E59F
:10FD50000E942B55882309F49CC00E94035A20E07E
:10FD600030E048E052E40F9403A120E030E040EAA4
:10FD700050E40F9403A16C8B7D8B8E8B9F8B87E55A
:10FD80000E942B55882309F489C00E94035A2A85B2
:10FD90003B854C855D850F9404A120E030E048E868
:10FDA00052E40F9404A1698F7A8F8B8F9C8F88E423
:10FDB0000E942B55882309F47AC00E94035A2C898B
:10FDC0003D894E895F890F9404A120E030E048E826
:10FDD00052E40F9404A16D8F7E8F8F8F98A30F94A0
:10FDE000F15580912C0290912D02A0912E02B0919C
:10FDF0002F0280939D1290939E12A0939F12B09316
:10FE0000A0120F940B8B05EC1FE0C8010F94EA9F22
:10FE1000019609F051C00E5F1F4F053D8FE0180796
:10FE2000A1F7212CACE9B2E1BAA3A9A3B987A887AD
:10FE3000512C412C312C042D842D63E00F948BA088
:10FE4000988B6884798410E0F889F11137C0812F8C
:10FE500063E00F948BA0911131C021103FC17E81CE
:10FE6000733009F470C08F818E8737C01E836AE9B2
:10FE700079E989E19FE36A837B838C839D833DCF0E
:10FE800080E090E0A0E8BFEF8A879B87AC87BD87C2
:10FE90005ECF60E070E080E89FEF6DCF80E090E0A3
:10FEA000A0E8BFE7898F9A8FAB8FBC8F80CF60E0CF
:10FEB00070E080E89FE78FCF2F80B4CF60E070E0E4
:10FEC00080EC9FE7D30111966D937D938D939C9366
:10FED0001497BE81B330C1F11E86812F0F94658BBC
:10FEE0004B015C01802F0F94658B6B017C01A50198
:10FEF00094016A857B858C859D850F948DA318164A
:10FF00000CF41CC1298D3A8D4B8D5C8DC501B4015B
:10FF10000F948DA318160CF411C1A70196016C89DA
:10FF20007D898E899F890F948DA318160CF406C1C4
:10FF30002D8D3E8D4F8D58A1C701B6010F948DA315
:10FF400018160CF4FBC033941F5F24E0620E711C82
:10FF5000173009F079CF6FEF461A560A88859985D0
:10FF60004C969987888797E04916510409F063CF2A
:10FF70000E94FCF0A091C706AF83B091AC03B88794
:10FF800081E08093C7068AE0830D8093AC0381E013
:10FF90000E94426980E090E0A0EAB0E48093FD1105
:10FFA0009093FE11A093FF11B093001265E575E5E3
:10FFB00085E591E40F94708480E00E94EE5F9CA33D
:10FFC0008BA3312C832D67E00F948BA0F82E092F83
:10FFD000682F70E07F876E8780FF03C076E0791B13
:10FFE000072F802F63E00F948BA0911105C08F2DF8
:10FFF0000F948BA011E0911110E0802F0F94658B6E
:020000021000EC
:10000000688B798B8A8B9B8B8F2D0F94658B4B0123
:100010005C018E81833009F099C01111C8C027E0BE
:10002000AE85BF852A9FF0012B9FF00D1124E00FB4
:10003000F11DEE0FFF1FEE0FFF1FE456FD4E60E0B7
:1000400070E080EC9FE761837283838394833394B1
:10005000E1E33E12B7CF80E090E0A0EAB0E4809305
:10006000FD119093FE11A093FF11B093001265E56E
:1000700075E585E591E40F9470840F944222B1E315
:100080003B1609F43CC280913F0391E0980F909396
:100090003F03882309F4D3C160E080E00E9492EF1F
:1000A00084E396E30E94B16C0F94470B80E00F94B9
:1000B000C12F81E08093780287E69BE60E9465E687
:1000C0002F812093C70668856093AC0382E00E946D
:1000D00042690F94422210920612D6CD011103C03C
:1000E000112309F4BCCE812F63E00F9497A0840DF7
:1000F000952D911D880F991F8D53904F0F94EA9F56
:10010000BC01990F880B990B0F946A9A2AE037ED7E
:1001100043E25CE30F94A99A9B01AC0160919D12AC
:1001200070919E1280919F129091A0120F9404A141
:10013000F301618372838383948391CEFE85FF23D1
:1001400009F402CF222009F4FECEFECE2889398997
:100150004A895B896A857B858C859D850F948DA3F3
:10016000181604F1288939894A895B89698D7A8D45
:100170008B8D9C8D0F94F9A187FD14C0A50194016E
:100180006C897D898E899F890F948DA3181654F0F0
:10019000A50194016D8D7E8D8F8D98A10F94F9A18D
:1001A00087FF05C0112309F452CF211050CF10E072
:1001B000A7E08E859F85A89FF001A99FF00D1124CF
:1001C000E00FF11FEE0FFF1FEE0FFF1FE456FD4E75
:1001D0004180528063807480C12CD12CE0EAEE2EE5
:1001E000E0E4FE2E222051F023E333E343EB5EE311
:1001F000C301B2010F9404A16B017C01A701960118
:100200006091FD117091FE118091FF11909100128B
:100210000F94F9A187FF10C0C092FD11D092FE117A
:10022000E092FF11F092001265E575E585E591E435
:100230000F9470840F944222688979898A899B89F6
:100240006093F5117093F6118093F7119093F81164
:100250008092F9119092FA11A092FB11B092FC11C8
:1002600069EF71E185EF91E10E94A66360E070E0C3
:1002700086E193E40F9470840F9442228091AC0D38
:10028000882339F07F817093C70688858093AC03FB
:10029000FBCC812C912C70E2A72E71ECB72E222082
:1002A00051F02A813B814C815D81C301B2010F94E1
:1002B00003A14B015C01488DC501B4010F94FB55AE
:1002C00081110BC087E292E60E94B16C9F938F93DD
:1002D0000F949E9E0F900F90BECE2091FD113091F5
:1002E000FE114091FF1150910012C701B6010F9409
:1002F00003A120E030E0A9010F94F9A187FF36C0E7
:1003000060E070E080EA90E46093FD117093FE116C
:100310008093FF119093001265E575E585E591E402
:100320000F9470840F944222488DC501B4010F943C
:10033000FB55882339F22091FD113091FE11409137
:10034000FF115091001260E070E080EA90E40F9499
:1003500003A12DEC3CEC4CEC5DE30F94F9A187FF7D
:1003600005C08DEF96E70F94C59E75CEC090FD1128
:10037000D090FE11E090FF11F09000122220A1F029
:10038000A7019601C301B2010F9403A19B01AC0127
:100390005F776A817B818C819D810F94F9A187FFB2
:1003A00003C084EC96E7DFCF8FEA9FE00F94DC9FD9
:1003B000882309F440C086EA9FE00F94DC9F8823DD
:1003C000D1F160918E0670918F0680919006909188
:1003D00091060E94045620913E0430913F044091C2
:1003E0004004509141040F9403A29B01AC01E7E04B
:1003F000AE85BF85EA9FC001EB9F900D1124080FC9
:10040000191F000F111F000F111F04561D4EC701A9
:10041000B6010F9403A1D80111966D937D938D932E
:100420009C9314978091AC0381508093AC0381E03E
:100430000E9442690CCE20E030E0A901D8CF85E0CF
:100440000F949F2CC12CD12C90EAE92E90E4F92E28
:1004500080E096E30E94B16C0F94C00A90E080E0C7
:100460000F94A13481E00F94FD3480E00F947A2C36
:10047000182F60E070E080E89FEB0E94DD6681E06D
:100480000F947A2CC092FD11D092FE11E092FF11D0
:10049000F092001265E575E585E591E40F947084AE
:1004A0000F944222812F0F947A2C82E00F942E22F7
:1004B00020E030E040EA50E40F948DA3181644F297
:1004C000EF81E093C706F885F093AC0381E00E94CA
:1004D000C069DD24D394DF92812C912C5401CC246B
:1004E000C394E12CF12C870121E040E050E0BA01F7
:1004F00081E00E947367D092E6110F90C5CB1092F5
:100500003F038BA19CA10E94D45F10922A051092F8
:10051000290580E10E9455D8882391F00E94B2728B
:1005200081EA9DE00F94DC9F2BE0829FC0011124A3
:10053000805B924F0F94EA9F90932A058093290540
:100540006091290570912A05072E000C880B990BE4
:100550000F946A9A905820913E0430913F04409144
:100560004004509141040F9403A20F94D18A80EC6F
:100570009FE00F94DC9F91E0813009F090E0998337
:100580004FEB5FE06CE4CE0101960E945A55F82EC5
:100590004EEB5FE062E5CE0101960E945A55082FAE
:1005A0004DEB5FE066E4CE0101960E945A55182F8C
:1005B0004CEB5FE062E4CE0101960E945A55212F78
:1005C000110F330B082E000C990B5C01A21AB30A11
:1005D0008F2DFF0C990B280F391F46E0429F6001B9
:1005E000439FD00C1124F12CE12C002E000C110B98
:1005F000081B190BB70163567D4E3B01460177E09E
:100600007A83D3012D903D904D905D903D01FD0189
:100610003497FB87EA87B401092C000C880B990BEF
:100620000F946A9A2FE333EC4EE259E30F94A99AA0
:10063000A20191010F9404A1AA85BB856D937D93BE
:100640008D939C931397BA81B150BA83800E911EFB
:10065000B111D7CFCA0CDB1CECE1EE0EF11CF4ECAF
:10066000EF16F10439F60E94FCF08DE40E942B5540
:10067000882309F484C00E9440552E81273009F058
:1006800094C0882309F491C0BB24B394AA24AA94EB
:10069000AB0C09A11AA1612C8EEF882E8B0C6A2D50
:1006A000862D0F949C8A99249394960C81116EC088
:1006B0006B2D862D0F949C8AC12CD12C7601712C28
:1006C000882381F020E030E0A901D8015D966D918A
:1006D0007D918D919C9190970F9404A16B017C0169
:1006E00077247394682D862D0F949C8A882369F053
:1006F000F8017B972081318142815381C701B60186
:100700000F9404A16B017C0173946A2D892D0F94C1
:100710009C8A882361F0F8012581368147815085C4
:10072000C701B6010F9404A16B017C0173946A2D7B
:100730008FEF860D0F949C8A882331F1F80133974F
:100740002081318142815381C701B6010F9404A1F8
:100750006B017C017394672D70E090E080E00F9452
:100760006A9A9B01AC01C701B6010F9403A2D8019C
:1007700011966D937D938D939C93149707C08CEA8B
:100780009DE00F94DC9F79CF7110E5CF692C0C5F51
:100790001F4FB7E09B1283CFB394E9A1FAA17C96D7
:1007A000FAA3E9A3F8E0BF1271CF81E080939C1215
:1007B0008FE40E942B55811103C00F94268B79CCB6
:1007C0000E9440558111F9CF0E94C95F72CC2F92CF
:1007D0003F924F925F926F927F928F929F92AF92D1
:1007E000BF92CF92DF92EF92FF920F931F93CF931E
:1007F000DF93CDB7DEB7C356D1090FB6F894DEBF8D
:100800000FBECDBF82E0809378020091CB11109192
:10081000CC110F51104F45E050E060E271E8C80183
:100820000F94BB9D892B09F09BC18091CA0D882331
:1008300009F44DC08EE29EE70F945174882379F03D
:100840008091F7161F928F9382EF94E69F938F9378
:100850000F949E9E0F900F900F900F9008C08AE209
:100860009EE70F945174882341F01092D60381E0E3
:10087000809378020E9406733AC287E29EE70F9443
:100880005174882321F18091F5169091F61661E05C
:1008900003960F94064C0F94CE488C01809102165B
:1008A00090910316A0910416B091051680937E16C0
:1008B00090937F16A0938016B0938116802F0E948C
:1008C00041700A30110539F70F94E441D0CF86E129
:1008D00091E80F9451748111CACF82E191E80F948D
:1008E0005174882321F140918703509188032CE3B0
:1008F000249FC001259F900D11249F938F934091B9
:10090000850350918603249FC001259F900D1124DB
:100910009F938F9386E297E69F938F930F949E9E6B
:100920000F900F900F900F900F900F90A0CF8DE031
:1009300091E80F945174882311F18CE89FE00F9493
:10094000DC9F811110C061E085EE9BE60E94AF7CC8
:1009500060E085EA9FE00F9400A060E08FE79CE0F4
:100960000F9400A084CF813009F081CF0F945620DE
:1009700085ED91E10F94D60F0F94800F78CF86E02C
:1009800091E80F945174882321F080E00F945D6208
:100990006ECF80E091E80F94517481110E94A7609E
:1009A0008DEF90E80F9451748823A9F044E150E052
:1009B00065E17DE0CE0101960F94CC9F8C89882360
:1009C00029F082EF90E80F94C59E51CFCE01019699
:1009D0000F946BA64CCF8EEE90E80F945174882341
:1009E00029F082EE90E80E94537241CF8EED90E89C
:1009F0000F945174882319F08EEB90E8F4CF89EBB3
:100A000090E80F945174882319F00E94B46B2FCF93
:100A100086EB90E80F945174882379F081EA9DE089
:100A20000F94DC9F2BE0829FC001112470E060E0F6
:100A3000805B924F0F941EA01ACF83EB90E80F9427
:100A40005174882351F00E94AE6940E070E060E08C
:100A500084E690E00F94C531D8CF8FEA90E80F94E8
:100A600051748823E1F086E50E942B55882309F410
:100A7000FECE0E944D5511E0892B09F410E00F9431
:100A8000422280919C1290E01817190609F4EFCECB
:100A900010939C128DEF91E10F94FB74E8CE88EADD
:100AA00090E80F945174882309F4E1CE84E40E9405
:100AB0002B558823A1F00E94035A20E030E04AE73A
:100AC00054E40F94A99A20E030E040E05FE30F94F3
:100AD00004A10F947CA2CB010E941EF0C8CE84EA30
:100AE00090E80F945174882349F18091CA0D8823AE
:100AF00029F18091F5169091F61602969093F616CC
:100B00008093F5160E94035A6B017C016FEF87EA10
:100B10009DE00F9400A020E030E04AE754E4C701D4
:100B2000B6010F94A99A20E030E040E05FE30F9413
:100B300004A10F947CA285EA9DE07CCF85EA9DE02C
:100B40000F94EA9FBC0190E080E00F94689A20E047
:100B500030E04AE754E40F9403A20F948D4187CE0E
:100B6000D8018C91873411F00C94DB901093F61619
:100B70000093F5160E944D559093580380935703A8
:100B80008B34910509F445C60CF04BC184309105B6
:100B900009F4AAC50CF0C5C097FDCFC002970CF0B0
:100BA000A2C10E9475548C010E942A5B6091840648
:100BB0007091850680918606909187060F94689AB9
:100BC0006B017C0140900112509002126090031260
:100BD0007090041280909F069090A006A090A106AD
:100BE000B090A206A5019401C301B2010F9403A124
:100BF00020E030E048EC52E40F94A99A9B01AC014C
:100C0000C701B6010F948DA31816D4F4A301920165
:100C1000C501B4010F9403A120E030E048EC52E498
:100C20000F94A99AA70196010F9404A10F947CA296
:100C3000609384067093850680938606909387065A
:100C40008091B404882309F446C188E50E942B559D
:100C5000811141C189E50E942B5581113CC18AE572
:100C60000E942B55811137C185E40E942B558823A2
:100C700009F431C120910112309102124091031206
:100C80005091041260919F067091A0068091A10678
:100C90009091A2060F9403A16B017C012DEC3CEC1A
:100CA0004CEC5DEB0F94F9A187FF07C18091030520
:100CB00081110C941EB00F94422280919F06909156
:100CC000A006A091A106B091A20680930112909374
:100CD0000212A0930312B093041281E092E10F94E8
:100CE000C8749091030581E089270E9453BECD59B5
:100CF000DF4F0FB6F894DEBF0FBECDBFDF91CF91AF
:100D00001F910F91FF90EF90DF90CF90BF90AF9029
:100D10009F908F907F906F905F904F903F902F901B
:100D200008958531910509F4D9C0FCF48A30910504
:100D300009F423C50B9709F424C58091CB11909138
:100D4000CC118F51904F9F938F931F9287E48F9375
:100D500088E496E69F938F930F949E9E0F900F903A
:100D60000F900F900F900F90B9C08C31910509F43E
:100D70000AC54E9711F70F94422281E08093051225
:100D80000E94EE5F8C0180E090E0A8E4B4E48093E0
:100D90007A0290937B02A0937C02B0937D0243E0A1
:100DA00060E070E080E291EC0F94FB557090FD11D3
:100DB0006090FE115090FF1140900012B090F91118
:100DC000A090FA119090FB118090FC11F090F51119
:100DD000E090F611D090F711C090F8118DE695E5EE
:100DE0000E94B16C4F925F926F927F928F929F920E
:100DF000AF92BF92CF92DF92EF92FF929F938F9329
:100E000081E097E69F938F930F949E9EC8010E9466
:100E1000D45F109205120FB6F894DEBF0FBECDBF9F
:100E20005DC08835910509F459C0F4F48135910508
:100E300011F40C9421905CF48C34910509F40CC5E8
:100E40008035910509F079CF0E940D7E47C0863527
:100E5000910511F40C9425908735910509F06DCF1B
:100E600080E10E9486C63AC08C35910511F40C943D
:100E7000319074F48A35910511F40C942A908B35D5
:100E8000910509F05ACF8091EB1187600C942D9059
:100E90008236910511F40C94C8908336910509F0BF
:100EA0004CCF1092CA0D60E084EC9FE00F9400A03C
:100EB00082E00E9442690C94D7902DEC3CEC4CEC03
:100EC0005DE3C701B6010F948DA3181624F4809139
:100ED00003058111F0CEC8010E94046510925803E9
:100EE00010925703C4CC0E9475542E969FAF8EAFBC
:100EF0002E970E942A5B89E40E942B55882309F4CF
:100F0000A0C30E94035A60934F03709350038093D1
:100F10005103909352038AE40E942B55C12CD12C8B
:100F20007601882321F00E94035A6B017C01C09254
:100F30005303D0925403E0925503F0925603E0918C
:100F40005703F0915803A496FFAFEEAFA49780909B
:100F50004F0390905003A0905103B0905203A7010B
:100F60009601C501B4010F94A0A324966CAF7DAF88
:100F70008EAF9FAF249760918E0270918F02072EE3
:100F8000000C880B990B0F946A9A20917A02309189
:100F90007B0240917C0250917D020F94A99A2EE32E
:100FA00033EC4EE259E30F94A99A68AF79AF8AAF58
:100FB0009BAF80E1E5EFF1E1DE01119601900D922A
:100FC0008A95E1F7A5019401505828A739A74AA7A7
:100FD0005BA7D701C601B0588CA79DA7AEA7BFA736
:100FE00029813A814B815C8128962CAF3DAF4EAF71
:100FF0005FAF2897C501B4010F9404A162966CAF4E
:101000007DAF8EAF9FAF62978D819E81AF81B88596
:101010002C968CAF9DAFAEAFBFAF2C979C01AD01AE
:10102000C701B6010F9404A166966CAF7DAF8EAF79
:101030009FAF669729853A854B855C8560919B06B5
:1010400070919C0680919D0690919E060F9403A13D
:101050006A966CAF7DAF8EAF9FAF6A972091930673
:101060003091940640919506509196066E962CAF5D
:101070003DAF4EAF5FAF6E9762962CAD3DAD4EADBE
:101080005FAD62976E966CAD7DAD8EAD9FAD6E9788
:101090000F9403A16B017C018091970690919806B3
:1010A000A0919906B0919A06A2968CAF9DAFAEAF73
:1010B000BFAFA29766962CAD3DAD4EAD5FAD6697C6
:1010C000BC01CD010F9403A14B015C013090F604EB
:1010D0002090F7049091F8049CABA091F904ACAF78
:1010E000B091FE04B8ABA701960168A579A58AA5C1
:1010F0009BA50F94A99A2B013C01A50194016CA515
:101100007DA58EA59FA50F94A99A9B01AC01C30153
:10111000B2010F9404A12B013C01A501940168A523
:1011200079A58AA59BA50F94A99A4B015C01A701FB
:1011300096016CA57DA58EA59FA50F94A99A9B01EC
:10114000AC01C501B4010F9403A1A30192010F9456
:1011500083A16B017C0120E030E0A9010F94F9A18B
:1011600087FF0AC02BED3FE049EC50E4C701B60110
:101170000F9404A16B017C016091FF047091000544
:101180006115710509F461C290E080E00F94689ADE
:101190009B01AC016BED7FE089EC90E40F9403A21E
:1011A00024962CAD3DAD4EAD5FAD24970F94A99A1A
:1011B0005B018C016091010570910205611571055B
:1011C000E1F090E080E00F94689A20E030E040E7A2
:1011D00052E40F94A99A9B01AC0168AD79AD8AAD38
:1011E0009BAD0F9403A23B014C019501A8010F9404
:1011F000F9A187FF02C0530184014090FA04509086
:10120000FB046090FC047090FD049501A801B201FC
:10121000C3010F948DA3181684F09501A801632DC6
:10122000722D8CA99CAD0F94F9A12501380187FF7F
:1012300004C0432C522C6CA87CACA496EEADFFAD40
:10124000A497329751F42BED3FE049EC50E4C701ED
:10125000B6010F9403A16B017C016E962CAD3DADE0
:101260004EAD5FAD6E9728966CAD7DAD8EAD9FADEA
:1012700028970F94F9A1811123C0A2962CAD3DAD02
:101280004EAD5FADA2972C966CAD7DAD8EAD9FAD92
:101290002C970F94F9A1811113C020E030E0A9012F
:1012A000C701B6010F94F9A181110AC02BED3FE0EF
:1012B00049EC50E4C701B6010F9404A16B017C0115
:1012C000A701960124966CAD7DAD8EAD9FAD2497A0
:1012D0000F94A99A6A962CAD3DAD4EAD5FAD6A975D
:1012E0000F94A0A34B015C012FE632E143E85AE3DF
:1012F0000F94F9A187FD9EC19201A301C501B4011C
:101300000F9403A20F94E2A10F947CA27DAB6CAB6F
:101310006230710508F45EC12E964EAD5FAD2E971A
:10132000452B09F457C190E080E00F94689A4B0177
:101330005C01AC019B01C701B6010F9403A22B0114
:101340003C01A50194016A966CAD7DAD8EAD9FAD5B
:101350006A970F9403A228966CAF7DAF8EAF9FAFB4
:1013600028972D853E854F85588960919F067091FD
:10137000A0068091A1069091A2060F9403A1A50159
:1013800094010F9403A22C966CAF7DAF8EAF9FAFEC
:101390002C97A3019201C301B2010F94A99A6B018A
:1013A0007C01AC019B01C301B2010F94A99A20E01A
:1013B00030E040EC50E40F9403A29B01AC01C30168
:1013C000B2010F9403A16CAF7DAF8EAF9FAF20E051
:1013D00030E040E05FE3C701B6010F94A99A9B019A
:1013E000AC0160E070E080E89FE30F9403A12496D5
:1013F0006CAF7DAF8EAF9FAF249722242394312C06
:10140000D8A8DA9458A9511125C1B10190E080E023
:101410000F94689AA30192010F94A99A6B017C0121
:101420000F94FEA16CA77DA78EA79FA7C701B60149
:101430000F94C4A44B015C01C0904F03D0905003A3
:10144000E0905103F0905203F7FAF094F7F8F0941B
:101450008091530390915403A0915503B09156038A
:1014600088AB99ABAAABBBABA70196016CA57DA5D8
:101470008EA59FA50F94A99A68A779A78AA79BA76D
:1014800028A939A94AA95BA9C501B4010F94A99A51
:101490009B01AC0168A579A58AA59BA50F9404A121
:1014A00068A779A78AA79BA7A7019601C501B401E0
:1014B0000F94A99A6B017C0128A939A94AA95BA9B3
:1014C0006CA57DA58EA59FA50F94A99A9B01AC0143
:1014D000C701B6010F9403A16CA77DA78EA79FA794
:1014E0009091FE0498AB28A539A54AA55BA5629604
:1014F0006CAD7DAD8EAD9FAD62970F9404A16983F5
:101500007A838B839C832CA53DA54EA55FA566960B
:101510006CAD7DAD8EAD9FAD66970F9404A16D83CC
:101520007E838F83988728962CAD3DAD4EAD5FAD01
:10153000289769857A858B859C850F9404A1698796
:101540007A878B879C872C962CAD3DAD4EAD5FADD9
:101550002C976D857E858F8598890F9404A16D8762
:101560007E878F87988BCE0101960E94C5642E9648
:10157000AEADBFAD2E972A163B06F8F0E984FA848B
:101580000B851C852D813E814F81588569817A812B
:101590008B819C813F922F92E5EFF1E1FF93EF93D6
:1015A00088AC99ACAAACBBACFE013D966F010F9420
:1015B00022750F900F900F900F908091AC0D8111BC
:1015C00039C0FFEF2F1A3F0A2CA93DA92215330578
:1015D00009F016CF83E996E00E94C564E0909B066F
:1015E000F0909C0600919D0610919E062091970612
:1015F000309198064091990650919A066091930611
:101600007091940680919506909196061F921F9274
:10161000E5EFF1E1FF93EF9388AC99ACAAACBBACDA
:10162000EFE9CE2EE6E0DE2E0F9422750F900F909C
:101630000F900F900E94AC548AE493E00F94A11194
:101640004DCC60E070E0CB015ECCA32CB22C0CA999
:101650001CADB0CD28A539A54AA55BA56CAD7DAD67
:101660008EAD9FAD0F94A99A4B015C012CA53DA5B1
:101670004EA55FA524966CAD7DAD8EAD9FAD249734
:101680000F94A99A9B01AC01C501B4010F9404A168
:101690007B018C0128A539A54AA55BA524966CADD4
:1016A0007DAD8EAD9FAD24970F94A99A4B015C013F
:1016B0002CA53DA54EA55FA56CAD7DAD8EAD9FADB6
:1016C0000F94A99A9B01AC01C501B4010F9403A129
:1016D00068A779A78AA79BA7D8AAC701D8018CA712
:1016E0009DA7AEA7BFA7FFCE80E50E942B55C12CBA
:1016F000D12C7601882331F00E94035A0F947CA2EA
:101700006B017C0183E50E942B55882361F00E94C8
:10171000035A20E030E04AE754E40F94A99A0F946A
:101720007CA26B017C01C114D104E104F10441F0FD
:101730008091C706873021F08DE197E60E9465E62B
:101740000F9442220F94740FC60ED71EE81EF91E86
:101750008AE493E00F94A1110F94740F6C157D052A
:101760008E059F0508F0BACB0F945B3280E00E9493
:10177000017A80E00E944269EFCF81E00E9453BE6F
:10178000ADCB80E0FBCF88E50E942B55382E412C55
:10179000512C3201882321F00E9493552B013C01EA
:1017A00089E50E942B55282E882371F10E949355BC
:1017B0006CA77DA78EA79FA78AE50E942B55D82EE0
:1017C000812C912C5401882321F00E9493554B01C8
:1017D0005C0187E50E942B5588A78F93CD2CECA444
:1017E000FDA40EA51FA5222DB301A201832D0E94E9
:1017F00073670F90311072CB211070CB38A5311167
:101800006DCBD1106BCB20CB1CA61DA61EA61FA690
:10181000D3CF08E210E098EFE92E96E6F92E602F7C
:1018200070E090E080E00F94689A0E9404569F93C5
:101830008F937F936F931F930F93FF92EF920F9469
:101840009E9E0F5F1F4F0FB6F894DEBF0FBECDBF39
:101850000F36110521F742CB0F94B214811105C048
:1018600080E990E80E94537239CB82E00E9455D8FB
:10187000811107C08AED99E30E94B16C0F94470B68
:101880002DCB8091A306882341F08091A406882364
:1018900021F0D090A506D11008C081E08093E61118
:1018A00082E198E60F94574319CB81E999E30E94AE
:1018B000B16C0F94470B89ED90E50E94B16C41E04B
:1018C00060E00F94E02D81116EC080E090E0A0EA0E
:1018D000B0E48093FD119093FE11A093FF11B0939B
:1018E000001260E070E088E492E40F94708480E07D
:1018F00090E0A8E4B2E48093FD119093FE11A093D0
:10190000FF11B093001280E090E0A4E3B3E4809371
:10191000F9119093FA11A093FB11B093FC1160E0C0
:1019200070E088E492E40F9470840F9442228FEA6E
:1019300090E50E94B16C0F94470BE0E5F8E88591C3
:101940009591A591B4918093F9119093FA11A09378
:10195000FB11B093FC11ECE4F8E885919591A59109
:10196000B4918093F5119093F611A093F711B09371
:10197000F81160E070E088E492E40F9470840F94B2
:10198000422281E08F93812C912C5401CC24C3946A
:10199000E12CF12C870120E040E050E0BA0180E02A
:1019A0000E9473670F9020E030E04CE052E46091B9
:1019B0008E0670918F0680919006909191060F94FB
:1019C0008DA318160CF076C08091CA0D811172C0DB
:1019D00080E090E0A8ECB2E48093FD119093FE11BA
:1019E000A093FF11B093001260E070E088E492E4ED
:1019F0000F9470840F945F1219821A821B821C82CA
:101A00001D82CE0101960F94A11183E2F82E0FE101
:101A10001EE720E030E04CE052E460918E067091C9
:101A20008F0680919006909191060F948DA31816C1
:101A3000C4F583E499E30E94B16C0F94C00A42E8B4
:101A400064E080E00E949B691F92FF9260918E0685
:101A500070918F0680919006909191060F9475A2D7
:101A60007F936F931F930F930E94546981E80E94A4
:101A70006A6988EE93E00E94487C0E94687040E0AA
:101A800053E567E070E0CE0101960F94E20F0F90EE
:101A90000F900F900F900F900F90882309F4B9CFFB
:101AA000D12C81E00E94C069D11004C080E00F9465
:101AB000D80B14CA0F94422281E0809305120E9431
:101AC000C06982E790E80E94537280908E069090E1
:101AD0008F06A0909006B090910620E030E040EA9A
:101AE00050E4C501B4010F9403A20F9475A225E040
:101AF000269FA001279F500D1124BA01550F880B76
:101B0000990B0F946A9A1B017C0120E030E04CE0B5
:101B100052E40F94F9A187FF06C0212C312C1CE060
:101B2000E12E02E4F02E222D332D4E2D5F2DC50126
:101B3000B4010F948DA3181664F420E030E040EA5D
:101B400050E4622D732D8E2D9F2D0F9404A11B0147
:101B50007C01FF92EF923F922F928FED96E69F933A
:101B60008F930F949E9E20E030E040EF51E4622D71
:101B7000732D8E2D9F2D0F9403A120E030E04CE8B3
:101B800052E40F9404A10F9475A27093EE11609328
:101B9000ED1184E08093C70681E08093AC0385EE6D
:101BA0009AE30E94B16C0E9465E680E090E0A0EAB2
:101BB000B0E48093FD119093FE11A093FF11B093B8
:101BC000001260E070E088E492E40F94708480E09A
:101BD00090E0A0EAB1E48093F5119093F611A09300
:101BE000F711B093F81180E090E0A0E7B2E48093A1
:101BF000F9119093FA11A093FB11B093FC1160E0DE
:101C000070E088E492E40F9470848AE999E9A9E18C
:101C1000BEE38093FD119093FE11A093FF11B0934A
:101C2000001260E070E088E492E40F9470840F94F6
:101C300042220F900F900F900F900F900F902091D5
:101C40008E0630918F064091900650919106622D3C
:101C5000732D8E2D9F2D0F948DA318163CF488EEB6
:101C600093E00E94487C0E946870E9CF60E086EAB9
:101C70009FE00F9400A080E090E0A0EAB0E48093A1
:101C8000FD119093FE11A093FF11B093001260E03C
:101C900070E088E492E40F947084ECE4F8E88591B5
:101CA0009591A591B4918093F5119093F611A0931D
:101CB000F711B093F811E0E5F8E885919591A591B9
:101CC000B4918093F9119093FA11A093FB11B09302
:101CD000FC1160E070E088E492E40F9470840F944B
:101CE000422243E060E070E080E89FEB0F94FB55F8
:101CF000811105C00F94D80B10920512EFC8909176
:101D0000FD1198A7A091FE11ACA7B091FF11B8AB3F
:101D1000E0910012E8AFEF93BF93AF939F9382EDF2
:101D200096E69F938F930F949E9E0F900F900F9027
:101D30000F900F900F90AEEA8A2EAFE09A2EB3E28A
:101D4000CB2ED12C0FEF1FEFB6010D2C000C880B02
:101D5000990B0F946A9A2B013C01DF92CF92C80134
:101D600002969F938F9326E936E63F932F930F9425
:101D70009E9E58015FEFA51AB50A0F900F900F9025
:101D80000F900F900F9011F40C942CB070E060E065
:101D9000C4010F941EA0A3019201622D732D8E2DFC
:101DA0009F2D0F94F9A1181644F485E0A816B104EC
:101DB00011F00C9438B005E010E0580197E2A91A30
:101DC00098EFB90AAA0CBB1C85E0809F1001819F87
:101DD000300C11240D5F1F4FEAE94E2EE9E95E2E0B
:101DE000E9E16E2EEEE37E2EFDE58F2EF6E69F2EC8
:101DF000C801029705970CF0D4C0B101635D7F4F15
:101E0000072E000C880B990B0F946A9A6B017C01CA
:101E10001F930F93A9E8B6E6BF93AF930F949E9ECE
:101E20000093AC0320E030E040EF51E4C701B6017D
:101E30000F9403A120E030E040E251E40F94A99A0E
:101E400020E030E040EA50E40F9403A220E030E0CC
:101E500048E452E40F9404A10F9475A27093EE111C
:101E60006093ED1180E090E0A0EAB0E48093FD1172
:101E70009093FE11A093FF11B093001260E070E008
:101E800088E492E40F94708420E030E040EA51E46A
:101E90002093F5113093F6114093F7115093F811F8
:101EA00080E090E0A0E7B2E48093F9119093FA11FA
:101EB000A093FB11B093FC1160E070E088E492E421
:101EC0000F9470844092FD115092FE116092FF11A8
:101ED0007092001260E070E088E492E40F947084E5
:101EE0000F9442220F900F900F900F9020918E062A
:101EF00030918F064091900650919106C701B6012E
:101F00000F948DA318163CF488EE93E00E94487C51
:101F10000E946870EBCF80E090E0A0EAB0E480938C
:101F2000FD119093FE11A093FF11B093001260E099
:101F300070E088E492E40F947084ECE4F8E8859112
:101F40009591A591B4918093F5119093F611A0937A
:101F5000F711B093F811E0E5F8E885919591A59116
:101F6000B4918093F9119093FA11A093FB11B0935F
:101F7000FC1160E070E088E492E40F9470840F94A8
:101F8000422243E060E070E080E89FEB0F94FB5555
:101F900095E0290E311C0F5F1F4F811104C00F9473
:101FA000D80B81E0A7CE78A56CA598A988AD272F7E
:101FB000362F492F582F6091FD117091FE1180919D
:101FC000FF11909100120F9403A1F62EE72ED82E48
:101FD000C92E20913E0430913F044091400450911D
:101FE0004104D701F6016B2F7A2F8F2F9E2F0F946C
:101FF000A99A0F9475A26CAB7DAB8EAB9FABCF92C1
:10200000DF92EF92FF92809191068F9380919006DC
:102010008F9380918F068F9380918E068F939F92DE
:102020008F920F949E9E6CA97DA9C5010F941EA04E
